:100000000C9474280C94A5280C94A5280C94A5286D
:100010000C94A5280C94A5280C94A5280C94A5282C
:100020000C94A5280C94A5280C94A5280C94A5281C
:100030000C94A5280C948AD90C94A5280C94A52876
:100040000C94A5280C941A7B0C94A5280C94A52834
:100050000C94A5280C94A5280C9481600C94EDD4E4
:100060000C94A5280C946C880C94A5280C94A528B5
:100070000C94A5280C94A5280C94A5280C94A528CC
:100080000C94A5280C94A5280C94A5280C94A528BC
:100090000C94A5280C94A5280C94A5280C94A528AC
:1000A0000C94A5280C94A5280C94A5280C94A5289C
:1000B0000C94A5280C94A5280C94A5280C94A5288C
:1000C0000C94A5280C94A5280C94A5280C94A5287C
:1000D0000C94A5280C94A5280C94A5280C94A5286C
:1000E0000C94A5280D5A105AFF59035A095A475A19
:1000F000145A185A1E5A225A265A2C5A305A345A0E
:10010000475A3A5A3E5A425AFF5A045B095B135BFC
:100110001D5B965B275B2F5B375B415B4B5B555BE6
:10012000645B6E5B965B785B825B8C5B084AD73B5B
:100130003BCE016E84BCBFFDC12F3D6C74319ABDB6
:1001400056833DDA3D00C77F11BED9E4BB4C3E91DA
:100150006BAAAABE000000803F05A84CCDB2D44EC9
:10016000B93836A9020C50B9918688083CA6AAAACB
:100170002ABE000000803F004E414E494E4954596E
:10018000494E46CDCCCC3D0AD7233C17B7D1387762
:10019000CC2B329595E6241FB14F0A000020410078
:1001A00000C84200401C4620BCBE4CCA1B0E5AAEC2
:1001B000C59D74434F4D4D554E49434154494F4E93
:1001C0000044525952554E004552524F5253004925
:1001D0004E464F004543484F0020746F6F206C6FB0
:1001E0006E6720657874727573696F6E20707265C2
:1001F00076656E7465640A0020636F6C64206578B0
:1002000074727573696F6E2070726576656E746551
:10021000640A0047322F47332062616420706172A4
:10022000616D65746572730A00536C6565702E2E7E
:100230002E00205A3A200020593A200042656420BE
:10024000583A20004368656170334420563330309B
:100250002072656164792E00526573756D696E67F1
:10026000207072696E7400436C69636B20746F2038
:10027000726573756D652E2E2E004E6F206D6F7634
:10028000652E00456E642066696C65206C69737428
:100290000A00426567696E2066696C65206C697347
:1002A000740A005344207072696E74696E6720622C
:1002B00079746520004E6F74205344207072696E0B
:1002C00074696E670A0046696C652064656C6574C4
:1002D00065643A0044656C6574696F6E2066616997
:1002E0006C65642C2046696C653A20006F70656E01
:1002F000206661696C65642C2046696C653A200053
:100300002569730025696D202569730025696820BA
:1003100025696D2025697300256964202569682099
:1003200025696D2025697300256979202569642078
:100330002569682025696D20256973005072696EF2
:10034000742074696D653A200050726F746563742F
:1003500065642050696E0A004525692025730043B5
:1003600068656170334420563330302072656164B3
:10037000792E00D401CF01C801C101B3016F6666B7
:100380000044454255473A004B494C4C45442E20C9
:10039000004D3131332053006F6B00486561746943
:1003A0006E6720646F6E652E003F0A0020573A008A
:1003B00045256920257300436865617033442056E4
:1003C0003330302072656164792E004265642064A8
:1003D0006F6E652E003F0A0020573A004265642088
:1003E00048656174696E672E0043686561703344C7
:1003F0002056333030204F66662E00563330302082
:100400004C312050494420423A312054303A352072
:1004100054313A30204649524D574152455F4E4182
:100420004D453A4D61726C696E20312E312E30206F
:10043000284769746875622920534F555243455FB8
:10044000434F44455F55524C3A68747470733A2F69
:100450002F6769746875622E636F6D2F4D61726CC2
:10046000696E4669726D776172652F4D61726C6954
:100470006E2050524F544F434F4C5F564552534994
:100480004F4E3A312E30204D414348494E455F543E
:100490005950453A436865617033442056333030D3
:1004A0002045585452554445525F434F554E543A97
:1004B0003120555549443A63656465326132662D91
:1004C000343161322D343734382D396231322D6375
:1004D00035356336326633363766660A007A5F6DC5
:1004E000696E3A2000795F6D696E3A2000785F6D21
:1004F000696E3A20005265706F7274696E6720658C
:100500006E6473746F70207374617475730A004D38
:1005100031343520533C696E6465783E206F7574C4
:10052000206F662072616E67652028302D31290AA0
:100530000053657474696E672054726176656C202F
:10054000416363656C65726174696F6E3A20005334
:10055000657474696E6720526574726163742041BA
:100560006363656C65726174696F6E3A20005365F0
:100570007474696E67205072696E7420416363659C
:100580006C65726174696F6E3A20005365747469AA
:100590006E67205072696E7420616E6420547261BF
:1005A00076656C20416363656C65726174696F6E1A
:1005B0003A2000205A00205900580020204D617830
:1005C0003A2000205A00205900580020204D696E22
:1005D0003A20004F6E20004F666600536F6674200D
:1005E000656E6473746F70733A200020643A002063
:1005F000693A0020703A004F666673657473206133
:1006000070706C696564004572723A20546F6F2097
:100610006661722100546F6F206661722066726F8E
:100620006D207265666572656E636520706F696EB8
:10063000740A00454550524F4D2064697361626CE5
:1006400065640A003A20007A5F6D696E3A20202DB9
:100650003230207A5F6D61783A20203230005A20A3
:100660004F666673657420004E6F2063617365206A
:100670006C696768740A004163746976652045781F
:100680007472756465723A2000556E6B6E6F776E8A
:1006900020636F6D6D616E643A2022004861726460
:1006A000636F6465642044656661756C742053658E
:1006B0007474696E6773204C6F616465640A00200E
:1006C000204D383531205A005A2D50726F62652006
:1006D0004F666673657420286D6D293A0A002044C0
:1006E0000020490020204D333034205000204400A9
:1006F00020490020204D3330312050005049442003
:1007000073657474696E67733A0A0020460020426C
:100710000020480020204D3134352053004D6174B5
:10072000657269616C2068656174757020706172B2
:10073000616D65746572733A0A00205A0020590091
:1007400020204D323036205800486F6D65206F668E
:10075000667365743A0A00204500205A002059004B
:1007600020580020420020540020204D32303520F7
:100770005300416476616E6365643A20533C6D6951
:100780006E5F66656564726174653E20543C6D6998
:100790006E5F74726176656C5F66656564726174C4
:1007A000653E20423C6D696E5F7365676D656E7472
:1007B0005F74696D655F6D733E20583C6D61785F55
:1007C00078795F6A65726B3E205A3C6D61785F7A1A
:1007D0005F6A65726B3E20453C6D61785F655F6A5C
:1007E00065726B3E0A0020540020520020204D32DA
:1007F0003034205000416363656C65726174696FC9
:100800006E2028756E6974732F7332293A20503C1C
:100810007072696E745F616363656C3E20523C72F6
:100820006574726163745F616363656C3E20543C00
:1008300074726176656C5F616363656C3E0A00206B
:100840004500205A0020590020204D3230312058D8
:10085000004D6178696D756D20416363656C6572EB
:100860006174696F6E2028756E6974732F733229F5
:100870003A0A00204500205A0020590020204D321D
:1008800030332058004D6178696D756D206665655F
:100890006472617465732028756E6974732F73298F
:1008A0003A0A00204500205A0020590020204D39E6
:1008B0003220580053746570732070657220756E15
:1008C00069743A0A0020204D3230302044300A004A
:1008D00020204D3230302044002044697361626C26
:1008E00065640A0046696C616D656E742073657499
:1008F00074696E67733A002020473231203B2055DF
:100900006E69747320696E206D6D0A0A0025753A50
:100910002530327500253032753A25303275002584
:10092000756420253032753A25303275005A0059E9
:100930000058000920000000000000000000000036
:1009400000007FFFE0000000000000000000000049
:10095000007000E000000000000000000000000047
:1009600061F860000000000000000000000000418D
:10097000F82000000000000000000000000040F02F
:100980002000000000000000000000000040602087
:100990000000000000000000000000005801A07FDF
:1009A00080000000000000004104005C63A0FFC064
:1009B000000000000000002082005EF7A0FFC000E1
:1009C0000000000000002082005EF7A0FFC00000D1
:1009D00000000000004104005C63A07F8000000074
:1009E000000000008208005801A07F800000000085
:1009F000000001041000406020FFC0000000000063
:100A0000000104100040F020FFC0000000000000C2
:100A10000082080041F820FFC00000000000000034
:100A200041040061F8603F00000000000000000089
:100A300000007000E01E0000000000000001FFFF49
:100A4000807FFFE00C0000000000000001FFFF803D
:100A50000000000000000000000000000000007F17
:100A6000FFE0000000000000000000000000700037
:100A7000E0000000000000000000000000630C60C7
:100A8000000000000000000000000000470E2000F1
:100A900000000000000000000000004F0F200000D8
:100AA000000000000000000000005F0FA000000038
:100AB0000000000000000000005E07A07F80000032
:100AC0000000000000410400406020FFC000000062
:100AD0000000000020820040F020FFC00000000065
:100AE00000000020820040F020FFC0000000000055
:100AF00000004104004060207F80000000000000F2
:100B0000008208005E07A07F800000000000000156
:100B10000410005F0FA0FFC00000000000000104EF
:100B200010004F0F20FFC0000000000000008208EE
:100B300000470E20FFC0000000000000004104003C
:100B4000630C603F00000000000000000000007027
:100B500000E01E0000000000000001FFFF807FFF9A
:100B6000E00C0000000000000001FFFF800000001A
:100B70005072696E742061626F72746564004E6FAA
:100B80002053442063617264005072696E74206661
:100B9000726F6D2053440053746F70207072696ED1
:100BA0007400526573756D65207072696E740050C3
:100BB00061757365207072696E7400436F6E747234
:100BC0006F6C00507265706172650054756E6500DF
:100BD000496E666F2073637265656E0000060900DA
:100BE000FE000000000001090008FE0000050808E2
:100BF00006000040F0C888889878100508080600AC
:100C000000C0F88888888888F80505050600012056
:100C100030F830200508080600002070F820202059
:100C200020E00509090600FF2070A8A8B888887090
:100C3000200509090600FFE080C0B0A82830282858
:100C40000509090600FFF8A88888888888A8F8059B
:100C50000A0A0600FE205050505088A8A888700349
:100C6000030306000340A0400000210024002700E9
:100C70002A002D00300033000101000004010701AB
:100C80000A0100002200250028002B002E00310060
:100C9000340002010000050108010B0100002000E2
:100CA0002300260029002C002F0032000001000044
:100CB00003010601090105050505070508080808DF
:100CC000020202020A0A08080404040401010101E4
:100CD00001010101030303030303030304070707DF
:100CE0000C0C0C0C0C0C0C0C020202020606060684
:100CF000060606060B0B0B0B0B0B0B0B0102102051
:100D00002008081020401020408002010201080441
:100D100002010102040810204080804020100804D5
:100D2000020180040201804020100804020108042E
:100D30000201010204081020408001020408102072
:100D4000408000000A0B02090C0D0E080703040185
:100D50000000000000000000000000000000000093
:100D60000000000000000000000000000000121160
:100D70001000000000000000000000000000000063
:100D800000000000000000004B494C4C45442E2060
:100D900000202D20496E76616C696420657874723C
:100DA00075646572206E756D62657220210A00207F
:100DB00020506C616E6E657242756666657242792E
:100DC0007465733A20002046726565204D656D6F2D
:100DD00072793A2000436F6D70696C65643A204DFA
:100DE000617920313720323031370A00207C2041B0
:100DF0007574686F723A20286E6F6E652C2064657A
:100E00006661756C7420636F6E666967290A0032CB
:100E10003031372D30352D30342031323A303000FA
:100E2000204C61737420557064617465643A2000CD
:100E3000312E312E300A004D61726C696E002053E4
:100E40006F6674776172652052657365740A00205D
:100E50005761746368646F672052657365740A0034
:100E60002042726F776E206F7574205265736574BF
:100E70000A002045787465726E616C205265736556
:100E8000740A00506F77657255700A00737461724E
:100E9000740A006572726F722077726974696E6786
:100EA00020746F2066696C650A00456E6473746F08
:100EB000707320256320256320256320256300208F
:100EC0005A3A0020593A0020583A00656E6473740B
:100ED0006F7073206869743A2000446F6E652073E8
:100EE0006176696E672066696C652E0A004D32393D
:100EF000001000C90210012C0140012201700118EC
:100F000001B0010E01F00104015002FA00B002F03C
:100F1000003003E600D003DC009004D2007005C866
:100F200000A006BE000008B400B009AA00D00BA0C3
:100F300000600E960060118C000015820020197868
:100F400000C01D6E00A0226400B0275A00902C50F3
:100F50000000314600E0343C0010383200903A285E
:100F600000603C1E00A03D1400803E0A00203F00AF
:100F7000004572723A204D494E54454D502042452D
:100F800044004572723A204D494E54454D50004D33
:100F9000494E54454D5020747269676765726564A7
:100FA000004572723A204D415854454D50204245FB
:100FB00044004572723A204D415854454D50004D01
:100FC000415854454D502074726967676572656475
:100FD000001FFFFFFFFFFFFF600000000001FF4058
:100FE0000000000000FF8000000000007F83CF00B1
:100FF000000C303F87FF80000C301F867980000C8A
:10100000000F8C30C7838C30E78C30CFC7CC31F3E6
:101010008C30DCECEC33B98C30D86C6C33198C3000
:10102000D06C0C33198C30D86C0C33198C30DC6CD0
:101030000E3B198C30CF7C079F198C30C77C038FF7
:101040001940000000000002600000000000061FC0
:10105000FFFFFFFFFFF800600000000000600000DD
:10106000E00000E0000001F80000000001F80003CB
:10107000F80003F8000007FE0000000007FE000F64
:10108000FE000F1E00001F0F81C000381F0F803FA1
:101090000F803E0F80007C03E1C000387C03E0FC41
:1010A00003E0F803E000F000F1C00038F000F1F0D8
:1010B00000F1E000F000C00071C00038C00071C055
:1010C0000071C0007000C00001C00038C003E1C062
:1010D0000031C0003000C00001C00038C00F81C026
:1010E0000031C0003000C00001FFFFF8C07E01FFEA
:1010F000FC31C0003000C00001FFFFF8C1F001FF6B
:10110000FC31C0003000C00001FFFFF8C7C001FF84
:10111000FC31C0003000C00001C00038FF0001C039
:101120000031C0003000C00001C00038FC0001C028
:101130000031C0003000C00031C00038E00031C0D4
:101140000031C0003000E000F1C00038E000F1C024
:101150000031C00070007C03E1C000387C03E1C0B6
:101160000031F001E0001F0F81C000381F0F81C067
:101170000031FC07C00007FE0000000007FE000071
:101180000001CF0F000001F80000000001F800008E
:101190000001C3FC000000600000000000600000CF
:1011A0000001C0F00000000000000000000000008E
:1011B00000000060000000000000000000000000CF
:1011C000000000000000000000000000000000001F
:1011D000000000000000000000000000000000000F
:1011E000000E00001F0300000000000000000000CF
:1011F000003F80007FC300000000000000000000EE
:1012000000FFE001FBF30000000000000000000010
:1012100003E0F807E0FF000000000000000000000D
:101220000F803E1F8E3F0000000000000000000005
:101230000E001F9E3F8F0000000000000000000015
:1012400000001F98FFE30000000000000000000005
:1012500000007E19FFF30000000000000000000005
:101260000001F819FFF3000000000000000000007A
:10127000000FE019FFF30000000000000000000074
:10128000001F8019FFF300000000000000000000B4
:101290000007E019FFF3000000000000000000005C
:1012A0000001FC19FFF30000000000000000000036
:1012B00000003F19FFF300000000000000000000E4
:1012C0000C000F9C7FC70000000000000000000021
:1012D0000F001F9F1F1F0000000000000000000003
:1012E0000FC07E0FC07E0000000000000000000064
:1012F00003F1F803F1F80000000000000000000016
:1013000000FFE000FFE0000000000000000000001F
:10131000003F80003F80000000000000000000004F
:10132000000E00000E0000000000000000000000A1
:1013300000000000000000000000000000000000AD
:10134000000000000000000000000000000000009D
:10135000000000000000000000000000000000008D
:10136000000000000000000000000000000000007D
:1030500000000000000043616E6E6F7420656E74A6
:103060006572207375626469723A2000022E2E0028
:103070004D61696E00436172642072656D6F7665A3
:1030800064004361726420696E73657274656400E4
:10309000466C6F7700466C6F770046616E207370E8
:1030A0006565640046616E20737065656400426505
:1030B0006400426564004E6F7A7A6C65004E6F7AE8
:1030C0007A6C6500537065656400537065656400D3
:1030D0004D61696E005072656865617420504C41A5
:1030E00020426564005072656865617420504C41EF
:1030F00020456E64005072656865617420504C41D3
:103100000050726570617265005072656865617427
:1031100020414253204265640050726568656174C5
:103120002041425320456E640050726568656174A9
:10313000204142530050726570617265004D343217
:1031400038005072656865617420414253005072C6
:10315000656865617420504C4100436F6F6C646F0B
:10316000776E004D38340044697361626C6520737A
:10317000746570706572730053657420686F6D6557
:10318000206F66667365747300473238004175744A
:103190006F20686F6D65004D6F766520617869738B
:1031A000004D61696E004D6F76652058004D6F7659
:1031B000652059004D6F7665205A00457874727508
:1031C000646572004D6F766520302E316D6D004D57
:1031D0006F766520316D6D004D6F76652031306DF5
:1031E0006D004D6F76652061786973004578747263
:1031F00075646572004D6F7665205A004D6F766577
:103200002059004D6F766520580053442063617249
:1032100064206F6B0A006F70656E526F6F7420666A
:1032200061696C65640A00766F6C756D652E696EF8
:103230006974206661696C65640A00534420696E94
:103240006974206661696C0A006175746F25692E66
:1032500067004D3234004D323320257300577269B8
:1032600074696E6720746F2066696C653A20006F20
:1032700070656E206661696C65642C2046696C65BA
:103280003A20006F70656E206661696C65642C2061
:1032900046696C653A200046696C652073656C650B
:1032A000637465640A002053697A653A20004669B0
:1032B0006C65206F70656E65643A20006F70656E96
:1032C000206661696C65642C2046696C653A200053
:1032D0002066696C653A20004E6F772000222070CE
:1032E0006F73002220706172656E743A220053552C
:1032F00042524F5554494E452043414C4C20746135
:10330000726765743A22004B494C4C45442E2000AC
:10331000747279696E6720746F2063616C6C2073BE
:1033200075622D67636F64652066696C65732077CD
:1033300069746820746F6F206D616E79206C65769A
:10334000656C732E204D4158206C6576656C206944
:10335000733A004572726F723A0024F4D43050C34D
:103360008E20C2A24017828B7011127A910D816C4F
:10337000D90AA861E108C7586607615143061E4B88
:103380005D05C145A7041A411104093D980371392F
:1033900031034036DB0265339102D4305402802E73
:1033A0001D02632CEE01752AC501B028A00110276B
:1033B00081018F2564012B244B01E0223401AC21D3
:1033C0001F018D200D01801FFC00841EED00971D44
:1033D000DF00B81CD200E61BC600201BBC00641A2C
:1033E000B200B219A8000A19A0006A189900D117F2
:1033F000910040178B00B516840031167E00B3157E
:1034000079003A157300C7146F0058146A00EE1360
:1034100066008813630025135E00C7125B006C1200
:10342000570015125400C111510070114F002111A5
:103430004B00D61049008D10470046104400021082
:103440004200C00F4000800F3E00420F3C00060FBC
:103450003B00CB0E3800930E37005C0E3500270E74
:103460003400F30D3200C10D3100900D3000600DBD
:103470002E00320D2D00050D2C00D90C2B00AE0CAA
:103480002900850C29005C0C2700350C27000E0C48
:103490002600E80B2400C40B2400A00B23007D0BA6
:1034A00023005A0B2100390B2100180B2000F80AC9
:1034B0001F00D90A1E00BB0A1E009D0A1D00800ABB
:1034C0001D00630A1C00470A1B002C0A1B00110A7E
:1034D0001A00F7091A00DD091900C4091900AB091F
:1034E0001900920917007B091800630917004C099D
:1034F000160036091600200916000A091500F508FD
:103500001500E0081400CC081400B8081400A40842
:103510001400900813007D0812006B08130058086F
:103520001200460812003408110023081100120886
:10353000110001081100F0071000E0071000D0078B
:103540001000C0071000B0070F00A107100091077E
:103550000E0083070F0074070F0065070E00570762
:103560000E0049070E003B070D002E070E00200736
:103570000D0013070D0006070D00F9060C00ED06FF
:103580000D00E0060C00D4060C00C8060C00BC06BA
:103590000C00B0060C00A4060B0099060C008D066A
:1035A0000B0082060B0077060B006C060B00610611
:1035B0000A0057060B004C060A0042060A003806AD
:1035C0000A002E060A0024060A001A060A0010063F
:1035D000090007060A00FD050900F4050900EB05CE
:1035E0000900E2050900D9050900D0050900C70551
:1035F0000900BE050900B5050800AD050800A505D0
:1036000009009C050800940508008C050800840545
:1036100008007C050800740508006C0507006505B6
:1036200008005D050700560508004E050700470520
:1036300007004005080038050700310507002A0586
:103640000700230507001C050600160507000F05E7
:1036500007000805060002050700FB040600F50444
:103660000700EE040600E8040600E2040700DB049D
:103670000600D5040600CF040600C9040600C304F2
:103680000600BD040600B7040600B1040500AC0442
:103690000600A6040600A00405009B04060095048D
:1036A0000500900406008A040500850405008004D6
:1036B00006007A04050075040500700405006B041B
:1036C000050066040500610405005C04050057045C
:1036D0000500520405004D0405004804050043049C
:1036E00005003E0404003A040500350405003004DA
:1036F00004002C04050027040400230405001E0414
:1037000004001A04040016040500110404000D044A
:103710000400090405000404040000040400FC0380
:103720000400F8030400F4030400F0030400EC03B5
:103730000400E8030400E4030400E0030400DC03E5
:103740000400D8030400D4030400D0030400CC0315
:103750000400C8030300C503030024F404D9201B9C
:10376000C40C5C0E9804C4095F0265077101F4057E
:10377000F900FB04B30048048700C1036900580343
:10378000550003034500BE023A0084023100530293
:103790002A002902250004022000E4011C00C801BF
:1037A0001900AF0117009801140084011300710182
:1037B00010006101100051010E0043010D0036019F
:1037C0000B002B010B0020010B00150109000C015F
:1037D000090003010800FB000800F3000800EB00EB
:1037E0000700E4000600DE000600D8000600D20054
:1037F0000600CC000500C7000500C2000500BD00A2
:103800000400B9000400B5000400B1000400AD00DC
:103810000400A9000400A5000300A20003009F000B
:1038200004009B0003009800030095000200930031
:103830000300900003008D0002008B00030088004D
:1038400002008600020084000300810002007F0065
:1038500002007D0002007B00020079000200770078
:103860000100760002007400020072000100710085
:1038700002006F0002006D0001006C0002006A008F
:103880000100690002006700010066000100650098
:10389000010064000200620001006100010060009C
:1038A00001005F0002005D0001005C0001005B00A0
:1038B00001005A00010059000100580001005700A2
:1038C00001005600010055000100540001005300A2
:1038D000000053000100520001005100010050009F
:1038E00001004F0001004E0000004E0001004D009D
:1038F00001004C0001004B0000004B0001004A0099
:103900000100490001004800000048000100470094
:10391000010046000000460001004500000045008F
:103920000100440001004300000043000100420088
:103930000000420001004100000041000100400081
:1039400001003F0000003F0001003E0000003E007B
:1039500001003D0000003D0001003C0000003C0073
:1039600000003C0001003B0000003B0001003A0069
:1039700000003A0001003900000039000100380061
:103980000000380000003800010037000000370058
:10399000010036000000360000003600010035004E
:1039A0000000350000003500010034000000340044
:1039B0000000340001003300000033000000330039
:1039C000010032000000320000003200010031002E
:1039D0000000310000003100010030000000300024
:1039E0000000300001002F0000002F0000002F0019
:1039F00000002F0001002E0000002E0000002E000D
:103A000001002D0000002D0000002D0000002D0001
:103A100001002C0000002C0000002C0000002C00F5
:103A200001002B0000002B0000002B0000002B00E9
:103A300001002A0000002A0000002A0000002A00DD
:103A400001002900000029000000290000002900D1
:103A500000002900010028000000280000002800C4
:103A600000002800000028000100270000002700B7
:103A700000002700000027000000270001002600AA
:103A8000000026000000260000002600000026009E
:103A90000100250000002500000025000000250091
:103AA0000000250000002500010024000000240083
:103AB0000000240000002400000024000100230076
:103AC000000023000000230000002300000023006A
:103AD000000023000000230001002200000022005B
:103AE000000022000000220000002200000022004E
:103AF0000100210000002100000021000000210041
:103B00000000210000002100000021000100200031
:103B10000000200000002000000020000000200025
:103B200000002000000020000000200001001F0015
:103B300000001F0000001F0000001F0000001F0009
:103B400000001F0000001F0001001E0000001E00FA
:103B500000001E0000001E0000004D3834205820D8
:103B600059205A204500526573656E643A20006FF3
:103B70006B00627573793A207061757365642066B5
:103B80006F7220696E7075740A00627573793A20DD
:103B900070617573656420666F7220757365720A53
:103BA00000627573793A2070726F63657373696E22
:103BB000670A004B494C4C45442E20004B494C4C65
:103BC00020636175736564206279204B494C4C20F9
:103BD000627574746F6E2F70696E0A004B494C4C9D
:103BE00045442E20004B494C4C206361757365643D
:103BF00020627920746F6F206D75636820696E6133
:103C000063746976652074696D65202D2063757213
:103C100072656E7420636F6D6D616E643A20005042
:103C20006C65617365207265736574005052494E0E
:103C30005445522048414C544544005072696E74BA
:103C400065722068616C7465642E206B696C6C28E9
:103C5000292063616C6C6564210A00656E7175656D
:103C60007565696E672022000000000000000000FA
:103C7000000000005761726E696E673A20486F6DF0
:103C8000696E672042756D702044697669736F7242
:103C9000203C20310A000000A0400000A0400000AD
:103CA0000040000096430000964300009643FFFF4B
:103CB000FF7C3C3E5E2B3D3F2F5B5D3B2C2A225C14
:103CC0000020746F6F206C6F6E672065787472755A
:103CD00073696F6E2070726576656E7465640A0034
:103CE00020636F6C6420657874727573696F6E20E1
:103CF00070726576656E7465640A0020706F736912
:103D000074696F6E206F7574206F662072616E67C4
:103D1000652E0A003F50726F62652000486F6D6526
:103D200020257325732573206669727374002066DD
:103D3000697273740A005A0059005800486F6D6523
:103D400020005374616E6461726420446576696119
:103D500074696F6E3A20002052616E67653A2000E8
:103D6000204D61783A2000204D696E3A20004D6563
:103D7000616E3A200046696E6973686564210020AF
:103D800072616E67653A2000206D61783A200020EC
:103D90006D696E3A2000207369676D613A200020DA
:103DA0006D65616E3A20003A207A3A2000206F66F5
:103DB0002000205A00205900205800476F696E6784
:103DC00020746F3A00436C6F636B776973650A0008
:103DD000436F756E7465722D00204469726563745B
:103DE000696F6E3A2000202020616E676C653A2072
:103DF000005374617274696E6720726164697573CF
:103E00003A2000506F736974696F6E696E67207431
:103E100068652070726F62652E2E2E0A003F4E7507
:103E20006D626572206F66206C65677320696E2015
:103E30006D6F76656D656E74206E6F7420706C6149
:103E4000757369626C652028302D3135292E0A0082
:103E5000590058003F53616D706C652073697A6535
:103E6000206E6F7420706C61757369626C652028B8
:103E7000342D3530292E0A004D3438205A2D5072F9
:103E80006F6265205265706561746162696C697406
:103E90007920546573740A003F566572626F7365CA
:103EA000204C6576656C206E6F7420706C61757344
:103EB00069626C652028302D34292E0A002042408A
:103EC0003A0020403A00202F0020423A00202F00E4
:103ED00020543A004578747275646572004D6F76AF
:103EE00065205A004D6F76652059004D6F7665202C
:103EF00058005072657061726500526573746F721C
:103F000065206661696C736166650046696C616D08
:103F1000656E74004D6F74696F6E0054656D7065E9
:103F2000726174757265004D61696E0050726568EA
:103F30006561742041425320636F6E660050726564
:103F40006865617420504C4120636F6E6600504973
:103F5000442D44005049442D44005049442D49000B
:103F60005049442D49005049442D50005049442D9A
:103F700050002008204661637400200820466163D9
:103F800074002008204D6178002008204D617800E1
:103F90002008204D6178002008204D696E0020081F
:103FA000204D696E002008204D696E004F66660046
:103FB0004F6E20004175746F74656D700046616EC0
:103FC0002073706565640046616E2073706565647A
:103FD0000042656400426564004E6F7A7A6C650049
:103FE0004E6F7A7A6C6500436F6E74726F6C00422C
:103FF000656400426564004E6F7A7A6C65004E6FAE
:104000007A7A6C650046616E20737065656400465F
:10401000616E2073706565640054656D70657261D2
:1040200074757265004573746570732F6D6D00450E
:1040300073746570732F6D6D005A73746570732F90
:104040006D6D005A73746570732F6D6D00597374C4
:104050006570732F6D6D005973746570732F6D6D7E
:10406000005873746570732F6D6D005873746570AC
:10407000732F6D6D00412D74726176656C00412D5A
:1040800074726176656C00412D726574726163743F
:1040900000412D7265747261637400416D61782016
:1040A0004500416D6178204500416D6178205A00DE
:1040B000416D6178205A00416D6178205900416D51
:1040C0006178205900416D6178205800416D617818
:1040D0002058005654726176206D696E00565472F5
:1040E0006176206D696E005654726176206D696E3E
:1040F00000566D696E00566D696E00566D696E00F2
:10410000566D6178204500566D6178204500566DEA
:104110006178204500566D6178205A00566D6178AF
:10412000205A00566D6178205A00566D61782059EA
:1041300000566D6178205900566D617820590056FF
:104140006D6178205800566D6178205800566D6179
:104150007820580056652D6A65726B0056652D6A89
:1041600065726B0056652D6A65726B00567A2D6A12
:1041700065726B00567A2D6A65726B0056792D6AEE
:1041800065726B0056792D6A65726B0056792D6ADF
:1041900065726B0056782D6A65726B0056782D6AD1
:1041A00065726B0056782D6A65726B0041636365BA
:1041B0006C00416363656C005A204F6666736574DA
:1041C000005A204F666673657400436F6E74726F99
:1041D0006C0046696C2E204469612E0046696C2E85
:1041E000204469612E004F6666004F6E2000452016
:1041F000696E206D6D3300436F6E74726F6C004E8C
:104200006F204C696E65204E756D6265722077690E
:10421000746820636865636B73756D2C204C6173E3
:1042200074204C696E653A20004B494C4C45442E35
:10423000200053544F505045442E20005072696E58
:104240007465722073746F70706564206475652086
:10425000746F206572726F72732E204669782074B5
:104260006865206572726F7220616E642075736577
:10427000204D39393920746F2072657374617274FE
:104280002E202854656D70657261747572652069A1
:10429000732072657365742E2053657420697420D1
:1042A00061667465722072657374617274696E6799
:1042B000290A004E6F20436865636B73756D207724
:1042C000697468206C696E65206E756D6265722C0C
:1042D000204C617374204C696E653A2000636865F8
:1042E000636B73756D206D69736D617463682C20E9
:1042F0004C617374204C696E653A20004C696E65A0
:10430000204E756D626572206973206E6F74204C4B
:10431000617374204C696E65204E756D6265722BF9
:10432000312C204C617374204C696E653A20004D2D
:10433000313130004D3331004D3834205820592070
:104340005A20450053442072656164206572726F83
:10435000720A00446F6E65207072696E74696E67D0
:104360002066696C650A0020496E76616C6964207C
:1043700065787472756465722000000096430000D1
:10438000964300009643000000000000000000007B
:104390000000205A3A200020593A2000426564204B
:1043A000583A200043616E6E6F74206F70656E2006
:1043B00073756264697220006563686F3A00205A01
:1043C0003A0020593A0020436F756E7420583A0025
:1043D00020453A00205A3A0020593A00583A002025
:1043E000643A0020693A0020703A0043290A0061CB
:1043F000626C656420286D696E2074656D702000A4
:10440000436F6C64206578747275646573206172A3
:104410006520004B64200023646566696E6520207A
:1044200044454641554C545F004B69200023646568
:1044300066696E65202044454641554C545F004BEB
:1044400070200023646566696E65202044454641FE
:10445000554C545F00504944204175746F74756E1B
:10446000652066696E6973686564212050757420E3
:10447000746865206C617374204B702C204B69202C
:10448000616E64204B6420636F6E7374616E74732D
:104490002066726F6D2062656C6F7720696E746F35
:1044A00020436F6E66696775726174696F6E2E68FE
:1044B0000A00504944204175746F74756E6520661A
:1044C00061696C6564212074696D656F75740A009B
:1044D000504944204175746F74756E65206661693A
:1044E0006C6564212054656D7065726174757265C8
:1044F00020746F6F20686967680A00204B643A2057
:1045000000204B693A2000204B703A20000A2043DB
:104510006C617373696320504944200A002054750C
:104520003A2000204B753A2000206D61783A200037
:10453000206D696E3A200020643A20002062696193
:10454000733A20006265640A002C207379737465E5
:104550006D2073746F7070656421204865617465A7
:10456000725F49443A200048656174696E6720664D
:1045700061696C65640048656174696E6720666195
:10458000696C65640048656174696E67206661697D
:104590006C65640048656174696E67206661696C6A
:1045A00065640070012C0190012701B0012201C057
:1045B000011D01F00118011002130130020E01600B
:1045C00002090190020401C002FF000003FA00404A
:1045D00003F5008003F000D003EB002004E6007038
:1045E00004E100E004DC004005D700C005D2004033
:1045F00006CD00D006C8008007C3003008BE00F01A
:1046000008B900C009B400B00AAF00B00BAA00D0CE
:104610000CA500000EA000500F9B00C0109600508B
:1046200012910000148C00C0158700B0178200B0F2
:10463000197D00D01B7800001E730040206E009092
:10464000226900F024640040275F0090295A00E0AE
:104650002B5500102E500020304B0010324600E049
:1046600033410090353C001037370070383200A0DD
:10467000392D00B03A2800A03B2300603C1E0010FA
:104680003D1900903D1400103E0F00703E0A00C01E
:104690003E0500003F0000403FFBFF803FF6FFC0AB
:1046A0003FF1FF544845524D414C2052554E415721
:1046B000415900546865726D616C2052756E617766
:1046C00061790000060900FE070192032120FFFF27
:1046D00008FF07FF000000060000010707060200B0
:1046E00080808080800080030202060105A0A00572
:1046F00007070600005050F850F85050050707060D
:1047000000002078A07028F020050707060000C0F0
:10471000C810204098180507070600006090A040C8
:10472000A89068020303060104C04080030707063F
:1047300001002040808080402003070706010080A0
:1047400040202020408005050506000120A870A813
:10475000200505050600012020F82020020303069D
:1047600002FFC04080050101060003F802020206B4
:104770000200C0C0050505060001081020408005A4
:104780000707060000708888888888700307070676
:10479000010040C040404040E005070706000070AF
:1047A0008808708080F8050707060000F8102010C0
:1047B0000808F005070706000010305090F81010A8
:1047C000050707060000F880F0080888700507074D
:1047D000060000708080F0888870050707060000DA
:1047E000F8081020202020050707060000708888A0
:1047F00070888870050707060000708888780808A8
:1048000070020505060200C0C000C0C00206060610
:1048100002FFC0C000C0408004070706000010204F
:104820004080402010050303060002F800F804074A
:104830000706010080402010204080050707060081
:104840000070880810200020050707060000708807
:104850000868A8A870050707060000708888F8880F
:104860008888050707060000F08888F08888F0052A
:10487000070706000070888080808870050707069B
:104880000000F08888888888F0050707060000F88F
:104890008080F08080F8050707060000F88080F02F
:1048A000808080050707060000708880B8888870BF
:1048B000050707060000888888F8888888010707A8
:1048C0000602008080808080808005070706000047
:1048D000381010101090600507070600008890A09F
:1048E000C0A0908805070706000080808080808037
:1048F000F805070706000088D8A888888888050773
:10490000070600008888C8A8988888050707060059
:104910000070888888888870050707060000F0887E
:1049200088F080808005070706000070888888A8C6
:104930009068050707060000F08888F0A0908805B9
:104940000707060000788080700808F00507070652
:104950000000F820202020202005070706000088FE
:1049600088888888887005070706000088888888F6
:104970008850200507070600008888888888A85086
:10498000050707060000888850205088880507071B
:1049900006000088888850202020050707060000B0
:1049A000F80810204080F8030707060100E0808027
:1049B000808080E005050506000180402010080386
:1049C0000707060100E02020202020E00503030661
:1049D0000004205088050101060000F802020206CA
:1049E00002058040050505060000700878887805F6
:1049F00007070600008080B0C88888F00505050616
:104A000000007080808870050707060000080868AD
:104A1000988888780505050600007088F88070057C
:104A200007070600003048E0404040400506060603
:104A300000FF7088887808700507070600008080EE
:104A4000B0C888888801070706020080008080803F
:104A500080800308080601FF200020202020A040BD
:104A6000040707060000808090A0C0A090030707FD
:104A7000060100C04040404040E00505050600003A
:104A8000D0A8A8A8A8050505060000B0C888888891
:104A90000505050600007088888870050606060072
:104AA000FFF08888F080800506060600FF78888879
:104AB000780808050505060000B0C8808080050557
:104AC0000506000070807008F0040707060000402B
:104AD00040E0404040300505050600008888889881
:104AE000680505050600008888885020050505062C
:104AF00000008888A8A850050505060000885020F9
:104B000050880506060600FF888888780870050525
:104B100005060000F8102040F803070706010020F2
:104B200040408040402001070706020080808080CE
:104B300080808003070706010080404020404080BD
:104B40000502020600026890000000060000000056
:104B50000006000000000006000000000006000043
:104B60000000000600000000000600000000000633
:104B70000000000000060000000000060000000029
:104B80000006000000000006000000000006000013
:104B90000000000600000000000600000000000603
:104BA00000000000000600000000000600000000F9
:104BB00000060000000000060000000000060000E3
:104BC00000000006000000000006000000000006D3
:104BD00000000000000600000000000600000000C9
:104BE00000060000000000060000000000060000B3
:104BF00000000006000000000006000000000006A3
:104C00000000000000060000000000060000000098
:104C100000060000010707060200800080808080F7
:104C2000800507070600002070A8A0A870200507CF
:104C300007060000304040E04050A805050506008A
:104C4000008870507088050707060000885020F81B
:104C500020F8200107070602008080800080808005
:104C600005080806000030482050502090600301DD
:104C700001060107A0050707060000F888B8B8B8C4
:104C800088F8050707060001700878887800F8059D
:104C900005050600012850A0502805030306000161
:104CA000F80808020202060206408005070706000F
:104CB00000F888A88898A8F8050101060006F804FD
:104CC00004040600036090906005070706000020BA
:104CD00020F8202000F8040505060003609020401D
:104CE000F0030505060003E020E020E002020206D2
:104CF000020640800508080600FF8888888898E832
:104D00008080050707060000789898781818180220
:104D10000202060202C0C00202020602FF40800335
:104D2000050506000340C04040E0050707060001F6
:104D3000708888887000F8050505060001A05028D5
:104D400050A00507070600008890A858B808080575
:104D500007070600008890B848982038050808061C
:104D60000000C040C048D838080805070706000002
:104D700020002040808870050808060000402000C0
:104D80007088F888880508080600001020007088E0
:104D9000F888880508080600002050007088F88808
:104DA000880508080600006890007088F888880563
:104DB00008080600005000708888F88888050808F0
:104DC0000600002050207088F88888050707060034
:104DD000003860A0B8E0A0B80508080600FF708899
:104DE000808088702060050808060000402000F8D8
:104DF00080F080F8050808060000081000F880F030
:104E000080F8050808060000205000F880F080F8BF
:104E10000507070600005000F880F080F803080836
:104E2000060100804000E0404040E0030808060121
:104E300000204000E0404040E00308080601004038
:104E4000A000E0404040E0030707060100A000E0AA
:104E5000404040E0050707060000704848E8484821
:104E60007005080806000068900088C8A8988805A2
:104E700008080600004020708888888870050808A7
:104E800006000010207088888888700508080600D1
:104E900000205000708888887005080806000068A7
:104EA000900070888888700508080600005000701F
:104EB000888888887005050506000188502050887C
:104EC0000508080600FF1070A8A8A8A870400508EB
:104ED0000806000040208888888888700508080631
:104EE000000010208888888888700508080600005F
:104EF0002050008888888870050808060000500047
:104F00008888888888700508080600001020885066
:104F1000202020200509090600FFC0407048487085
:104F20004040E00408080601FF609090A09090E0E7
:104F30008005080806000040200070087888780581
:104F40000808060000102000700878887805080816
:104F500006000020500070087888780508080600D0
:104F600000689000700878887805070706000050F0
:104F70000070087888780508080600002050207026
:104F800008788878050606060000D02878A0A85082
:104F90000506060600FF7080887020600508080678
:104FA00000004020007088F88070050808060000A6
:104FB0001020007088F88070050808060000205056
:104FC000007088F8807005070706000050007088A0
:104FD000F8807003080806010080400040C040408F
:104FE000E003080806010020400040C04040E00304
:104FF000080806010040A00040C04040E003070749
:10500000060100A00040C04040E005070706000080
:10501000A040A0107888700508080600006890007D
:10502000B0C88888880508080600004020007088FD
:10503000888870050808060000102000708888889D
:1050400070050808060000205000708888887005E8
:1050500008080600006890007088888870050707B7
:10506000060000500070888888700505050600015C
:105070002000F800200507070600FF1070A8A8A868
:10508000704005080806000040200088888898685D
:105090000508080600001020008888889868050820
:1050A00008060000205000888888986805070706D1
:1050B0000000500088888898680509090600FF10DC
:1050C0002000888888F808700407070601FFC040A0
:1050D00060506040E00508080600FF50008888889E
:1050E0007808700277E201E211241FBECFEFD1E20F
:1050F000DEBFCDBF00E00CBF14E0A0E0B2E0E2E212
:10510000F0EE01E00BBF02C007900D92A636B1078A
:10511000D9F724E1A6E6B4E001C01D92A339B20795
:10512000E1F718E2C3E7D8E200E006C021970109E1
:10513000802FFE010E947AEFC237D10780E0080776
:10514000A9F70E9452DA0C9400F00C9400002F9200
:105150003F924F925F926F927F928F929F92AF9207
:10516000BF92CF92DF92EF92FF920F931F93CF9354
:10517000DF93CDB7DEB7C657D1090FB6F894DEBFBF
:105180000FBECDBF8091AE0620E6829FC0011124E4
:10519000825D9A4F90932C0D80932B0D8091EE0D94
:1051A00080FF1BC0E8EBF3E484918F010F5F1F4F7A
:1051B000882321F00E945C87F801F6CF00912B0D27
:1051C00010912C0DD8018D918D01882319F00E942A
:1051D0005C87F8CF8AE00E945C87E0912B0DF0910C
:1051E0002C0D8081803231F43196F0932C0DE093B8
:1051F0002B0DF3CF8E3469F010912B0D00912C0DF7
:105200006AE270E0812F902F0E94C8EF009721F58D
:105210002AC0818190ED980F9A3010F08D3261F79D
:105220003296F0932C0DE0932B0DE0912B0DF09125
:105230002C0D808180538A3010F43196F2CFE091AA
:105240002B0DF0912C0D80818032B1F63196F093C8
:105250002C0DE0932B0DF3CFFC013196829180321F
:1052600031F08A3221F0A12FB02F9D9102C010821F
:10527000F5CFFD01808111968032D9F380538A30B9
:1052800020F0E8EBF3E40C94B140E12CF12C2AE09F
:105290002E9DB0012F9D700D11247B01B0E3EB1A00
:1052A000F1088191E80EF11C87FDFA94808180530A
:1052B0008A3070F38F013196D8018C918032D1F30E
:1052C000109371040093700421E030E030932A0DB4
:1052D0002093290D9D3411F40C943A32943511F435
:1052E0000C944740973411F00C945F40B4E0EB16F7
:1052F000F10409F486C640F48091AA02F2E0EF16A8
:10530000F10408F020C11FC02AE5E216F10411F4EF
:105310000C94893160F44CE1E416F10409F4AFC651
:105320005EE1E516F10409F42FC70C94A8408BE563
:10533000E816F10409F4F1C79CE5E916F10409F453
:10534000F1C70C94A840882311F40C94A8400E9443
:105350002AAC80913102882321F08DE49DE00E94E7
:105360009A880E944D498091EE0D83FD9BC0C090AC
:10537000590DD0905A0DE0905B0DF0905C0D20918E
:10538000090530910A0540910B0550910C05C701A4
:10539000B6010E946CE8882309F484C08091E90D6D
:1053A00081113CC0609198047091990480919A0495
:1053B00090919B040E94D3ED072E000C880B990B53
:1053C0000E9472E820913F023091400240914102D8
:1053D000509142020E946CE887FF20C0C0920905EC
:1053E000D0920A05E0920B05F0920C05E8EBF3E48D
:1053F00084918F010F5F1F4F882321F00E945C87EB
:10540000F801F6CFE8EFF1E084918F010F5F1F4FB5
:10541000882321F00E945C87F801F6CFC090590DD7
:10542000D0905A0DE0905B0DF0905C0D2091090535
:1054300030910A0540910B0550910C05C701B6014A
:105440000E948EEC0E94D3ED97FF07C09095809547
:10545000709561957F4F8F4F9F4F693C7105810516
:10546000910504F1C0920905D0920A05E0920B055E
:10547000F0920C05E8EBF3E484918F010F5F1F4F6E
:10548000882321F00E945C87F801F6CFE9EDF1E076
:1054900084918F010F5F1F4F882321F00E945C874A
:1054A000F801F6CF20914D0D30914E0D40914F0DEA
:1054B0005091500D6091FD047091FE048091FF04A5
:1054C000909100050E946CE881111DC02091510D42
:1054D0003091520D4091530D5091540D6091010542
:1054E0007091020580910305909104050E946CE87B
:1054F000811109C060910002709101028091020245
:10550000909103021AC06091230270912402072E29
:10551000000C880B990B0E9472E8209100023091D8
:10552000010240910202509103020E94D1E82AE058
:1055300037ED43E25CE30E94D1E80E9426BE0E9460
:105540001CBE0C94A840882311F40C94A84011E0D0
:10555000A2E0EA16F10409F010E00E942AAC82E50C
:105560000E9493BE882309F452C10E9455BF6B016B
:105570007C014090FD045090FE046090FF04709008
:1055800000052091010530910205409103055091DD
:1055900004052BAF3CAF4DAF5EAF80914D0D9091A8
:1055A0004E0DA0914F0DB091500D23968CAF9DAF35
:1055B000AEAFBFAF23972091510D3091520D409166
:1055C000530D5091540D2B962CAF3DAF4EAF5FAFA6
:1055D0002B9720E030E0A901C701B6010E946CE8DA
:1055E000882309F4F4C4A301920123966CAD7DAD28
:1055F0008EAD9FAD23970E946CE881110FC02BAD3B
:105600003CAD4DAD5EAD2B966CAD7DAD8EAD9FAD21
:105610002B970E946CE8882309F4D9C420E030E07D
:10562000A901C701B6010E946CE8881F8827881F5E
:1056300018130BC080E090E0A0E8BFE367968CAF42
:105640009DAFAEAFBFAF67970AC020E030E040E843
:105650005FEB67962CAF3DAF4EAF5FAF6797A3018F
:10566000920123966CAD7DAD8EAD9FAD23970E94C8
:105670008EEC2F966CAF7DAF8EAF9FAF2F972BAD7B
:105680003CAD4DAD5EAD2B966CAD7DAD8EAD9FADA1
:105690002B970E948EEC63966CAF7DAF8EAF9FAF61
:1056A00063972F962CAD3DAD4EAD5FAD2F97CA01E0
:1056B000B9010E94D1E84B015C0163962CAD3DAD70
:1056C0004EAD5FAD6397CA01B9010E94D1E89B015D
:1056D000AC01C501B4010E948FEC0E94FAEE27963E
:1056E0006CAF7DAF8EAF9FAF279720E030E040E0FA
:1056F0005FE30E94D1E84B015C01A7019601C7015D
:10570000B6010E94D1E86B017C01A5019401C5019D
:10571000B4010E94D1E89B01AC01C701B6010E940F
:105720008EEC0E94FAEE9B01AC0167966CAD7DADEC
:105730008EAD9FAD67970E94D1E84B015C01239627
:105740002CAD3DAD4EAD5FAD2397C301B2010E94BC
:105750008FEC20E030E040E05FE30E94D1E86B0195
:105760007C0163966CAD7DAD8EAD9FAD6397905817
:1057700027962CAD3DAD4EAD5FAD27970E946BEDEA
:105780009B01AC01C501B4010E94D1E89B01AC01B1
:10579000C701B6010E948FECA30192010E948EEC1A
:1057A0006B017C012B962CAD3DAD4EAD5FAD2B97C3
:1057B0006BAD7CAD8DAD9EAD0E948FEC20E030E0F6
:1057C00040E05FE30E94D1E82B013C0127962CAD1D
:1057D0003DAD4EAD5FAD27972F966CAD7DAD8EADD7
:1057E0009FAD2F970E946BED9B01AC01C501B401E9
:1057F0000E94D1E89B01AC01C301B2010E948FEC71
:105800002BAD3CAD4DAD5EAD0E948EEC14C089E475
:105810000E9493BE882329F00E9455BF6B017C0132
:1058200003C0C12CD12C76018AE40E9493BE882348
:10583000F9F00E9455BF2B966CAF7DAF8EAF9FAF36
:105840002B9720E030E0A901C701B6010E946CE867
:1058500081111EC020E030E0A9012B966CAD7DAD1A
:105860008EAD9FAD2B970E946CE8811111C0AFC324
:1058700020E030E0A901C701B6010E946CE888234E
:1058800009F4A5C32B961CAE1DAE1EAE1FAE2B9702
:10589000D701C601B0588BAF9CAFADAFBEAF2B9652
:1058A0002CAD3DAD4EAD5FAD2B97505823962CAF30
:1058B0003DAF4EAF5FAF23979C01AD01BC01CD0161
:1058C0000E94D1E84B015C0123962CAD3DAD4EAD5D
:1058D0005FAD2397CA01B9010E94D1E89B01AC01D9
:1058E000C501B4010E948FEC0E94FAEEA7966CAF3E
:1058F0007DAF8EAF9FAFA7978091FD049091FE047E
:10590000A091FF04B091000527968CAF9DAFAEAF7C
:10591000BFAF2797A7019601BC01CD010E948FEC74
:1059200067966CAF7DAF8EAF9FAF679720910105F3
:105930003091020540910305509104052F962CAF3C
:105940003DAF4EAF5FAF2F972B962CAD3DAD4EAD1B
:105950005FAD2B972F966CAD7DAD8EAD9FAD2F9724
:105960000E948FEC6B966CAF7DAF8EAF9FAF6B9745
:1059700080914D0D90914E0DA0914F0DB091500D15
:105980006F968CAF9DAFAEAFBFAF6F9767962CADE4
:105990003DAD4EAD5FAD6797BC01CD010E948EEC71
:1059A0006B017C012091510D3091520D4091530DAE
:1059B0005091540DA3962CAF3DAF4EAF5FAFA39760
:1059C0006B962CAD3DAD4EAD5FAD6B97A3966CADB8
:1059D0007DAD8EAD9FADA3970E948EEC4B015C0117
:1059E0008091050590910605A0910705B0910805E5
:1059F000AF968CAF9DAFAEAFBFAFAF979C01AD017F
:105A00006091550D7091560D8091570D9091580DE4
:105A10000E948EEC63966CAF7DAF8EAF9FAF6397A5
:105A20002091590D30915A0D40915B0D50915C0DB4
:105A3000AB962CAF3DAF4EAF5FAFAB9780910905F2
:105A400090910A05A0910B05B0910C05E3968CAFDF
:105A50009DAFAEAFBFAFE397A70196016BAD7CAD35
:105A60008DAD9EAD0E94D1E82B013C01A5019401B2
:105A700023966CAD7DAD8EAD9FAD23970E94D1E88E
:105A80009B01AC01C301B2010E948FEC2B013C01D0
:105A9000A50194016BAD7CAD8DAD9EAD0E94D1E8AA
:105AA0004B015C01A701960123966CAD7DAD8EADD7
:105AB0009FAD23970E94D1E89B01AC01C501B401C1
:105AC0000E948EECA30192010E9402ED6B017C0109
:105AD00020E030E0A9010E946CE887FF0AC02BEDAE
:105AE0003FE049EC50E4C701B6010E948FEC6B0126
:105AF0007C01112351F02BED3FE049EC50E4C7014C
:105B0000B6010E948EEC6B017C0120E030E0A9011F
:105B1000C701B6010E946CE881112AC06F962CADB6
:105B20003DAD4EAD5FAD6F9727966CAD7DAD8EAD43
:105B30009FAD27970E946CE881111AC0A3962CADE7
:105B40003DAD4EAD5FADA3972F966CAD7DAD8EADE7
:105B50009FAD2F970E946CE881110AC02BED3FE0AA
:105B600049EC50E4C701B6010E948FEC6B017C0147
:105B7000A7962CAD3DAD4EAD5FADA797C701B60161
:105B80000E94D1E89B01AC010E94D1E84B015C016D
:105B900063962CAD3DAD4EAD5FAD6397CA01B901C3
:105BA0000E94D1E89B01AC01C501B4010E948FECB9
:105BB0000E94FAEE4B015C012FE632E143E85AE322
:105BC0000E946CE887FDFFC1C501B4010E9404EE8C
:105BD0000E94D8ED2D967FAF6EAF2D97DB01AB2BDA
:105BE00031F4E1E0F0E02D96FFAFEEAF2D972D966A
:105BF0002EAD3FAD2D97B90180E090E00E9470E896
:105C00004B015C019B01AC01C701B6010E946BED29
:105C100027966CAF7DAF8EAF9FAF2797A5019401FC
:105C200063966CAD7DAD8EAD9FAD63970E946BEDBD
:105C3000A7966CAF7DAF8EAF9FAFA797E3962CADC5
:105C40003DAD4EAD5FADE397AB966CAD7DAD8EAD2A
:105C50009FADAB970E948EECA50194010E946BED65
:105C6000AB966CAF7DAF8EAF9FAFAB9727962CAD49
:105C70003DAD4EAD5FAD2797CA01B9010E94D1E895
:105C800020E030E040E05FE30E94D1E89B01AC01FE
:105C900060E070E080E89FE30E948EEC63966CAF5A
:105CA0007DAF8EAF9FAF6397AF968CAD9DADAEAD20
:105CB000BFADAF9789879A87AB87BC87E3962CAD3A
:105CC0003DAD4EAD5FADE3972D873E874F87588B37
:105CD0006091230270912402072E000C880B990B0F
:105CE0000E9472E82091000230910102409102026C
:105CF000509103020E94D1E82AE037ED43E25CE3D1
:105D00000E94D1E86F966CAF7DAF8EAF9FAF6F975B
:105D10000E94D75B9B01AC0128533F4F4F4F5F4F11
:105D2000A3962CAF3DAF4EAF5FAFA3974BAC5CAC2F
:105D30006DAC7EAC22242394312CD12C2D968EADCB
:105D40009FAD2D972816390609F429C10E9488D3E2
:105D50000E94D75BDC01CB01A3962CAD3DAD4EADCF
:105D60005FADA397821B930BA40BB50BB7FD10C0BF
:105D70000E94D75B9B01AC0128533F4F4F4F5F4FB1
:105D8000A3962CAF3DAF4EAF5FAFA3970E941F8B82
:105D9000D39438E13D150CF44BC063962CAD3DAD6A
:105DA0004EAD5FAD639723966CAD7DAD8EAD9FAD6F
:105DB00023970E94D1E84B015C0127962CAD3DADA5
:105DC0004EAD5FAD2797B201C3010E94D1E8A50196
:105DD00094010E948FEC7B018C0163962CAD3DAD4C
:105DE0004EAD5FAD6397B201C3010E94D1E84B0194
:105DF0005C0127962CAD3DAD4EAD5FAD2797239648
:105E00006CAD7DAD8EAD9FAD23970E94D1E89B0117
:105E1000AC01C501B4010E948EEC2B013C01C7010D
:105E2000D80123968CAF9DAFAEAFBFAF239756C0BE
:105E3000B10180E090E00E9470E827962CAD3DAD66
:105E40004EAD5FAD27970E94D1E84B015C010E94E7
:105E500068ED6B017C01C501B4010E94F0EE4B01BD
:105E60005C01A70196016BAD7CAD8DAD9EAD0E942E
:105E7000D1E82B013C01A50194012B966CAD7DADC1
:105E80008EAD9FAD2B970E94D1E89B01AC01C30161
:105E9000B2010E948FEC2B013C01A50194016BAD76
:105EA0007CAD8DAD9EAD0E94D1E84B015C01A70198
:105EB00096012B966CAD7DAD8EAD9FAD2B970E945C
:105EC000D1E89B01AC01C501B4010E948EEC239680
:105ED0006CAF7DAF8EAF9FAF2397D12C9201A30102
:105EE00067966CAD7DAD8EAD9FAD67970E948FECD0
:105EF00069837A838B839C8323962CAD3DAD4EAD15
:105F00005FAD23976B966CAD7DAD8EAD9FAD6B97FE
:105F10000E948FEC6D837E838F839887A7962CAD2C
:105F20003DAD4EAD5FADA79769857A858B859C8524
:105F30000E948FEC69877A878B879C87AB962CAD04
:105F40003DAD4EAD5FADAB976D857E858F859889F4
:105F50000E948FEC6D877E878F87988B80913102AE
:105F6000882321F0CE0101960E949A88C0906A048D
:105F70006F96ECACFDAC0EAD1FAD6F979E01235F2D
:105F80003F4FAE01475F5F4FBE016B5F7F4FCE015A
:105F900001960E94B7984FEF241A340ACFCEC090D2
:105FA0006A046F96ECACFDAC0EAD1FAD6F9729E5A2
:105FB0003DE045E55DE061E57DE08DE49DE00E942A
:105FC000B7980E941CBE0E944D490C94A840E3E57E
:105FD000F3E384918F010F5F1F4F882321F00E940C
:105FE0005C87F801F6CFE3E1F2E084918F010F5F67
:105FF0001F4F882311F40C94A8400E945C87F8017D
:10600000F4CF80E50E9493BE882329F00E944ABF06
:106010006B017C0103C0C12CD12C760183E50E9469
:1060200093BE882321F00E947EBF6B017C010E94F9
:10603000E3D40E944D4980912D0D90912E0DA09199
:106040002F0DB091300DC80ED91EEA1EFB1E809197
:106050006702811105C060E089E292E00E9437D9B1
:106060000E94D75BDC01CB018C199D09AE09BF09E9
:10607000B7FD02C00C94A8400E941F8BF1CF0E9474
:10608000E3D40E94DFBA81E080930B0288E50E948E
:1060900093BEE82E89E50E9493BE082F8AE50E94F0
:1060A00093BEF82EE11005C0011105C011E01827BC
:1060B00005C0011102C010E001C0182F80E1EDEF12
:1060C000F4E0ADE4BDE001900D928A95E1F7111185
:1060D00005C0E11003C0002309F444C020E030E013
:1060E00040EA50E460913D0D70913E0D80913F0D6E
:1060F0009091400D0E948FEC6093550D7093560D5A
:106100008093570D9093580D209105053091060509
:1061100040910705509108050E94B5EE18167CF4D1
:1061200019821A821B821C829E012F5F3F4F45E518
:106130005DE061E075E08DEF94E00E94FFBA11111F
:1061400005C0E11003C0011107C00CC080E090E061
:106150000E942C891123B9F381E090E00E942C89E0
:10616000111102C0FF2021F082E090E00E942C89F2
:106170000E943D498091680480930B020E94C5BA39
:106180000E9482CD0C94A84088E50E9493BE88238B
:1061900019F00E9455BF0EC020E030E040E251E40B
:1061A0006091FD047091FE048091FF0490910005C0
:1061B0000E948FEC4B015C0189E50E9493BE88230D
:1061C00019F00E9455BF0EC020E030E040E251E4DB
:1061D000609101057091020580910305909104057D
:1061E0000E948FEC2B013C0120913D0D30913E0D22
:1061F00040913F0D5091400D2BAF3CAF4DAF5EAF86
:106200002091350D3091360D4091370D5091380D5C
:10621000C501B4010E948EEC2091390D30913A0DE8
:1062200040913B0D50913C0D23962CAF3DAF4EAFAE
:106230005FAF239720E030E040E251E40E948EEC13
:106240006B017C0127E137EB41ED58EB0E94B5EE85
:1062500087FF02C00C94A84023E030E046E953E4F5
:10626000C701B6010E946CE8181614F40C94A840FB
:1062700023962CAD3DAD4EAD5FAD2397C301B2016A
:106280000E948EEC20E030E040E251E40E948EEC6F
:106290006B017C0127E137EB41ED58EB0E94B5EE35
:1062A00087FF02C00C94A84023E030E046E953E4A5
:1062B000C701B6010E946CE8181614F40C94A840AB
:1062C00020E030E0A9016BAD7CAD8DAD9EAD0E94AC
:1062D0008FEC2BAD3CAD4DAD5EAD0E948EEC6B01F5
:1062E0007C0127E137EB41ED58EB0E94B5EE87FFCB
:1062F00002C00C94A84023E030E046E953E4C70113
:10630000B6010E946CE8181614F40C94A8400C9482
:10631000614010926F040C94A84081E080936F0458
:106320000C94A94085E40E9493BEB82E811102C04E
:106330000E94E3D4BCEB8B2EB2E09B2E1DEFC12E4E
:1063400014E0D12E01E4E02E0DE0F02E00E010E08C
:10635000A12CD4018D914D010E9493BE8823F1F1AF
:10636000F6012081318142815381E4962FAFE49779
:10637000E5963FAFE597E6964FAFE697E7965FAFB6
:10638000E7970E9455BFD6016D937D938D939C93A3
:106390001397E4962FADE497E5963FADE597E69623
:1063A0004FADE697E7965FADE79703301105B1F083
:1063B0000E948EEC9B01AC01F701608171818281AA
:1063C00093810E948FECD7016D937D938D939C9365
:1063D0001397C8010E943FBEAA24A3940F5F1F4FCA
:1063E000B4E0CB0ED11CE4E0EE0EF11C043011053C
:1063F00009F0AFCFAA2019F00E943D4937C0BB2059
:10640000A9F1C0900905D0900A05E0900B05F09025
:106410000C0520912D0E30912E0E40912F0E509193
:10642000300EC701B6010E94D1E80E94C0EE609311
:106430005611709357118093581190935911C701B9
:10644000B6010E94D3ED2FB7F89460932714709390
:1064500028148093291490932A142FBF1092461168
:106460001092471110924811109249110E9482CD4A
:106470000C94A840F1E7EF16F10409F493C608F074
:10648000E6C030E3E316F10409F47CC508F077C0F8
:1064900058E1E516F10409F4C3C208F044C092E1E2
:1064A000E916F10409F45AC7E8F4B2E0EB16F10476
:1064B00008F4EFC1E1E1EE16F10411F00C94A840EC
:1064C00060E08AE792E00E9437D95F988A989FB788
:1064D000F894809108018E7F809308019FBF1298E5
:1064E0000C94A840F5E1EF16F10409F48FC248F4CA
:1064F00034E1E316F10411F00C94A840E2E9F2E073
:1065000042C246E1E416F10409F484C257E1E516FB
:10651000F10411F00C94A84040E061E0C8010E9431
:10652000B0740C94A8408CE1E816F10409F4CDC2D3
:1065300068F4AAE1EA16F10409F47DC208F089C200
:1065400010928A110E94BB790C94A840EFE1EE16DC
:10655000F10409F429C438F42EE1E216F10409F437
:10656000BBC20C94A84030E2E316F10409F4CCC39A
:106570004AE2E416F10409F4BDC40C94A8405CE5B9
:10658000E516F10409F428C768F591E5E916F10468
:1065900009F4C7C6A0F4BCE4EB16F10409F4F6C490
:1065A000EDE4EE16F10409F4F5C4FBE4EF16F10492
:1065B00011F00C94A8400E947B790C94A84023E52C
:1065C000E216F10409F4C6C608F4C1C644E5E416AF
:1065D000F10409F4C3C655E5E516F10409F4EBC668
:1065E0000C94A8408CE6E816F10409F4D8C5C8F468
:1065F000A9E6EA16F10409F412C638F4E8E6EE1644
:10660000F10409F4CBC40C94A840FAE6EF16F104A7
:1066100009F453C62BE6E216F10409F472C60C9491
:10662000A8403EE6E316F10409F409C508F414C6CF
:106630005FE6E516F10409F415C580E7E816F104F4
:1066400011F00C94A84088E893E00E94B78A92EE7B
:10665000E916F10411F40C94BF3D08F080C0BEEBC4
:10666000EB16F10409F410C660F5F7E7EF16F10434
:1066700009F44CC798F433E7E316F10409F439C779
:1066800008F432C755E7E516F10411F00C94A84060
:1066900060E0C8010E944CD90C94A84089E7E81634
:1066A000F10409F49FC708F497C7ACE8EA16F104AF
:1066B00009F4A1C5B1E9EB16F10409F498C70C94EB
:1066C000A840EDECEE16F10411F40C945D3CE0F4FE
:1066D00029ECE216F10411F40C94B33B38F448ECC5
:1066E000E416F10409F4F7C70C94A8405BECE51636
:1066F000F10411F40C94D53B8CECE816F10411F480
:106700000C94F33B0C94A84093EDE916F10411F4BA
:106710000C94013DB0F4BEECEB16F10411F00C94B6
:10672000A8403CEBA32E32E0B32E4DEFC42E44E044
:10673000D42E51EFE52E54E0F52E00E010E00C943D
:10674000C83CECEDEE16F10411F40C94993DFDED0E
:10675000EF16F10411F40C94A63D0C94A84022E924
:10676000E21621E0F20611F40C94B83E08F041C0A4
:106770004FE2E41641E0F40611F40C94B23E98F4B2
:106780008DE2E81681E0F80611F40C94103E10F04A
:106790000C94AF3EACE2EA16A1E0FA0611F40C94B8
:1067A000EA3D0C94A840B3E6EB16B1E0FB0611F409
:1067B0000C941E4058F4F0E3EF16F1E0FF0611F0E0
:1067C0000C94A8400E9403CD0C94A84020E9E21646
:1067D00021E0F20611F40C94B53E31E9E31631E004
:1067E000F30611F00C94A84081E00E944DBC0C947B
:1067F000A84046EFE41641E0F40611F40C94DC3FA7
:1068000040F58CEAE81681E0F80611F40C94BC3EE1
:1068100058F4AAE9EA16A1E0FA0611F00C94A8408F
:106820000E943BC80C94A840B4EFEB16B1E0FB0605
:1068300011F40C94C33FE5EFEE16E1E0FE0611F013
:106840000C94A8400E94F44D80E00E94074A0C94EA
:10685000A840F3E5EF16F3E0FF0611F40C94EB3FCC
:1068600048F437EFE31631E0F30611F40C94DF3F00
:106870000C94A84040EAE41643E0F40609F48AC206
:1068800057EEE51653E0F50611F40C9437400C94DE
:10689000A84080E50E9493BE882361F00E944ABF11
:1068A0006B017C01BB24B394672B682B692B31F4FB
:1068B000B12C04C0B12CC12CD12C760183E50E94EF
:1068C00093BE882399F00E947EBF6B017C01B110BA
:1068D0000FC0672B682B692B59F4D8018C91882342
:1068E00039F061E0C8010E944CD907C0BB20A9F370
:1068F00060E087E692E00E9437D983E090E09093D1
:106900002A0D8093290D81E08093DA070E94E3D459
:106910000E944D49C114D104E104F104E9F08091D1
:106920002D0D90912E0DA0912F0DB091300DC80E10
:10693000D91EEA1EFB1E0E94D75BDC01CB018C191D
:106940009D09AE09BF09B7FF1AC08091DA078823F5
:10695000B1F00E941F8BEFCF8091DA07882319F0E6
:106960000E941F8BF9CF80918A1160E0882319F073
:1069700088E592E002C084E492E00E9437D9109248
:10698000DA070C94A84084918F010F5F1F4F882372
:1069900021F00E945C87F801F6CF1092101410923B
:1069A0000F1440E050E0BA018BEB91E10E94308F70
:1069B0008BE1EBEBF1E1DE01159601900D928A95EA
:1069C000E1F78091B9119091BA119C838B8380E893
:1069D00093E09A83898340E050E0BE016F5F7F4F70
:1069E0008AE094E00E9450C6CE0101960E94AF4F0B
:1069F000E3E8F2E084918F010F5F1F4F882311F4C9
:106A00000C94A8400E945C87F801F4CF0E94E277C2
:106A10000C94A84010928A1110928B110C94A840EB
:106A200080918B11882319F081E080938A110E9454
:106A30007B790C94A84080918B11882311F40C94DD
:106A4000A84083E50E9493BE81110C94CE400C9423
:106A5000A84080918B11882351F1E3EAF2E0849100
:106A60008F010F5F1F4F882321F00E945C87F80180
:106A7000F6CF6091061470910714809108149091DC
:106A800009144AE00E9463878FE20E945C8760914C
:106A900002147091031480910414909105144AE03B
:106AA0000E9463878AE00E945C870C94A840E5EB13
:106AB000F2E084918F010F5F1F4F882311F40C9433
:106AC000A8400E945C87F801F4CF40E060E0C80174
:106AD0000E94B0740C94A84080918B11882311F40B
:106AE0000C94A84085E593E10E94ED8E85E593E145
:106AF0000E948C911092891110928811E09070047C
:106B0000F090710480918B11882311F40C94A840AB
:106B10000E9465741D8218861C821B8280E893E0A7
:106B20009A83898387EB91E19093D7118093D61153
:106B3000F70180818F3209F068C06FE270E0C70111
:106B40000E94C8EF8C010F5F1F4F9E012F5F3F4FC8
:106B500049010115110509F45EC06FE270E0C8013A
:106B60000E94C8EF6C01009709F456C00817190776
:106B700008F052C05C01A01AB10AA501B801CE010B
:106B800080960E94F1EFE0E2F0E0EC0FFD1FEA0DCD
:106B9000FB1D10828E01005E1F4FD8018D918D016B
:106BA000882319F00E945C87F8CF8AE00E945C87F6
:106BB0006091D6117091D7116115710511F06C5F5C
:106BC0007F4F21E0AE01405E5F4FCE0105960E94EF
:106BD0001294811112C0BE01605E7F4F8CEE92E074
:106BE0000E9455828EE20E945C878AE00E945C8748
:106BF000C4010E94AF4F0C94A8409092D71180928C
:106C0000D61186010F5F1F4FA4CF88ED91E19093BD
:106C1000D7118093D61187016091D6117091D71149
:106C20006115710511F06C5F7F4F18A21BA222E065
:106C3000A801CE0180960E941294811102C0F12C0D
:106C40001EC0CE0180960E94BEC58823C1F36CA5EC
:106C50007DA58EA59FA541E00E94BB82882379F384
:106C6000E8A9B0E2EB9FF0011124E551F14F309714
:106C700031F385EE80831BA20E947B82F82ECE0129
:106C800080960E94A94FFF2009F1E6ECF2E0849182
:106C90007F012FEFE21AF20A882321F00E945C871D
:106CA000F701F5CFD8018D918D01882319F00E944D
:106CB0005C87F8CF8AE00E945C87109206141092DD
:106CC0000714109208141092091418C0E4EDF2E0B1
:106CD00084917F01BFEFEB1AFB0A882321F00E9409
:106CE0005C87F701F5CFF80181918F01882319F0B6
:106CF0000E945C87F8CF8EE20E945C87CE010196ED
:106D00000E94AF4F0C94A84080918A1181110E947B
:106D1000E3D4009170041091710461E270E0C80145
:106D20000E94C8EF009719F08C010F5F1F4F80E59C
:106D30000E9493BE882349F0FF24F3948091660457
:106D4000909167048017910708F0F12C80918B11C6
:106D5000882311F40C94A8404F2D61E0C8010E94D3
:106D6000B07483E50E9493BE882349F08091660445
:106D7000909167048017910710F40C94DF40809184
:106D80008B11882319F081E080938A11F1100C9403
:106D9000A8404DCE81E08093891140E060E0C801B9
:106DA0000E94B0740C94A8400E9469C5ACE3CA2E3E
:106DB000D12CE12CF12CA70196010E9431EC762E0A
:106DC000672ECA01B901A70196010E9431EC6B013F
:106DD0007C01CA01B90128E130E040E050E00E94A6
:106DE00031EC4B015C01C9016DE671E00E9453EF8B
:106DF0008E010F5F1F4F6115710599F06F927F92A1
:106E0000DF92CF929F928F929F938F937F936F93F6
:106E100088E293E09F938F931F930F930E9405E85E
:106E200012C00097B1F06F927F92DF92CF929F9243
:106E30008F929F938F9388E193E09F938F931F93FB
:106E40000F930E9405E80FB6F894DEBF0FBECDBFCA
:106E500036C081149104A104B10479F06F927F923D
:106E6000DF92CF929F928F928CE093E09F938F93CB
:106E70001F930F930E9405E8E6CFC114D104E104EB
:106E8000F10469F06F927F92DF92CF9284E093E0F9
:106E90009F938F931F930F930E9405E8D4CF6F9217
:106EA0007F9280E093E09F938F931F930F930E94B4
:106EB00005E80F900F900F900F900F900F9060E0EB
:106EC000C8010E944CD9E8EBF3E484917F01BFEF45
:106ED000EB1AFB0A882321F00E945C87F701F5CFAB
:106EE000B8018CE393E00E9455828AE00E945C879F
:106EF0000C94A84083E50E9493BE882311F40C945F
:106F0000A8400E943DBF7C018F3F910519F010F011
:106F10000C94A84080E50E9493BE882339F00E941B
:106F20003DBF8C0197FF04C00C94A8400DE010E019
:106F3000D02EE0ECF2E0C801992721913191281779
:106F4000390731F023E0E031F207B9F70C94F14052
:106F5000E3E5F3E384918F010F5F1F4F882321F056
:106F60000E945C87F801F6CFE9E4F3E084918F0199
:106F70000F5F1F4F882311F40C94A8400E945C8778
:106F8000F801F4CF0E9437A60C94A8400E94BB7968
:106F90000C94A8400E9450C50C94A84088E690E04C
:106FA0000E94D5BE81110C94A8408091EE0D83FF04
:106FB00002C00C94A84083E50E9493BE8823D9F1B7
:106FC0000E943DBF909312088093110880E00E94B8
:106FD00013D10E943DBF863591053CF40E9450C5F7
:106FE00060E08FE593E00E9437D90E943DBF8C019D
:106FF000609198047091990480919A0490919B04F7
:107000000E94D3ED60177107B4F48BE993E09F936E
:107010008F938091690490E001969F938F9388E508
:1070200093E09F938F931F920E9460790FB6F8941C
:10703000DEBF0FBECDBF0E9422E20C94A8408EE4BA
:107040000E9493BE882311F40C94A8400E946DE224
:107050006093190D70931A0D80931B0D90931C0D66
:107060000C94A84083E50E9493BE882319F00E94E7
:10707000A6BE01C080E08093EE0DE8EBF3E48491BE
:107080008F010F5F1F4F882321F00E945C87F8015A
:10709000F6CFE1E8F3E084918F010F5F1F4F882363
:1070A00021F00E945C87F801F6CF8091EE0D8823D5
:1070B000A1F1F3E7CF2EF3E0DF2EE12CF12C20E05D
:1070C0008091EE0D90E00E2C02C0959587950A9464
:1070D000E2F780FF17C0BB24B394B20E222319F04D
:1070E0008CE20E945C87F60125913491F90184912C
:1070F00089010F5F1F4F882321F00E945C87980150
:10710000F5CF2B2DFFEFEF1AFF0A32E0C30ED11C93
:1071100045E0E416F104A1F63EC0EDE7F3E084910A
:107120008F010F5F1F4F8823B1F10E945C87F80128
:10713000F6CF8AE50E9493BE882309F472C70E94A5
:1071400055BF6B017C0120E030E040EA51EC0E9429
:10715000B5EE87FD59C720E030E040EA51E4C701B1
:10716000B6010E946CE818160CF44EC7C092750E5A
:10717000D092760EE092770EF092780EC0925F0277
:10718000D0926002E0926102F092620242E0C70196
:10719000B6010E94E3878AE00E945C87D9C71092FB
:1071A0000402D6C783E50E9493BE882359F00E944B
:1071B000A6BE80933A028D3308F4CAC78CE380934D
:1071C0003A02C6C7E8EBF3E484918F010F5F1F4FCB
:1071D000882321F00E945C87F801F6CF40913A02A3
:1071E00050E060E070E081E993E00E94ED818AE088
:1071F0000E945C87ADC78091EE0D83FF01C0A8C7D8
:1072000083E50E9493BE882309F4A2C70E943DBF74
:1072100090931608809315080E94E0D099C789E6DC
:1072200090E00E94D5BE811111C0E8E9F3E084919D
:107230008F010F5F1F4F882321F00E945C87F801A8
:10724000F6CF0E94ABA58AE00E945C8710922A0DBF
:107250001092290D0C946C448DE690E00E94D5BEEE
:10726000811176C78091EE0D83FD72C783E50E9480
:1072700093BE28968FAF28978111C8C782E50E94D8
:1072800093BE8111C3C764C78091EE0D83FD60C7B3
:1072900060E08CED93E00E9437D983E50E9493BEB5
:1072A00028968FAF289781110C94A84282E50E94FE
:1072B00093BE81110C94A8424BC783E50E9493BEF4
:1072C000882321F00E9461E28C0102C00FEF10E0E0
:1072D00080E50E9493BE882319F00E9461E202C0FB
:1072E00080E090E098010F3F110519F010F02FEFAA
:1072F00030E0892B09F02CC7309314082093130831
:1073000027C780E50E9493BE811105C01092140822
:10731000109213081DC70E9461E2892B09F018C75B
:10732000F5CF0E9446D10E94E3D40E94A68A109213
:1073300014081092130868EE73E080E090E00E9459
:107340007AD860E089EE93E00E9437D901C71092A5
:107350006E04FEC681E080936E04FBC683E50E9446
:1073600093BE882359F00E947EBF60933B027093C6
:107370003C0280933D0290933E02EAC688E50E945B
:1073800093BE81110C94184489E50E9493BE81112B
:107390000C9418448AE50E9493BE81110C94184401
:1073A00085E40E9493BE81110C9418440E94E3D49A
:1073B0000E94A68ACDC683E50E9493BE882309F465
:1073C000C7C60E947EBF6093310D7093320D8093CB
:1073D000330D9093340DBCC63CEBC32E32E0D32E5C
:1073E00041E2E42E4EE0F42E10E0D6018D916D01C5
:1073F0000E9493BE882309F46DC0133009F063C066
:107400000E9455BF4B015C0120E030E040EA51E4AE
:107410000E946CE887FF4EC0A501940160912D0E7B
:1074200070912E0E80912F0E9091300E0E946BED78
:107430002B013C019B01AC0160916D0E70916E0EB1
:1074400080916F0E9091700E0E94D1E860936D0E46
:1074500070936E0E80936F0E9093700EA301920145
:1074600060915D0E70915E0E80915F0E9091600E46
:107470000E94D1E860935D0E70935E0E80935F0E64
:107480009093600E6091FB0D7091FC0D8091FD0D4D
:107490009091FE0D0E9470E8A30192010E94D1E834
:1074A0000E94D8ED6093FB0D7093FC0D8093FD0D51
:1074B0009093FE0D80922D0E90922E0EA0922F0E84
:1074C000B092300E07C00E9455BFF70160837183F0
:1074D000828393831F5FF4E0EF0EF11C143009F0F8
:1074E00084CF0E948D9834C60E94E3D40E9482CD3E
:1074F0002FC6EBEFF3E084918F010F5F1F4F8823BE
:1075000009F426C60E945C87F801F5CFE5EFF4E0A8
:1075100084918F010F5F1F4F882321F00E945C87A9
:10752000F801F6CFEDEEF4E084918F010F5F1F4F6D
:10753000882321F00E945C87F801F6CF659B03C089
:107540000CE813E002C001E913E0D8018D918D0130
:10755000882319F00E945C87F8CF8AE00E945C873C
:10756000E5EEF4E084918F010F5F1F4F882321F037
:107570000E945C87F801F6CF8091030181FF03C070
:107580000CE813E002C001E913E0F80181918F01DA
:10759000882319F00E945C87F8CF8AE00E945C87FC
:1075A000EDEDF4E084918F010F5F1F4F882321F0F0
:1075B0000E945C87F801F6CF4B9B03C00CE813E0F8
:1075C00002C001E913E0D8018D918D01882309F4EF
:1075D000E2CD0E945C87F7CF81E080930B0280931D
:1075E0006804B7C510920B0210926804B1C583E518
:1075F0000E9493BE8823F1F00E943DBF182F823075
:10760000D0F0E3E5F3E384918F010F5F1F4F8823F0
:1076100021F00E945C87F801F6CFEFE0F5E084915D
:107620008F010F5F1F4F882309F492C50E945C876A
:10763000F801F5CF10E088E40E9493BE8823B1F0F2
:107640000E943DBFE12FF0E08A3A91053CF0853081
:10765000B1E09B072CF084E091E002C08AEA90E060
:10766000EE0FFF1FE35FF14F9183808386E40E945A
:1076700093BE8823A1F00E943DBFE12FF0E0EE0F02
:10768000FF1FEF5EF14F8F3F910519F014F08FEF60
:1076900090E097FF02C080E090E09183808382E4D5
:1076A0000E9493BE882309F453C50E943DBFE12F79
:1076B000F0E08530910534F0883891052CF087E8AA
:1076C00090E002C085E090E0EE0FFF1FE75FF14F12
:1076D000918380833DC588EC90E00E94D5BE8111E6
:1076E00037C584E40E9493BE8823D1F10E9455BF20
:1076F00011E020E030E0A9010E946CE8811101C096
:1077000010E01093790E112359F10091690410E0F3
:107710000E9455BF000F111F000F111FF801ED59F6
:10772000FD4F608371838283938320E030E0A90161
:10773000609163027091640280916502909166028B
:107740000E946CE881110CC080E090E0A0E4B0E4FD
:107750008093630290936402A0936502B0936602E3
:107760000E94CD84F5C4E9E3EE2EEEE0FE2E0CEB94
:1077700012E0F4E0DF2ED00EF80181918F010E941B
:1077800093BE882351F00E9455BF0E94D8EDD701C7
:107790006D937D938D939C931397B4E0EB0EF11C46
:1077A000D012EACF0E946097D3C461E5E62E6EE066
:1077B000F62E0CEB12E074E0D72ED00EF80181917A
:1077C0008F010E9493BE882341F00E9455BFD701CC
:1077D0006D937D938D939C931397B4E0EB0EF11C06
:1077E000D012ECCFB5C483E50E9493BE8823D9F0B4
:1077F0000E9455BFAB01BC014093710E5093720EB5
:107800006093730E7093740E4093310E5093320E4A
:107810006093330E7093340E8BE895E00E942382C0
:107820008AE00E945C8780E50E9493BE882399F0DD
:107830000E9455BFAB01BC014093710E5093720E74
:107840006093730E7093740E8EE695E00E9423820F
:107850008AE00E945C8782E50E9493BE882399F0AB
:107860000E9455BFAB01BC014093350E5093360EBC
:107870006093370E7093380E8FE495E00E94238258
:107880008AE00E945C8784E50E9493BE882309F405
:107890005FC40E9455BFAB01BC014093310E5093B1
:1078A000320E6093330E7093340E81E395E00E94A4
:1078B00023828AE00E945C874BC483E50E9493BECA
:1078C000882351F00E9455BF60934D0E70934E0E69
:1078D00080934F0E9093500E84E50E9493BE8823B0
:1078E00051F00E9455BF6093490E70934A0E8093E9
:1078F0004B0E90934C0E82E40E9493BE882351F06D
:107900000E944ABF6093EA0D7093EB0D8093EC0DDB
:107910009093ED0D88E50E9493BE882351F00E945C
:1079200055BF6093610E7093620E8093630E9093C7
:10793000640E89E50E9493BE882351F00E9455BFD2
:107940006093650E7093660E8093670E9093680E39
:107950008AE50E9493BE882351F00E9455BF609330
:10796000690E70936A0E80936B0E90936C0E85E493
:107970000E9493BE882309F4EBC30E9455BF609315
:107980006D0E70936E0E80936F0E9093700EE0C329
:10799000F50181915F010E9493BE882311F10E943D
:1079A00055BF2B013C01D7012D913D914D915C912B
:1079B0000E948EEC9B01AC01F60160817181828195
:1079C00093810E948FECD6016D937D938D939C9350
:1079D0001397F7014082518262827382C8010E942C
:1079E0003FBE0F5F1F4FF4E0CF0ED11C24E0E20E2C
:1079F000F11C0330110561F60E943D490E9482CDC1
:107A0000A7C3E8EBF3E484918F010F5F1F4F882336
:107A100021F00E945C87F801F6CF83E50E9493BEB7
:107A2000882321F00E9412BF80933102EBEDF5E034
:107A300084918F010F5F1F4F882321F00E945C8784
:107A4000F801F6CF80913102811103C0E7EDF5E036
:107A500002C0E3EDF5E084918F010F5F1F4F882393
:107A600021F00E945C87F801F6CFEBECF5E0849101
:107A70008F010F5F1F4F882321F00E945C87F80160
:107A8000F6CF4091E8075091E9076091EA077091BD
:107A9000EB0789EC95E00E9423824091EC0750911E
:107AA000ED076091EE077091EF0786EC95E00E947C
:107AB00023824091F0075091F1076091F207709195
:107AC000F30783EC95E00E942382EBEBF5E08491D1
:107AD0008F010F5F1F4F882321F00E945C87F80100
:107AE000F6CF4091250250912602609127027091B5
:107AF000280289EB95E00E9423824091290250914F
:107B00002A0260912B0270912C0286EB95E00E9474
:107B1000238240912D0250912E0260912F0270918C
:107B2000300283EB95E00E9423828AE00E945C870A
:107B30000FC383E50E9493BE882309F409C30E9402
:107B40003DBF909324028093230202C38DED90E009
:107B50000E94D5BE8111FCC283E50E9493BE88239A
:107B600009F4F6C20091690410E00E943DBF000FC5
:107B7000111FF801EF5DFD4F91838083E9C280E51D
:107B80000E9493BE882309F4E3C20E943DBF8C018A
:107B900083E50E9493BE882321F00E943DBF7C01B3
:107BA00003C0EE24EA94FE2CC7010196039708F067
:107BB000CFC217FDCDC2E0ECF2E0C80199272191B8
:107BC00031912817390709F4C3C233E0E031F307D4
:107BD000B1F75AC683E50E9493BE882319F00E942C
:107BE00061E202C084E091E099A388A380E50E944D
:107BF00093BE882349F00E9461E2893843E19407EB
:107C000028F088E893E102C088EE93E09A838983A4
:107C1000BE01605E7F4FCE0101960E942C7998C212
:107C200085E40E9493BE811110C080E50E9493BE3E
:107C3000882399F00E9455BF6093470270934802D1
:107C40008093490290934A0208C00E943DBF1816D3
:107C500019065CF7E3E5F3E371C089E40E9493BE83
:107C6000882381F00E9455BF2CEA35EC47E25EE3A1
:107C70000E94D1E860934F027093500280935102AA
:107C80009093520284E40E9493BE882381F00E9464
:107C900055BF2CEA35EC47E25EE30E946BED609342
:107CA0004B0270934C0280934D0290934E02E8EB8E
:107CB000F3E484918F010F5F1F4F882321F00E940E
:107CC0005C87F801F6CF40914702509148026091DD
:107CD000490270914A0283EF95E00E9423822CEAC8
:107CE00035EC47E25EE360914F0270915002809163
:107CF0005102909152020E946BEDAB01BC018FEEDC
:107D000095E00E9408822CEA35EC47E25EE3609140
:107D10004B0270914C0280914D0290914E020E9454
:107D2000D1E8AB01BC018BEE95E00E9408828AE0AD
:107D30000E945C870DC20E945C87F80184918F01CC
:107D40000F5F1F4F8111F7CF06EA13E0D8018D9125
:107D50008D01882309F41FCA0E945C87F7CF0E9417
:107D60008ACCF6C10E9472C8F3C10E94E3D4F0C16C
:107D700080E00E944DBCECC1E1EFF4E0FCAFEBAF62
:107D80008DEF282E84E0382E20EA34E021963FAF94
:107D90002EAF219700E010E021964EAD5FAD219708
:107DA000405A544029965FAF4EAF29972196AEAD09
:107DB000BFAD21978D912196BFAFAEAF219788239C
:107DC00009F4ACC0F801EB5DFD4F208131814281A7
:107DD0005381F801E851F84F60817181828193816C
:107DE0000E948FEC20E030E040E05FE30E94D1E8A9
:107DF0009B01AC01F10160817181828193810E94BC
:107E0000B5EE181634F4C8018859934C0E944749BE
:107E100003C060E070E0CB01D1018D909D90AD90EA
:107E2000BC90F801EB5CF24F20813181428153819B
:107E30000E948FEC9B01AC01C501B4010E948EEC45
:107E40006B017C0120E030E040EA51EC0E94B5EE8D
:107E500087FD35C020E030E040EA51E4C701B601BB
:107E60000E946CE818165CF1EBADFCAD40805180CF
:107E700062807380A7019601C301B2010E948EEC5B
:107E80006B017C01A30192010E948EEC9B01AC016D
:107E9000C501B4010E948FECD1016D937D938D9348
:107EA0009C931397EBADFCADC082D182E282F3824A
:107EB00029968EAD9FAD29970E943FBE2FC0E3E566
:107EC000F3E384918F010F5F1F4F882321F00E94FD
:107ED0005C87F801F6CFE5E1F6E084918F010F5F52
:107EE0001F4F882321F00E945C87F801F6CF61E0E4
:107EF00087E096E00E9437D90E94475888E290E0D8
:107F00009A83898388EC90E099A388A3BE016F5F70
:107F10007F4FCE0180960E942C791AC12BAD3CADCB
:107F20002C5F3F4F3CAF2BAF0C5F1F4F34E0230E55
:107F3000311C0C30110509F02FCF0E943D490E94E1
:107F400082CD60E087EF95E00E9437D983E992E027
:107F500099A388A304E610E01A830983BE01605E3A
:107F60007F4FCE0101960E942C798AEB92E099A373
:107F700088A31A830983BE01605E7F4FCE010196FC
:107F80000E942C79E5C0E3E5F3E384918F010F5F54
:107F90001F4F882321F00E945C87F801F6CFE3E3AE
:107FA000F6E084918F010F5F1F4F882309F4D0C042
:107FB0000E945C87F801F5CF0E94F44DC9C083E5AB
:107FC0000E9493BE882321F00E9412BF91E089276E
:107FD0000E94074ABDC0E8EBF3E484918F010F5F74
:107FE0001F4F882321F00E945C87F801F6CFEEE551
:107FF000F6E084918F010F5F1F4F882309F499C821
:108000000E945C87F801F5CFE7E4F6E084918F01E8
:108010000F5F1F4F882309F4BEC80E945C87F801D8
:10802000F5CF4091750E5091760E6091770E70915C
:10803000780E84E496E00E942382ADC8E3E5F3E382
:1080400084918F010F5F1F4F882321F00E945C876E
:10805000F801F6CFE8E6F6E084918F010F5F1F4F3D
:10806000882309F475C00E945C87F801F5CF81E090
:108070008093AA021092210883E50E9493BE882370
:1080800009F4FFC30E9412BF811162C0FAC3E092DB
:108090006A04E8EBF3E484918F010F5F1F4F88239C
:1080A00021F00E945C87F801F6CFB701772787E7B8
:1080B00096E00E943E828AE00E945C8749C080E090
:1080C00048C00E94DFBA83E50E9493BE882309F46A
:1080D00063C00E9412BFEE24E394F12C082FA30189
:1080E0009201C501B4010E9496BC6B017C012CEA8F
:1080F00035EC47E257E3C501B4010E948FECAB01B8
:10810000BC018CE392E00E9408822CEA35EC47E245
:1081100057E3C301B2010E948FECAB01BC0187E3BE
:1081200092E00E9408822CEA35EC47E257E3C7014F
:10813000B6010E948FECAB01BC0182E392E00E9489
:1081400008828AE00E945C870E94C5BA0E9482CDA4
:1081500081E010922A0D1092290D81111AC00C9401
:10816000412984918F010F5F1F4F882321F00E94C6
:108170005C87F801F6CF60912B0D70912C0D89E88A
:1081800096E00E94558282E20E945C878AE00E940B
:108190005C870E94A48DA0C381E09DCF0E946DE208
:1081A000AB01BC014093061450930714609308146C
:1081B0007093091485E593E10E94308FC9CF0E9426
:1081C0006DE2AB01BC014093061450930714609319
:1081D00008147093091485E593E10E94308F0C9484
:1081E000BF3661E08D2D0E949C5A6E2D8D2D0E9410
:1081F0006D5AB7018D2D0E94D85A0930110509F02A
:10820000A7CFF0921408E0921308A2CF0E943DBFBE
:10821000909312088093110880E00E9413D10E946D
:108220003DBF8635910544F40E9450C560E087EB60
:1082300093E00E9437D902C00E947B7960911108B7
:1082400070911208072E000C880B990B0E9472E89F
:10825000209198043091990440919A0450919B0484
:108260000E94B5EE1816B4F48BE993E09F938F93B8
:108270008091690490E001969F938F9380EB93E047
:108280009F938F931F920E9460790FB6F894DEBF80
:108290000FBECDBF0E9422E281E0809304021092C3
:1082A0002A0D1092290D23961CAE1DAE1EAE1FAED8
:1082B000239727961CAE1DAE1EAE1FAE27971BAE92
:1082C0002C961FAE2C979CE360969FAF6097ACE115
:1082D0006496AFAF6497B6E46896BFAF6897C12C59
:1082E000D12C70E8E72EEFEBFE2E812C912C54015F
:1082F0006091110870911208072E000C880B990BE1
:108300000E9472E8162F072F782E692E262F372FFE
:10831000482F592FB601C7010E946CE8882311F13C
:10832000209198043091990440919A0450919B04B3
:10833000612F702F872D962D0E946CE8881F88274B
:10834000881F8BAF2896EFAD2897EE2379F088230E
:1083500069F080910402882309F4FACE60E08BE989
:1083600093E06DC11C2D0D2D7E2C6F2C0E94D75BD0
:108370006B017C01DC01CB0127962CAD3DAD4EADF0
:108380005FAD2797821B930BA40BB50BB7FD47C0BE
:10839000D701C60188519C4FAF4FBF4F27968CAF76
:1083A0009DAFAEAFBFAF27970E94ABA5ECEAF3E05D
:1083B00084912F019FEF491A590A882321F00E94C6
:1083C0005C87F201F5CF81149104A104B104D1F0CE
:1083D000D501C401805F984DAF4FBF4FBC01CD01A7
:1083E0006C197D098E099F0928EE33E040E050E0CA
:1083F0000E9431ECCA01B9010E94C9878AE00E943B
:108400005C870DC0E9EAF3E084912F01AFEF4A1ACF
:108410005A0A882321F00E945C87F201F5CF0E945E
:108420001F8B3BD7609198047091990480919A04B6
:1084300090919B040E94D3ED072E000C880B990BA2
:108440000E9472E81B012C019B01AC01612F702F6F
:10845000872D962D0E948EEC9F7781149104A104A4
:10846000B10449F420E030E040E85FE30E946CE8AA
:1084700087FF0BC008C020E030E040E450E40E94D9
:10848000B5EE181614F446015701BBADBB2309F431
:1084900043C023962CAD3DAD4EAD5FAD2397211566
:1084A00031054105510541F0D701C601821B930BEF
:1084B000A40BB50BB7FD30C09101A2012C966FAD96
:1084C0002C9760967FAD609764968FAD64976896A1
:1084D0009FAD68970E948EEC20E030E040EC5FE3B7
:1084E0000E946CE887FD35CFD701C601805A9541BF
:1084F000AF4FBF4F23968CAF9DAFAEAFBFAF2397AB
:108500002C962FAE2C9760963FAE609764964FAE38
:10851000649768965FAE689780910402882309F497
:1085200018CF81149104A104B10429F4C12ED02ED6
:10853000E72CF62CDDCE90E1C91A97E2D90AE108C2
:10854000F108C818D908EA08FB08F7FE02CFEECFF9
:108550000E943DBF90931608809315080E94E0D0BA
:108560000E943DBF069714F00E947B7981E08093C2
:10857000040210922A0D1092290D80916A048093B2
:10858000690423961CAE1DAE1EAE1FAE2397279620
:108590001CAE1DAE1EAE1FAE27971BAE2C961FAE97
:1085A0002C97ACE36096AFAF6097BCE16496BFAF29
:1085B0006497E6E46896EFAF6897C12CD12C50E839
:1085C000E52E6FEBF62E812C912C5401609115084D
:1085D00070911608072E000C880B990B0E9472E808
:1085E000162F072F782E692E262F372F482F592F19
:1085F000B601C7010E946CE8882321F120919C04F8
:1086000030919D0440919E0450919F04612F702FE2
:10861000872D962D0E946CE8881F8827881F8BAFB6
:108620002896FFAD2897FF2389F0882379F0809161
:108630000402882309F48CCD60E08BEC93E00E9467
:1086400037D986CD1C2D0D2D7E2C6F2C0E94D75B2B
:108650006B017C01DC01CB0127962CAD3DAD4EAD0D
:108660005FAD2797821B930BA40BB50BB7FD47C0DB
:10867000D701C60188519C4FAF4FBF4F27968CAF93
:108680009DAFAEAFBFAF27970E94ABA5E8EDF3E07B
:1086900084912F019FEF491A590A882321F00E94E3
:1086A0005C87F201F5CF81149104A104B104D1F0EB
:1086B000D501C401805F984DAF4FBF4FBC01CD01C4
:1086C0006C197D098E099F0928EE33E040E050E0E7
:1086D0000E9431ECCA01B9010E94C9878AE00E9458
:1086E0005C870DC0E5EDF3E084912F01AFEF4A1AEE
:1086F0005A0A882321F00E945C87F201F5CF0E947C
:108700001F8BCBD560919C0470919D0480919E0439
:1087100090919F040E94D3ED072E000C880B990BBB
:108720000E9472E81B012C019B01AC01612F702F8C
:10873000872D962D0E948EEC9F7781149104A104C1
:10874000B10449F420E030E040E85FE30E946CE8C7
:1087500087FF0BC008C020E030E040E450E40E94F6
:10876000B5EE181614F446015701BBADBB2309F44E
:1087700043C023962CAD3DAD4EAD5FAD2397211583
:1087800031054105510541F0D701C601821B930B0C
:10879000A40BB50BB7FD30C09101A2012C966FADB3
:1087A0002C9760967FAD609764968FAD64976896BE
:1087B0009FAD68970E948EEC20E030E040EC5FE3D4
:1087C0000E946CE887FD33CFD701C601805A9541DE
:1087D000AF4FBF4F23968CAF9DAFAEAFBFAF2397C8
:1087E0002C962FAE2C9760963FAE609764964FAE56
:1087F000649768965FAE689780910402882309F4B5
:1088000016CF81149104A104B10429F4C12ED02EF5
:10881000E72CF62CDBCE90E1C91A97E2D90AE108E1
:10882000F108C818D908EA08FB08F7FE00CFEECF18
:108830000E94E3D488E50E9493BE882319F05F9AD2
:108840001092ED0489E50E9493BE882319F08A9A5C
:108850001092EE048AE50E9493BE882351F09FB7E0
:10886000F894809108018160809308019FBF109265
:10887000EF0485E40E9493BE882309F469CC129A20
:1088800067CC0E94C18D64CC0E94E3D4D02E60E0FE
:10889000802F0E949C5A4FEFE416F40659F4802F63
:1088A0000E9429DA31E020E0892B09F030E0032F23
:1088B000122F05C0EA94EF2861F000E010E08D2D42
:1088C0000E9429DA8017910709F442CC0E941F8B7D
:1088D000F6CF01E010E0F3CFCA58DF4F0FB6F8949F
:1088E000DEBF0FBECDBFDF91CF911F910F91FF90E3
:1088F000EF90DF90CF90BF90AF909F908F907F9040
:108900006F905F904F903F902F9008950895FC01D5
:10891000A681B7818281481B8581483018F0A80F55
:10892000B11D4770382F369536953695562F5770AE
:1089300080E890E002C0959587955A95E2F7439FAD
:10894000402D1124669566956695E62FF0E0E40FBC
:10895000F11DEA0FFB1F3081222311F0832B02C08F
:108960008095832380830895FB014181DC01129669
:108970002C911297421760F013962C91139724179D
:1089800038F0608115962C91621710F42481BFCFC6
:108990000895FC0180819281980F92832181921722
:1089A00060F494819F5F94839381890F821710F004
:1089B0008FEF820F838381E0089580E00895FC01AA
:1089C00012828081815083831482089580E008950B
:1089D0000B96FC01849108950A96FC0184910895F8
:1089E000FC0184910895FCDF882321F0823011F08E
:1089F00083E0089586E00895FC01E60FF11D84915F
:108A000090E0982F88273196E4918E0F911D08955C
:108A100068E0F2CF66E0F0CF81E008952F923F92B8
:108A20004F925F926F927F928F929F92AF92BF927E
:108A3000CF92DF92EF92FF920F931F93CF93DF932A
:108A400000D000D0CDB7DEB78C010E94D75BF80113
:108A5000C680D780E084F184C114D104E104F1041C
:108A600009F0F6C22485222309F460C3328521501F
:108A7000248721E0230F22874585241301C0128615
:108A8000F80124E0329FE00DF11D1124C684D78443
:108A9000E088F188F801C282D382E482F582DC01A9
:108AA000CB018C0D9D1DA11DB11D86839783A087D1
:108AB000B18784819581892B09F438C3FFB7FD8381
:108AC000F894F80122803380048115818091B702E7
:108AD000853221F08F3F09F0B8C205C0E3EEF0E522
:108AE00024912E83EDC085E28093B702E3EEF0E59A
:108AF000E491EF3F09F4A9C2E23009F474C054F5DF
:108B0000EE2309F453C0E13009F0D9C0109280007F
:108B10001092810080918100886080938100809113
:108B20008100816080938100EBEDFCE0E491F0E056
:108B3000EE0FFF1FEE57F34F8591949190937F04B2
:108B400080937E04E1E2FDE0E491E0937D0481E026
:108B50008E83B9C0E43009F48EC00CF468C0E530EF
:108B600009F0ADC0109220011092210180912101E5
:108B7000886080932101809121018160809321018F
:108B8000EBEDFCE0E491F0E0EE0FFF1FEE57F34F4A
:108B9000859194919093760480937504E1E2FDE0D1
:108BA000E491E093740425E02E838DC014BC15BCC1
:108BB00084B5826084BD85B5816085BDEBEDFCE048
:108BC000E491F0E0EE0FFF1FEE57F34F8591949183
:108BD0009093820480938104E1E2FDE0E491E093CC
:108BE00080041E8270C01092B0001092B10080917B
:108BF000B00082608093B0008091B100816080936A
:108C0000B100EBEDFCE0E491F0E0EE0FFF1FEE575A
:108C1000F34F859194919093871480938614E1E2A9
:108C2000FDE0E491E093881492E09E834CC01092A2
:108C30009000109291008091910088608093910043
:108C400080919100816080939100EBEDFCE0E491D4
:108C5000F0E0EE0FFF1FEE57F34F85919491909344
:108C60007C0480937B04E1E2FDE0E491E0937A04EC
:108C7000E3E0EE8328C01092A0001092A100809142
:108C8000A10088608093A1008091A1008160809301
:108C9000A100EBEDFCE0E491F0E0EE0FFF1FEE57DA
:108CA000F34F859194919093790480937804E1E255
:108CB000FDE0E491E0937704F4E0FE8304C0EE83EA
:108CC0008E8187FDC2C12101612C712C61E085E29A
:108CD0000E949C5A4801A12CB12C8E818D7F09F0F5
:108CE000BDC060E072E18AE790E0A50194010E94B6
:108CF00053EC29833A834B835C8369017A0191E0C9
:108D0000C91AD108E108F108EFEFCE16D104E10449
:108D1000F10409F008F44DC060E472E48FE090E0E3
:108D2000A50194010E9453EC69017A01F1E0CF1A88
:108D3000D108E108F1082E81223001F58FEFC81625
:108D4000D104E104F10409F008F4EEC160E970ED2A
:108D500083E090E0A50194010E9453EC69017A013F
:108D600091E0C91AD108E108F108EFEFCE16D1045D
:108D7000E104F10409F0E0F583E069C0FFEFCF16EC
:108D8000D104E104F104B9F0B0F068E478EE81E0D8
:108D900090E0A50194010E9453EC69017A0181E001
:108DA000C81AD108E108F1089E81992309F49AC1F3
:108DB00090C181E001C082E09E819923A1F047C06B
:108DC00089819A81AB81BC812AE0B595A795979559
:108DD00087952A95D1F76C017D01E1E0CE1AD10883
:108DE000E108F10885E095B5987F892B85BDA1C084
:108DF00068E478EE81E090E0A50194010E9453ECD4
:108E000069017A01F1E0CF1AD108E108F1082FEFEA
:108E1000C216D104E104F10409F008F428C164E2A7
:108E200074EF80E090E0A50194010E9453EC690189
:108E30007A01E1E0CE1AD108E108F108FFEFCF1680
:108E4000D104E104F10411F008F013C185E0909120
:108E5000B100987F892B8093B1006BC060E072E114
:108E60008AE790E0A50194010E9453EC69017A0120
:108E7000E1E0CE1AD108E108F108C114D104F1E013
:108E8000EF06F10488F068E478EE81E090E0A50157
:108E900094010E9453EC69017A0181E0C81AD1085B
:108EA000E108F10883E001C081E09E81913071F416
:108EB00090918100987F892B8093810045284628D6
:108EC0004728D9F52FEF3FEFA90168C0EE81E330C5
:108ED00071F490919100987F892B8093910045289F
:108EE0004628472851F52FEF3FEFA90179C0FE81B1
:108EF000F43071F49091A100987F892B8093A100A8
:108F0000452846284728C9F42FEF3FEFA9017AC02A
:108F10002E81253071F490912101987F892B8093C7
:108F2000210145284628472841F42FEF3FEFA901AA
:108F30007BC045284628472869F09801220F331F37
:108F4000D1010E947FEC28EE33E040E050E00E9427
:108F500031EC03C02FEF3FEFA9018E81823081F108
:108F60002CF4882361F08130C9F06FC09E81943069
:108F700009F448C0ACF1953009F456C066C0C7BCCE
:108F80002093930430939404409395045093960453
:108F900080916E00826080936E0057C0D0928900ED
:108FA000C092880020938F043093900440939104E2
:108FB0005093920480916F00826080936F0045C04F
:108FC000C092B3002093891430938A1440938B1479
:108FD00050938C148091700082608093700035C033
:108FE000D0929900C092980020938B0430938C0407
:108FF00040938D0450938E04809171008260809321
:10900000710023C0D092A900C092A80020938704C9
:10901000309388044093890450938A0480917200AD
:1090200082608093720011C0D0922901C092280101
:1090300020938304309384044093850450938604E2
:1090400080917300826080937300ED81EFBF6EC0EA
:10905000DC01CB018C199D09AE09BF09B7FD66C0C3
:109060004098F80116821782108611865FC084E04E
:10907000EECE62E17AE780E090E0A50194010E94E3
:1090800053EC69017A0181E0C81AD108E108F108BE
:109090009FEFC916D104E104F104C9F0C0F0898141
:1090A0009A81AB81BC815AE0B595A7959795879534
:1090B0005A95D1F76C017D0121E0C21AD108E1086F
:1090C000F1088E81882309F48DCE87E0C0CE86E03A
:1090D00073CEEFEFCE16D104E104F10409F048F6A7
:1090E00084E06ACE8FEFC816D104E104F104D1F018
:1090F000C8F062E17AE780E090E0A50194010E9467
:1091000053EC69017A01F1E0CF1AD108E108F108C6
:109110002FEFC216D104E104F10411F008F050CE93
:1091200084E061CE83E05FCE82E091CE26960FB6DA
:10913000F894DEBF0FBECDBFDF91CF911F910F918D
:10914000FF90EF90DF90CF90BF90AF909F908F9067
:109150007F906F905F904F903F902F900895209157
:10916000A30430E0F901E35FFA4F80832F5F3F4FA4
:10917000237033272093A3048091AF068F5F8093E1
:10918000AF060895CF93FC0180818B33A1F08091CD
:10919000AF06843080F4C62FBF018091A30420E67F
:1091A000829FC0011124825D9A4F0E94DCEF8C2FB8
:1091B000D6DF81E001C080E0CF910895DF92EF9289
:1091C000FF920F931F93CF93DF93CDB7DEB76E97C8
:1091D0000FB6F894DEBF0FBECDBF6091220870912C
:1091E00023086115710501F14DE150E0CE010196B2
:1091F0007C010E94DCE71E8EF7018F010E191F090A
:10920000D190DD2019F09AE0D912F7CFF701E00FE5
:10921000F11F108260E0C701B5DF882329F0C70184
:109220000E94888A811109C081E020912208309132
:109230002308232BA1F480E012C0DD2049F00F5F4A
:109240001F4F8091220890912308080F191F02C018
:1092500000E010E01093230800932208E5CF6E96FB
:109260000FB6F894DEBF0FBECDBFDF91CF911F9137
:109270000F91FF90EF90DF90089529E035E045E0F1
:1092800055E061E075E08DEF94E00C94CA97FC0125
:10929000659175918591949108950E94D75B609333
:1092A0002D0D70932E0D80932F0D9093300D0895FA
:1092B0000F931F93CF93DF93E0911914F0911A1439
:1092C00042815381648175811416150616061706AE
:1092D00004F52091F40C20FF1CC03CB120917304D4
:1092E00032953695377041E03427832F81702E7F79
:1092F000822B80937304909172049170892349F0BA
:1093000080912D05816080932D0580E090E00E9482
:10931000A2D4E0911914F0911A1486819781A08546
:10932000B185181619061A061B0654F58091F40C1F
:1093300081FF26C08091030120917304422F50E0E9
:10934000869591E08927082F017010E022273327A6
:10935000201B310B2427352722703327242735275C
:1093600020937304809172048270282349F08091C5
:109370002D05826080932D0581E090E00E94A2D4AB
:10938000E0911914F0911A1482859385A485B5850E
:10939000181619061A061B068CF58091F40C82FF2C
:1093A0002DC08091F004882349F199B18091730414
:1093B000282F30E0892F86958695869591E089271C
:1093C0008170C82F80E0D82F882799278C1B9D0B90
:1093D0008227932784709927822793278093730489
:1093E000909172049470892349F080912D058460D6
:1093F00080932D0582E090E00E94A2D480917304B6
:1094000080937204DF91CF911F910F910895AF92D5
:10941000BF92CF92DF92EF92FF920F931F93CF9361
:10942000C82F882319F0E7EFF8E00CC0E8EBF3E46D
:1094300084918F010F5F1F4F8823A9F30E945C87DF
:10944000F801F6CF84918F010F5F1F4F882321F021
:109450000E945C87F801F6CF8AE00E945C87C11108
:109460002CC0E8EBF3E484918F010F5F1F4F88233A
:1094700021F00E945C87F801F6CFE4EEF8E08491D9
:109480008F010F5F1F4F882321F00E945C87F80136
:10949000F6CF8091790E882321F08AE00E945C87C4
:1094A0003AC0E9EDF8E084918F010F5F1F4F8823E8
:1094B00091F10E945C87F801F6CF409163025091D0
:1094C0006402609165027091660280ED98E00E94EE
:1094D00023828AE00E945C878091790E811127C0E7
:1094E000CC2319F0E5ECF8E00CC0E8EBF3E4849150
:1094F0008F010F5F1F4F8823A9F30E945C87F8013B
:10950000F6CF84918F010F5F1F4F882381F00E9457
:109510005C87F801F6CFE8EBF3E484918F010F5FED
:109520001F4F882351F20E945C87F801F6CFC111CA
:1095300024C0E8EBF3E484918F010F5F1F4F882371
:1095400021F00E945C87F801F6CFE4EBF8E084910B
:109550008F010F5F1F4F882321F00E945C87F80165
:10956000F6CFE8EBF3E484918F010F5F1F4F882360
:1095700021F00E945C87F801F6CF4091210E5091B6
:10958000220E6091230E7091240E8CEA98E00E94C6
:1095900023824091250E5091260E6091270E7091E6
:1095A000280E89EA98E00E9423824091290E50916A
:1095B0002A0E60912B0E70912C0E86EA98E00E9484
:1095C000238240912D0E50912E0E60912F0E70919E
:1095D000300E83EA98E00E9423828AE00E945C8732
:1095E000C11124C0E8EBF3E484918F010F5F1F4F9A
:1095F000882321F00E945C87F801F6CFE5E8F8E0C7
:1096000084918F010F5F1F4F882321F00E945C8798
:10961000F801F6CFE8EBF3E484918F010F5F1F4F61
:10962000882321F00E945C87F801F6CF4091510E0B
:109630005091520E6091530E7091540E8CE798E049
:109640000E9423824091550E5091560E6091570E04
:109650007091580E89E798E00E9423824091590E3C
:1096600050915A0E60915B0E70915C0E86E798E007
:109670000E94238240915D0E50915E0E60915F0EBC
:109680007091600E83E798E00E9423828AE00E9436
:109690005C87C11124C0E8EBF3E484918F010F5F74
:1096A0001F4F882321F00E945C87F801F6CFE1E587
:1096B000F8E084918F010F5F1F4F882321F00E94F3
:1096C0005C87F801F6CFE8EBF3E484918F010F5F3C
:1096D0001F4F882321F00E945C87F801F6CF40914C
:1096E000390E50913A0E60913B0E70913C0E88E419
:1096F00098E00E94ED8140913D0E50913E0E6091A8
:109700003F0E7091400E85E498E00E94ED814091FB
:10971000410E5091420E6091430E7091440E82E4CE
:1097200098E00E94ED814091450E5091460E609167
:10973000470E7091480E8FE398E00E94ED818AE019
:109740000E945C87C11124C0E8EBF3E484918F018F
:109750000F5F1F4F882321F00E945C87F801F6CF2E
:10976000E5EFF7E084918F010F5F1F4F882321F011
:109770000E945C87F801F6CFE8EBF3E484918F0157
:109780000F5F1F4F882321F00E945C87F801F6CFFE
:109790004091710E5091720E6091730E7091740E23
:1097A0008CEE97E00E9423824091350E5091360E48
:1097B0006091370E7091380E89EE97E00E942382F7
:1097C0004091310E5091320E6091330E7091340EF3
:1097D00086EE97E00E9423828AE00E945C87C11196
:1097E00024C0E8EBF3E484918F010F5F1F4F8823BF
:1097F00021F00E945C87F801F6CFE2E7F7E0849160
:109800008F010F5F1F4F882321F00E945C87F801B2
:10981000F6CFE8EBF3E484918F010F5F1F4F8823AD
:1098200021F00E945C87F801F6CF40914D0E5091D7
:109830004E0E60914F0E7091500E89E697E00E9497
:1098400023824091490E50914A0E60914B0E7091C7
:109850004C0E86E697E00E9423824091EA0D5091DB
:10986000EB0D6091EC0D7091ED0D83E697E00E9499
:10987000ED814091610E5091620E6091630E709186
:10988000640E80E697E00E9423824091650E50911D
:10989000660E6091670E7091680E8DE597E00E94EC
:1098A00023824091690E50916A0E60916B0E709107
:1098B0006C0E8AE597E00E94238240916D0E5091D4
:1098C0006E0E60916F0E7091700E87E597E00E94AA
:1098D00023828AE00E945C87C11124C0E8EBF3E494
:1098E00084918F010F5F1F4F882321F00E945C87B6
:1098F000F801F6CFE9E4F7E084918F010F5F1F4F85
:10990000882321F00E945C87F801F6CFE8EBF3E4AE
:1099100084918F010F5F1F4F882321F00E945C8785
:10992000F801F6CF4091F1045091F2046091F304F4
:109930007091F40480E497E00E9423824091F50442
:109940005091F6046091F7047091F8048DE397E06C
:109950000E9423824091F9045091FA046091FB0423
:109960007091FC048AE397E00E9423828AE00E94BF
:109970005C87CC2379F08DE0A82E8EE0B82E99E09C
:10998000C92E9EE0D92E21E1E22E2EE0F22E00E03B
:1099900010E024C0E8EBF3E484918F010F5F1F4FC8
:1099A000882321F00E945C87F801F6CFEDE1F7E013
:1099B00084918F010F5F1F4F882321F00E945C87E5
:1099C000F801F6CFE8EBF3E484918F010F5F1F4FAE
:1099D000882389F20E945C87F801F6CFB80184E100
:1099E00097E00E943E82F501619171915F0181E1F2
:1099F00097E00E943E82F601619171916F018EE0C5
:109A000097E00E943E82F701619171917F018BE0A6
:109A100097E00E943E828AE00E945C870130110537
:109A200019F001E010E0DACFC11124C0E8EBF3E453
:109A300084918F010F5F1F4F882321F00E945C8764
:109A4000F801F6CFECEFF6E084918F010F5F1F4F26
:109A5000882321F00E945C87F801F6CFE8EBF3E45D
:109A600084918F010F5F1F4F882321F00E945C8734
:109A7000F801F6CF409147025091480260914902A7
:109A800070914A0283EF96E00E9423822CEA35EC23
:109A900047E25EE360914F02709150028091510263
:109AA000909152020E946BEDAB01BC0180EF96E0F9
:109AB0000E9408822CEA35EC47E25EE360914B029B
:109AC00070914C0280914D0290914E020E94D1E81B
:109AD000AB01BC018DEE96E00E9408828AE00E94F4
:109AE0005C87C1110CC0E8EBF3E484918F010F5F38
:109AF0001F4F882321F00E945C87F801F6CF409128
:109B0000B3025091B4026091B5027091B60284EE36
:109B100096E00E9423822CEA35EC47E25EE36091F6
:109B2000AF027091B0028091B1029091B2020E9496
:109B30006BEDAB01BC0181EE96E00E9408822CEA3D
:109B400035EC47E25EE36091AB027091AC0280912C
:109B5000AD029091AE020E94D1E8AB01BC018EED46
:109B600096E00E9408828AE00E945C87C11124C0AE
:109B7000E8EBF3E484918F010F5F1F4F882321F0FE
:109B80000E945C87F801F6CFE8ECF6E084918F0143
:109B90000F5F1F4F882321F00E945C87F801F6CFEA
:109BA000E8EBF3E484918F010F5F1F4F882321F0CE
:109BB0000E945C87F801F6CF4091750E5091760EA9
:109BC0006091770E7091780E8FEB96E00E94238261
:109BD0008AE0CF911F910F91FF90EF90DF90CF908F
:109BE000BF90AF900C945C87AF92BF92CF92DF9200
:109BF000EF92FF920F931F93CF93DF93CDB7DEB712
:109C0000E0970FB6F894DEBF0FBECDBF80E1E0E174
:109C1000F3E0DE01919601900D928A95E1F780E1E3
:109C2000E0E2F3E0DE01519601900D928A95E1F7B2
:109C300080E1E0E3F3E0DE01119601900D928A9558
:109C4000E1F7DE01919661E27EE0AE014F5E5F4F8B
:109C500021E53EE0CE0101965C0189E39EE08E01A4
:109C60000F5C1F4FCD90DD90ED90FD90FB01C192F8
:109C7000D192E192F192BF01FA01C190D190E190AD
:109C8000F190AF01F901C192D192E192F1929F015D
:109C9000F501C190D190E190F1905F01FC01C1927A
:109CA000D192E192F192CF01A017B107D9F680E0ED
:109CB00090E8ABEBB4E48093710E9093720EA09396
:109CC000730EB093740E8093350E9093360EA0935E
:109CD000370EB093380E80E090E8ABE3B5E48093A4
:109CE000310E9093320EA093330EB093340E109237
:109CF0004D0E10924E0E10924F0E1092500E80E2AA
:109D00009EE4A0E0B0E08093EA0D9093EB0DA09369
:109D1000EC0DB093ED0D1092490E10924A0E109278
:109D20004B0E10924C0E80E090E0A0E0B1E48093E6
:109D3000610E9093620EA093630EB093640E8093B5
:109D4000650E9093660EA093670EB093680E8DEC2F
:109D50009CECACECBEE38093690E90936A0EA093EA
:109D60006B0EB0936C0E80E090E0A0EAB0E48093BC
:109D70006D0E90936E0EA0936F0EB093700E8CE0EC
:109D8000E1EFF4E0DF011D928A95E9F71092750E7C
:109D90001092760E1092770E1092780E87ED90E06A
:109DA00090930E0E80930D0E80EF90E09093100E26
:109DB00080930F0E86E490E090930A0E8093090E34
:109DC0008EE690E090930C0E80930B0E1092120E84
:109DD0001092110E1092140E1092130E86EF98E24C
:109DE000A1E0B2E48093470290934802A093490215
:109DF000B0934A0284E795EDA7E1BFE380934F0259
:109E000090935002A0935102B093520280E590E0EB
:109E1000ACEDB3E480934B0290934C02A0934D02BF
:109E2000B0934E0286EF98EAA0EBB3E48093B302BE
:109E30009093B402A093B502B093B60283EA9FE573
:109E4000A6E3B1E48093AF029093B002A093B10275
:109E5000B093B20286E893E2ABE2B5E48093AB0242
:109E60009093AC02A093AD02B093AE021092790E23
:109E700080E090E0A0E4B0E48093630290936402F9
:109E8000A0936502B093660210920B0210926804D0
:109E90000E9460970E948D980E94CD8480E090E09F
:109EA0000E943FBE81E090E00E943FBE82E090E0D1
:109EB0000E943FBE8091750E9091760EA091770E14
:109EC000B091780E80935F0290936002A09361023C
:109ED000B0936202E8EBF3E484918F010F5F1F4FB0
:109EE000882321F00E945C87F801F6CFECE9F6E0C8
:109EF00084918F010F5F1F4F882321F00E945C87A0
:109F0000F801F6CFE0960FB6F894DEBF0FBECDBFD6
:109F1000DF91CF911F910F91FF90EF90DF90CF9045
:109F2000BF90AF900895FC0120E03EE2DB014C9130
:109F3000403241F0283011F430833196DB014C91EE
:109F4000408331962F5F6F5F7F4F2B3079F7108200
:109F50000895FC01238121110C948C91089520E82F
:109F600033E0FC01318320830496F3CFCF92DF925C
:109F7000FF920F931F93CF93DF931F921F92CDB742
:109F8000DEB76901DB0112960D911C9113974233E4
:109F900009F471C0B8F4453109F47AC0473109F4C5
:109FA0008BC0443109F0A1C0D80115962C911597AA
:109FB0001696ED91FC911797CF01820F911D820F9C
:109FC000911D5EC0463409F487C0473409F488C047
:109FD0004B3309F08AC0F90181819381913029F0D6
:109FE000933031F4482F885004C048E0480F01C036
:109FF000482F21E0D80113963C91381708F420E04F
:10A0000031E0F8015281451708F430E051E048177B
:10A0100008F050E0822F852B382319F4252309F40A
:10A0200064C0D6011296FC90913051F030F092301D
:10A0300049F0933051F42FEF09C020E031E007C020
:10A0400021E004C020E03FEF02C020E030E0F7FE56
:10A0500008C0B601C8012A8339830E94B4443981FB
:10A060002A81F6018081830F80838181820F818321
:10A07000FF0C69F73AC0B901C8010E94B44435C069
:10A080001192E817F907E1F7C8010E94DF442DC0DB
:10A09000C8010E94C944882349F1F801258106803E
:10A0A000F781E02DCF01820F911D820F911D11923A
:10A0B000E817F907E1F719C0D9011C92F80182816C
:10A0C00011968C9311978581815012968C931297DB
:10A0D000838113968C9309C0D80115968C9103C087
:10A0E000D80111968C91F601808381E00F900F903A
:10A0F000DF91CF911F910F91FF90DF90CF90089546
:10A10000DB01ED91FC9119948F929F92BF92CF92B7
:10A11000DF92EF92FF920F931F93CF93DF931F92E3
:10A12000CDB7DEB74C01062FF42E122F522FE62E9C
:10A13000E20EBB24BA946C018CE1C80ED11C8E2DAA
:10A14000851B583078F0F40162817381848FF58E1D
:10A15000178EB68E96014BE3C4015983D1DF598126
:10A160005850EDCF812F887F080F212F277019F1CC
:10A1700087E02827F40162817381048FF58E178EA2
:10A180002F5F27708FEF90E001C0880F2A95EAF7C4
:10A19000868F9401245E3F4F4BE3C4010F90DF9103
:10A1A000CF911F910F91FF90EF90DF90CF90BF90D4
:10A1B0009F908F90A5CF0F90DF91CF911F910F911E
:10A1C000FF90EF90DF90CF90BF909F908F90089579
:10A1D000EF92FF920F931F93CF93DF937C01D62FC3
:10A1E000122FC42F040F212F4C2F6D2FC7018CDF8E
:10A1F000CF5F0C13F8CFDF91CF911F910F91FF909C
:10A20000EF900895EF92FF920F931F93CF93DF93F8
:10A210001F92CDB7DEB78C01DC011296ED90FC9059
:10A220001397D196ED91FC91D29782E0199520E099
:10A2300030E04AE0B701C80163DFF82ED801D196BB
:10A24000ED91FC91D29783E01995D801D196ED91CB
:10A25000FC91D29780E01995FF2081F1F80162818D
:10A2600073819E012F5F3F4F46E4C80149DF89811A
:10A27000D8018C9312966D917C9113979E012F5F5C
:10A280003F4F47E4C8013CDF8981F8018183628147
:10A29000738120E030E048E4C80132DFD8011B962A
:10A2A0008C931B9798012D5C3F4F12966D917C917A
:10A2B000139747E1C80124DF81E001C080E00F90DF
:10A2C000DF91CF911F910F91FF90EF90089588E259
:10A2D00090E00197F1F708952EE93FE0009729F00B
:10A2E000F9013197F1F70197F9CF08950F93FC0128
:10A2F0000150040F84A996A9941718F0081728F4A0
:10A3000002C0081750F0041740F42150260F83A90B
:10A3100095A9961720F4281720F480E007C0281785
:10A3200020F481E0261710F0F8CF81E00F91089516
:10A33000DF92EF92FF920F931F93CF93DF93EC0185
:10A34000162FF42EE22ED2DF882329F02E2D4F2D4A
:10A35000612FCE013DDFDF91CF911F910F91FF90D3
:10A36000EF90DF9008952F923F925F926F927F92CD
:10A370008F929F92AF92BF92CF92DF92EF92FF9215
:10A380000F931F93CF93DF931F92CDB7DEB71C01BE
:10A39000C62E142FD22EDC011496ED90FC9015974A
:10A3A000C7010E94F044082FF101848195810E9429
:10A3B000F344982E013019F48FE0A82E02C0AA248D
:10A3C000AA94D10114968D919C9115970E94EC440A
:10A3D000082FF101848195810E94E844B82ED101B3
:10A3E00014968D919C9115970E940845B0E6BD1575
:10A3F00030F4009721F0E80EF91E01E611C0F101DA
:10A40000848195810E940A45F0E4FD1530F400979F
:10A4100021F0E80EF91E01E403C021E1E20EF11C77
:10A42000BD1480F4D10150961C92509753961C9203
:10A43000539754961C92549751961C92519752964A
:10A440001C92C5C0B01670F3892D90E0F7012491DD
:10A450002F3F21F4FFEFEF1AFF0A5AC00D114FC032
:10A46000D10114968D919C9115970E94F04497010B
:10A470002F5F3F4FF701882311F08230E1F4849180
:10A48000D10153968C935397F901249154962C93B0
:10A490005497F7013396E4915096EC935097F70157
:10A4A0003496E4915196EC935197F7013596E491E7
:10A4B0005296EC9320C08491982F9F709250D101B6
:10A4C00052969C93529782958F7051968C93519788
:10A4D000F9012491822F8F7054968C935497229572
:10A4E0002F7053962C935397F7013296E491E2958F
:10A4F000EF705096EC93E114F10479F468C0F70121
:10A500003296E491EA219C012E0F311DE20EF31EDA
:10A510000B1509F487CF0F5F99CFF10184819581E5
:10A520000E94F344B82ED10153969C9053975496B1
:10A53000DC90549751968C915197C80E52969C91ED
:10A540009D0D512E591A0D2D292D452D6C2DC10112
:10A55000CDDE8823C9F1C7018B0D911D5C0187E019
:10A56000890DF82EF694F694F694D50C41019CE1F1
:10A57000890E911C6F2C712C5D1431F15C2D8501BD
:10A58000802F8A198F15E0F4F8018491D101129679
:10A590006D917C9113975C965C935C975D965C9251
:10A5A0005D975F961C925F975E968C9394014BE348
:10A5B000C1015983A5DD0F5F1F4F5981585FE0CF5F
:10A5C000A60CB71C5394D8CFF101808901C080E05C
:10A5D0000F90DF91CF911F910F91FF90EF90DF903F
:10A5E000CF90BF90AF909F908F907F906F905F9033
:10A5F0003F902F9008954F925F926F927F928F922B
:10A600009F92AF92BF92CF92DF92EF92FF920F9301
:10A610001F93CF93DF93CDB7DEB762970FB6F89451
:10A62000DEBF0FBECDBF1092D7070E94D75B00914F
:10A63000C9041091CA042091CB043091CC046B0161
:10A640007C01C01AD10AE20AF30AF7FC13C0209178
:10A65000C80420952093C804DC01CB018A549C4F88
:10A66000AF4FBF4F8093C9049093CA04A093CB040B
:10A67000B093CC04FF24F3948091C804811101C0ED
:10A68000F12C0E94DBD880913011853198F4FF20A5
:10A6900049F08091130890911408892B19F003E573
:10A6A0001AE002C006E319E023E14FE061E089E02F
:10A6B0000E948DC2809130118D3108F091C1883097
:10A6C000D0F56091110870911208072E000C880BCC
:10A6D000990B0E9472E820E030E040E05FE30E94C6
:10A6E0008FEC0E94D3ED7C876B87643671052CF468
:10A6F0006A30710524F426E003C022E101C02CE099
:10A7000082E190E0821B910997FD019695958795CE
:10A710009195819591098B5F8093331187E08093A8
:10A720003411CE010B960E9441D80E94285F83E32A
:10A7300099E00E941B5F809130118D3108F044C078
:10A7400080913211853108F43FC060919804709176
:10A75000990480919A0490919B040E94D3ED072E56
:10A76000000C880B990B0E9472E820E030E040E07A
:10A770005FE30E948FEC0E94D3ED9B017E876D8783
:10A78000643671050CF066C32A3031050CF060C3E5
:10A7900026E082E190E0821B910997FD0196959554
:10A7A00087959195819591098B5F809333118CE109
:10A7B00080933411CE010D960E9441D80E94285FEB
:10A7C00083E399E00E941B5F80913011853138F559
:10A7D00080913211813118F1609111087091120845
:10A7E000072E000C880B990B0E9472E820919804A8
:10A7F0003091990440919A0450919B040E94B5EEC7
:10A8000018160CF029C310921C1102E022E041E15D
:10A810006DE08CEF90E18CDD81E080931C118091E4
:10A8200030118830D0F56091150870911608072E08
:10A83000000C880B990B0E9472E820E030E040E0A9
:10A840005FE30E948FEC0E94D3ED788B6F876436B4
:10A8500071052CF46A30710524F426E003C022E16E
:10A8600001C02CE082E190E0821B910997FD0196E6
:10A87000959587959195819591098F5A809333117C
:10A8800087E080933411CE010F960E9441D80E9438
:10A89000285F83E399E00E941B5F809130118D3126
:10A8A00008F044C080913211853108F43FC06091B6
:10A8B0009C0470919D0480919E0490919F040E943D
:10A8C000D3ED072E000C880B990B0E9472E820E054
:10A8D00030E040E05FE30E948FEC0E94D3ED9B01EB
:10A8E0007A8B698B643671050CF0C0C22A30310551
:10A8F0000CF0BAC226E082E190E0821B910997FD3C
:10A900000196959587959195819591098F5A809398
:10A9100033118CE180933411CE0141960E9441D8CD
:10A920000E94285F83E399E00E941B5F80913011B1
:10A93000853138F580913211813118F16091150817
:10A9400070911608072E000C880B990B0E9472E874
:10A9500020919C0430919D0440919E0450919F044D
:10A960000E94B5EE18160CF083C210921C1102E082
:10A9700022E042E168E58CEF90E1DADC81E080934F
:10A980001C11809130118C3158F580913211843135
:10A9900038F120911308309114082F5F3F4F44E69F
:10A9A000429FC001439F900D112497FF02C0815028
:10A9B0009F4F292F392F330F330B3A832983232BB2
:10A9C00079F088E6809333118BE180933411CE01C6
:10A9D00001960E9441D80E94285F85E20E9470740F
:10A9E00080913011843328F4809132118A3208F03A
:10A9F00047C280913011853328F480913211813320
:10AA000008F063C280918A11882309F44AC08091BA
:10AA10003011843308F045C080913211823308F43C
:10AA200040C020915813222319F180910214909173
:10AA30000314A0910414B09105140097A105B10569
:10AA400009F44AC2BC01CD016D597F4F8F4F9F4F12
:10AA500024E630E040E050E00E9431EC60910614C2
:10AA60007091071480910814909109140E9431ECA0
:10AA700048E4249FB0011124072E000C880B990B89
:10AA80000E9472E82AE037ED43E25CE30E94D1E8DD
:10AA90000E94D8ED262F02E042E367E38CEF90E1BD
:10AAA00047DC80913011813308F060C08091321111
:10AAB000893208F45BC00E9469C52B013C018CE31C
:10AAC000882E912CA12CB12CC301B201A5019401B7
:10AAD0000E9431ECCA01B901A50194010E9431EC38
:10AAE000CA01962E872E59018E010F5F1F4F41E834
:10AAF000441641E5540641E06406710408F4EEC1D1
:10AB0000B90128E130E040E050E00E9431EC290139
:10AB10003A018F929F92C50168E170E00E9453EF65
:10AB20009F938F935F924F928FE199E09F938F93C2
:10AB30001F930F930E9405E80FB6F894DEBF0FBE77
:10AB4000CDBF9AE0491651046104710408F0F5C1C3
:10AB500097E0892F880F980F9195955A909333110C
:10AB600080E380933411C8010E94285FE091F610C1
:10AB7000F091F71084818111D4C06091FD0470912F
:10AB8000FE048091FF04909100050E94D3ED7A832A
:10AB90006983CE0101960E94D5D7BC0189ED94E06E
:10ABA0000E94DCEF60910105709102058091030520
:10ABB000909104050E94D3ED7A836983CE010196BA
:10ABC0000E94D5D7BC0184ED94E00E94DCEF2CEA12
:10ABD00035EC47E257E360910505709106058091D9
:10ABE0000705909108050E948FEC20E030E048ECCA
:10ABF00052E40E94D1E80E94D3ED4B015C0197FD25
:10AC000019C090E1891697E29906A104B104E4F015
:10AC1000C501B40120E137E240E050E00E9453EC6E
:10AC2000CA01B9012AE030E040E050E00E9453EC54
:10AC3000605D0BC0B094A09490948094811C911C92
:10AC4000A11CB11C6DE201C060E260931A0828EEFD
:10AC5000821623E09206A104B10494F0C501B40168
:10AC600028EE33E040E050E00E9453ECCA01B90105
:10AC70002AE030E040E050E00E9453EC605D01C00B
:10AC800060E260931B08C501B40124E630E040E0B7
:10AC900050E00E9453EC9AE0492E512C612C712C0B
:10ACA000CA01B901A30192010E9453EC605D609357
:10ACB0001C08C501B401A30192010E9453EC4B0191
:10ACC0005C01672B682B692B79F08EE280931D085D
:10ACD000CA01B901A30192010E9453EC605D609327
:10ACE0001E0880E3880D15C0CA01B901A3019201B5
:10ACF0000E9453EC662339F08EE280931D08605D5C
:10AD000060931E0805C080E280931E0880931D0892
:10AD100080E280931F086AE178E08DEC94E00E9465
:10AD2000DCEF80913011883298F4809132118D31AE
:10AD300078F02BE040E86DE180E00E94B8C380919C
:10AD40003011873228F4809132118F3108F0F7C02A
:10AD500080913011823328F4809132118B3208F0C7
:10AD600053C180913011803428F48091321188339E
:10AD700008F064C18091D907882339F098D740E062
:10AD800050E0BA0182E698E526D72091230230915F
:10AD900024024091FF0750910008609101087091D2
:10ADA0000208C901840F951F2436310524F4853625
:10ADB00091053CF416C02436310531F084369105F6
:10ADC00084F484E690E00DC04B30510561057105B7
:10ADD00014F00A9706C0463F5F4F6F4F7F4F6CF4E9
:10ADE0000A9690932402809323021092FF071092F8
:10ADF000000810920108109202088091230290919D
:10AE000024028A3091053CF0883E43E094072CF000
:10AE100087EE93E002C08AE090E090932402809352
:10AE2000230262960FB6F894DEBF0FBECDBFDF914E
:10AE3000CF911F910F91FF90EF90DF90CF90BF9037
:10AE4000AF909F908F907F906F905F904F900895FC
:10AE50002CE09FCC22E19DCC02E022E041E16DE0BC
:10AE60008CEF90E165DADBCC2CE045CD22E143CDDF
:10AE700002E022E042E168E58CEF90E159DA81CD11
:10AE800007E028E04AE26AE28CEF90E151DA05E05F
:10AE900022E04CE262E38CEF90E14ADA24E04AE0FF
:10AEA00061E38AE20E94B8C36091FE107091FF10C6
:10AEB00082E3809318118BE28093191128E131E12C
:10AEC00042E38CEF90E11CD994CD24E04AE461E3A5
:10AED00086E30E94B8C396CD20E0CACD44E6A4160E
:10AEE000B104C0F48F929F92C50168E170E00E94A6
:10AEF00053EF9F938F9385E199E09F938F931F93D7
:10AF00000F930E9405E80FB6F894DEBF0FBECDBFC9
:10AF100095E01FCE8F929F923F932F938DE099E003
:10AF20009F938F931F930F930E9405E80FB6F89499
:10AF3000DEBF0FBECDBF96E00CCE98E00ACE83E018
:10AF40008093331186E280933411FF2021F081E356
:10AF500099E071D70DC08091A004811102C08FE3E8
:10AF600005C08091ED048111F2CF80E20E947074DF
:10AF70008BE08093331116E21093341189ED94E045
:10AF800067D78BE28093331110933411FF2021F0A7
:10AF90008FE299E050D70DC08091A104811102C0C9
:10AFA0008FE305C08091EE048111F2CF80E20E9410
:10AFB000707483E38093331116E21093341184ED9F
:10AFC00094E046D783E58093331110933411FF202A
:10AFD00021F08DE299E02FD70DC08091A20481115C
:10AFE00002C08FE305C08091EF048111F2CF80E2AF
:10AFF0000E9470748BE58093331186E28093341144
:10B000008DEC94E025D7A4CE84E037D683E08093FE
:10B01000331112E31093341186E0F9D60E94DBD885
:10B020008CE0809333111093341183E292E00E94FC
:10B0300041D80ED785E20E94707493CE10923311DE
:10B040008FE38093341187E692E002D793CE80910C
:10B0500097048630D8F496E0899FF0011124EC55CE
:10B06000FB4F209132023091330231832083409193
:10B07000FF07509100086091010870910208428317
:10B080005383648375838F5F80939704089540E0B2
:10B0900050E0BA018BEF92E59EC5E0919704EE2354
:10B0A00081F0E150E093970486E0E89FF0011124DD
:10B0B000EC55FB4F42815381648175818081918180
:10B0C0008AC5E5CF0F931F93CF93DF931092D707D5
:10B0D0008091FF0790910008A0910108B0910208AB
:10B0E00081309048A105B10540F01092FF07109201
:10B0F00000081092010810920208C091FF07809189
:10B10000DE041816DCF4282F082E000C330B215017
:10B1100031094C2F0C2E000C550B4217530774F0BD
:10B12000CFEFC80F8C2F90E0A0E0B0E08093FF0736
:10B1300090930008A0930108B09302081092C907E9
:10B140008091C807C81714F4C093C8078091C80736
:10B15000082E000C990B04962C2F0C2E000C330B90
:10B160008217930724F48CEF8C0F8093C8071091FB
:10B17000C807D0E001E0112341F080915A1190916D
:10B180005B11891B8F70B9F519C080913402882337
:10B1900049F081E0C11180E024E040ED5BE06D2FDB
:10B1A0000E949CD88091D907882339F3C111E5CF3B
:10B1B00074DF8091C907882301F30FC180918A1140
:10B1C000811119C01130D1F480913402882351F0DB
:10B1D00081E0C13009F080E023E043EC5BE06D2FBB
:10B1E0000E949CD88091D907882331F1C13021F584
:10B1F0008DEE9DE61BC0113009F4D6C01230E1F48B
:10B2000080913402882351F081E0C23009F080E05F
:10B2100023E04BEB5BE06D2F0E949CD88091D90717
:10B22000882351F0C23041F482E091EB0E94EA6B36
:10B230008091C9078111D1C080918B11882309F4B5
:10B240008BC080915813882309F476C080918A11AD
:10B250008823E9F01330D9F580913402882351F026
:10B2600081E0C33009F080E020E24FEA5BE06D2F1F
:10B270000E949CD88091D907882309F48CC0C330E0
:10B2800009F089C010928A110E94BB7950C0133016
:10B29000F1F480913402882351F081E0C33009F049
:10B2A00080E020E242EA5BE06D2F0E949CD8809112
:10B2B000D907882309F46FC0C33009F06CC08091AE
:10B2C0008B11811100938A110E947B7930C0143058
:10B2D00009F061C080913402882351F081E0C430CC
:10B2E00009F080E020E247E95BE06D2F0E949CD8E6
:10B2F0008091D907882309F44EC0C43009F04BC0AF
:10B300000E9465748091A3048093AE061092AF06EC
:10B310000E943BC80E9450C5109214081092130856
:10B320001092040260E080E79BE00E9437D9809190
:10B33000C907882381F151C0133011F084E02CC07B
:10B34000809134028823C1F081E0C33009F080E0AD
:10B3500023E049E85BE00DC0133081F780913402AF
:10B36000882351F081E0C33009F080E023E04EE70C
:10B370005BE06D2F0E949CD88091D9078823F1F261
:10B38000C330E1F684E197E60E94EA6B8091C90739
:10B390008823A1F222C085E0DF5F1F5FD53009F06E
:10B3A000EACE8093DE0419C080913402882351F0E4
:10B3B00081E0C13009F080E023E04BEC5BE06D2FD1
:10B3C0000E949CD88091D907882309F435CFC130D9
:10B3D00009F032CF89E391E729CFDF91CF911F9117
:10B3E0000F91089590E0FC013197E231F10508F0EA
:10B3F0004EC08827EE58FF4F8F4F0C947AEF809104
:10B4000080008F7703C0809180008F7D80938000C3
:10B41000089580918000877FF9CF84B58F7702C02F
:10B4200084B58F7D84BD08958091B0008F7703C06F
:10B430008091B0008F7D8093B0000895809190003E
:10B440008F7707C0809190008F7D03C0809190001E
:10B45000877F8093900008958091A0008F7707C028
:10B460008091A0008F7D03C08091A000877F809392
:10B47000A0000895809120018F7707C0809120015E
:10B480008F7D03C080912001877F809320010895E4
:10B490003FB7F8948091E3049091E404A091E5040F
:10B4A000B091E60426B5A89B05C02F3F19F0019680
:10B4B000A11DB11D3FBFBA2FA92F982F8827820F3A
:10B4C000911DA11DB11DBC01CD0142E0660F771F8A
:10B4D000881F991F4A95D1F708951F93CF93DF9343
:10B4E000282F30E0F901EE5BF24F8491F901E4502E
:10B4F000F34FD491F901EA54F34FC491CC23C1F036
:10B50000162F81116FDFEC2FF0E0EE0FFF1FEE57CB
:10B51000F34FA591B4918FB7F894111105C09C9188
:10B52000ED2FE095E92302C0EC91ED2BEC938FBF5A
:10B53000DF91CF911F910895CF93DF9390E0FC01AD
:10B54000E450F34F2491FC01EA54F34F8491882393
:10B5500061F190E0880F991FFC01E859F34FC59104
:10B56000D491FC01EE57F34FA591B491611109C03C
:10B570009FB7F8948881209582238883EC912E23AD
:10B580000BC0623061F49FB7F8943881822F8095A8
:10B5900083238883EC912E2B2C939FBF06C08FB7FB
:10B5A000F894E8812E2B28838FBFDF91CF910895E7
:10B5B0001F93CF93DF93182FEB0161E0BDDF20973E
:10B5C00011F460E004C0CF3FD10531F461E0812F78
:10B5D000DF91CF911F9181CFE12FF0E0EE5BF24F31
:10B5E000E4914E2F50E0FA013197E231F10508F075
:10B5F0009DC08827EC57FF4F8F4F0C947AEF84B58E
:10B60000806884BDC7BD97C084B5806284BDC8BD55
:10B6100092C080918000806880938000D0938900E0
:10B62000C093880088C080918000806280938000F1
:10B63000D0938B00C0938A007EC080918000886088
:10B6400080938000D0938D00C0938C0074C0809153
:10B65000B00080688093B000C093B3006CC080914C
:10B66000B00080628093B000C093B40064C0809149
:10B670009000806880939000D0939900C0939800C8
:10B680005AC080919000806280939000D0939B007C
:10B69000C0939A0050C08091900088608093900081
:10B6A000D0939D00C0939C0046C08091A00080680C
:10B6B0008093A0008091A0008F7B8093A000D09306
:10B6C000A900C093A80037C08091A0008062809339
:10B6D000A000D093AB00C093AA002DC08091A00021
:10B6E00088608093A000D093AD00C093AC0023C0CD
:10B6F00080912001806880932001D0932901C0931C
:10B70000280119C080912001806280932001D0938C
:10B710002B01C0932A010FC0809120018860809383
:10B720002001D0932D01C0932C0105C0C038D10554
:10B730000CF04CCF46CFDF91CF911F9108958F929F
:10B740009F92AF92BF92CF92DF92EF92FF926B01E6
:10B750007C019EDE4B015C01C114D104E104F104C3
:10B76000E9F096DEDC01CB0188199909AA09BB0929
:10B77000883E9340A105B10578F321E0C21AD108B3
:10B78000E108F10888EE880E83E0981EA11CB11C28
:10B79000C114D104E104F10421F7DECFFF90EF9052
:10B7A000DF90CF90BF90AF909F908F9008952FB76C
:10B7B000F8946091DF047091E0048091E10490912D
:10B7C000E2042FBF089511982FB787FD71C0F89438
:10B7D000909102019E7F909302012FBF119A000069
:10B7E0001198282F220F9FB786FD81C0F894809171
:10B7F00002018E7F809302019FBF119A0000119871
:10B80000922F990F26FD6DC02FB7F89480910201F9
:10B810008E7F809302012FBF119A00001198892F0B
:10B82000880F2FB796FD58C0F894909102019E7F23
:10B83000909302012FBF119A00001198982F990F31
:10B840002FB786FD44C0F894809102018E7F8093CB
:10B8500002012FBF119A00001198892F880F2FB76E
:10B8600096FD30C0F894909102019E7F9093020162
:10B870002FBF119A00001198982F990F2FB786FDAE
:10B880001CC0F894809102018E7F809302012FBF2B
:10B89000119A0000119896FD2FC09FB7F8948091DF
:10B8A00002018E7F809302019FBF119A00000895CC
:10B8B000F8949091020191608ECFF89480910201EA
:10B8C0008160E3CFF894909102019160CFCFF8941A
:10B8D000809102018160BBCFF89490910201916048
:10B8E000A7CF2FB7F89480910201816092CFF8948E
:10B8F0008091020181607ECF9FB7F8948091020110
:10B900008160D0CFFC011382128284E493E09183A2
:10B91000808313AE14AE15AE9F012C5F3F4F11868E
:10B92000108613861286158681E0848782E28687D8
:10B93000138A128ADF019796CF01C5964FEF4D9378
:10B94000A817B907E1F791E094A346EE54E4528FAB
:10B95000418F938F148E158E80E4868F178E86E824
:10B9600094E496AB85AB77836683C9010C9402514E
:10B970006F927F928F929F92AF92BF92CF92DF92FF
:10B98000EF92FF920F931F93CF93DF935C017B01A4
:10B99000742E69018AE0481709F474C0A5E14A13BE
:10B9A0004FC0DB011296ED91FC9113979280C681F6
:10B9B000D7819FB7F8948091020182608093020141
:10B9C0009FBF0E94675180EE882E890C90E1692EFE
:10B9D000690C88EFF8DE0E946751BFE1B91508F4E1
:10B9E00043C0892D80778068EEDE892D8295807F27
:10B9F000EADE0E94675180E8E6DE80E0E4DE0E9435
:10BA000067518AEFE0DE0E9467518E01005F1F4F91
:10BA10008881807FD8DE89918295807FD4DEC017AF
:10BA2000D107B1F70E946751939483949610D1CFB8
:10BA30009FB7F894809102018D7F809302019FBF90
:10BA40009601472DB701C501DF91CF911F910F914D
:10BA5000FF90EF90DF90CF90BF90AF909F908F902E
:10BA60007F906F900C94B64F882D80778068ABDE06
:10BA7000882D8295807FA7DE0E94675180E8A3DE33
:10BA800080E8BCCF809101018260809301019FB763
:10BA9000F894809102018D7F809302019FBF809175
:10BAA00001018160809301019FB7F89480910201A8
:10BAB0008E7F809302019FBF099A119A9FB7F894D5
:10BAC000809102018260809302019FBF0E946751B2
:10BAD00088E790E00E946C5188EF75DE0E94675104
:10BAE00080E071DE80E86FDE0E94675180E06BDEEF
:10BAF00080E169DE0E9467518FE090E00E946C5106
:10BB000080E361DE80EE5FDE0E946751D0E08D2F22
:10BB10008077806858DE8D2F8295807F54DE0E946A
:10BB2000675180E850DE80E04EDE0E9467518AEF68
:10BB30004ADE0E946751C0E280E045DE80E043DEDD
:10BB40000E946751C150C1F788EF3DDE0E946751E6
:10BB5000DF5FD032E1F680E036DE80EC34DE0E943A
:10BB6000675166CFCF92DF92EF92FF920F931F93B0
:10BB7000CF93DF931F92CDB7DEB76C01DC01DC966B
:10BB80001C91DC97DB960C917C01B4E0EB0EF11C70
:10BB9000DC015996ED91FC915A97C701698319957B
:10BBA000482F410F2981602FC7010E94B351F60130
:10BBB00023AD082E000C990B820F911D83AF81E0FD
:10BBC00090E00F90DF91CF911F910F91FF90EF9038
:10BBD000DF90CF90089520913202309133022817E0
:10BBE0003907D9F090933302809332024093FF07D4
:10BBF0005093000860930108709302088B5F924590
:10BC000021F41092D2071092970482E080933402BC
:10BC100081E08093C9071092D80708959CE0899F1E
:10BC2000802D112491E0980F909317082CE0280F95
:10BC3000209318084091301150E030E02E5F3F4FC4
:10BC400024173507CCF0292F30E04091321150E015
:10BC5000241735078CF4662341F08E5F0E949FC342
:10BC6000809118088E5F0E949FC3809118081092DF
:10BC700033118093341108950895CF93C82F8230E3
:10BC800059F02CF4813089F4CF910C94DBD88330B7
:10BC900031F0843021F009C08CED9BE002C083ECD0
:10BCA00096E40E9418C3C0938314CF910895EF9235
:10BCB000FF920F931F93CF93DF931F92CDB7DEB701
:10BCC00080913511811107C081E0809335118CEF8F
:10BCD00090E10E9402516091FE107091FF10198254
:10BCE0009E012F5F3F4F4FE08CEF90E10E9480500C
:10BCF00080911E02882371F10E947B7406E510E199
:10BD000020E440E160E080E00E948DC284E0B5DF85
:10BD10006091FD106E5147EB53E080E00E94E3C25A
:10BD20006091FD1062514CEB53E080E00E94E3C251
:10BD30006091FD10665043EC53E080E00E94E3C246
:10BD40000E9465C38111DACF68EB7BE080E090E070
:10BD50000E947AD8F090FC1080911E0281110AC0D6
:10BD600010921E020F90DF91CF911F910F91FF90C3
:10BD7000EF9008950E947B742F2D30E0C901C89781
:10BD800097FD019695958795E82E2E5131093695A8
:10BD90002795F22E01ED1FE023E147E06CE08E2DA8
:10BDA0000E948DC284E069DF0091FC1010E0025710
:10BDB0001109169507956091FD10625141ED53E010
:10BDC0008F2D0E94E3C26091FD10665047ED53E055
:10BDD000802F0E94E3C20E9465C38111DBCFC0CFD8
:10BDE000CF93C82F8FEF8C0F893058F48CED9BE0E8
:10BDF0000E9418C38C2F0E947074809183143DDFC1
:10BE000003C08C2F0E94707481E0CF910895CF936E
:10BE10009FEF980F993060F4C82F8CED9BE00E9443
:10BE200018C38C2F0E94707480918314CF9125CFFA
:10BE3000CF910C947074CF93DF93EC01FE01849149
:10BE4000882319F0E4DF2196F9CFDF91CF9108958F
:10BE50000F931F93CF938C01C0E0F801EC0FF11DFD
:10BE60008081882319F0D3DFCF5FF7CFCF911F9167
:10BE70000F9108959F92AF92BF92CF92DF92EF926F
:10BE8000FF920F931F93CF93DF931F92CDB7DEB72F
:10BE90005C017B0120E030E0F501E20FF31FE4914B
:10BEA000EE2319F02F5F3F4FF7CFF7016F01CE1848
:10BEB000DF0881918111FACFDD24332784E190E0FE
:10BEC0008C199D098217930714F001E001C002E06C
:10BED00010E08091FD1090E0B8016F5F7F4F0E94ED
:10BEE00067EF86E0982E960E80913011981648F0F4
:10BEF0002091321130E0892D90E00B9728173907F7
:10BF000094F5E114F104C1F101501109609F900C06
:10BF1000112480913011981678F12091321130E07F
:10BF2000892D90E00B972817390734F18AE30E9496
:10BF3000707425E130E02C193D09822F880F280FFD
:10BF4000220F2093331190923411C7010F90DF918B
:10BF5000CF911F910F91FF90EF90DF90CF90BF9006
:10BF6000AF909F9075CF1092331190923411C5010C
:10BF7000698361DF6981C5CF0F90DF91CF911F91F8
:10BF80000F91FF90EF90DF90CF90BF90AF909F9078
:10BF90000895CF93DF93EC0168E172E0B3DC8CE4A9
:10BFA00093E099838883DF91CF9108952F923F92F8
:10BFB0004F925F926F927F928F929F92AF92BF92B9
:10BFC000CF92DF92EF92FF920F931F93CF93DF9365
:10BFD000EC0145EF5EE081E090E0FA0125913491BB
:10BFE000C217D3070CF05DC09C0121503109220F0C
:10BFF000331F220F331FD901AD50B14FFD016591A1
:10C0000074912F50314FF901A590B490FC01EE0FBF
:10C01000FF1FEE0FFF1FED50F14FE590F490FD0173
:10C02000C590D490FA0105911491F90125903490AE
:10C03000072E000C880B990B0E9472E82B013C0123
:10C04000CA19DB09BE01DD0F880B990B0E9472E84B
:10C050004B015C01B7016C197D09072E000C880BA0
:10C06000990B0E9472E89B01AC01C501B4010E94CA
:10C07000D1E86B017C01B80162197309072E000C2D
:10C08000880B990B0E9472E89B01AC01C701B601B5
:10C090000E946BED9B01AC01C301B2010E948FECC9
:10C0A00011C001964C5F5F4F8032910509F095CF2A
:10C0B000EFE6FFE065917491072E000C880B990B59
:10C0C0000E9472E8DF91CF911F910F91FF90EF9046
:10C0D000DF90CF90BF90AF909F908F907F906F90A8
:10C0E0005F904F903F902F900895609198047091C9
:10C0F000990480919A0490919B040E94D3EDCB0106
:10C1000008951F920F920FB60F9211240BB60F9243
:10C110002F933F934F935F936F937F938F939F934F
:10C12000AF93BF93CF93DF93EF93FF938091B706C5
:10C13000811156C181E08093B70680916E008B7F9C
:10C1400080936E007894809117028F37B0F08F57EC
:10C150009091B6069093C707992311F02C9A01C0CD
:10C160002C989091B5069093C6072FB7992379F034
:10C17000F8949091020190620EC09091C7078917C0
:10C1800008F02C989091C607891740F02FB7F894C3
:10C19000909102019F7D909302012FBF8F5F80934A
:10C1A00017029091C50781E089278093C507811107
:10C1B0000E94E3D880911502909116028230910579
:10C1C000A1F1A4F4009761F1019709F048C08091B2
:10C1D0007800909179002091BA073091BB07820FC7
:10C1E000931F9093BB078093BA0739C083309105A2
:10C1F00041F10497A1F58091C407811103C086E045
:10C200008093C4078091C40781508093C40788231A
:10C2100031F183E090E090931602809315021FC0E5
:10C2200088E080937B0085E404C088E080937B00F5
:10C2300086E480937C0080917A00806480937A0009
:10C240000EC080917800909179002091B8073091CC
:10C25000B907820F931F9093B9078093B807809115
:10C26000150290911602892B09F060C0809114028A
:10C270008F5F80311CF48093140258C01092140216
:10C280008091B406811113C08091BA079091BB07C9
:10C290009093B3068093B2068091B8079091B90746
:10C2A0009093B1068093B00681E08093B4068AE053
:10C2B000EAEBF7E0DF011D928A95E9F71092B907E2
:10C2C0001092B807C091B206D091B306D195C1952E
:10C2D000D1098091E9049091EA04919581959109A1
:10C2E0008C179D07CCF180910702909108029195DF
:10C2F00081959109C817D9070CF43FC02091B00669
:10C300003091B1068091E7049091E8048217930779
:10C310000CF044C020910502309106028091B006D5
:10C320009091B106821793070CF049C080911502D5
:10C3300090911602019665E070E00E9467EF90937D
:10C34000160280931502F8941092B70680916E0041
:10C35000846080936E0044C080911108909112080F
:10C36000181619060CF0BFCF42EB5FE06FEB7FE0D1
:10C3700080E090E00E942FD2B6CF8091110890917A
:10C380001208181619060CF0B9CF42E85FE06FE802
:10C390007FE080E090E00E942FD2B0CF809115081E
:10C3A00090911608181619060CF0B4CF41EA5FE018
:10C3B0006FEB7FE08FEF9FEF0E942FD2ABCF80918A
:10C3C000150890911608181619060CF0AFCF41E722
:10C3D0005FE06FE87FE08FEF9FEF0E942FD2A6CF44
:10C3E000FF91EF91DF91CF91BF91AF919F918F918D
:10C3F0007F916F915F914F913F912F910F900BBE65
:10C400000F900FBE0F901F9018950F931F93CF930F
:10C41000DF9300D01F92CDB7DEB78091FF079091D8
:10C420000008A0910108B0910208B7FF08C010925F
:10C43000FF071092000810920108109202088091E4
:10C44000030890910408A0910508B0910608409156
:10C45000FF0750910008609101087091020884174D
:10C460009507A607B70744F48093FF079093000849
:10C47000A0930108B093020880913402882371F1DF
:10C480004091FF07509100086091010870910208E7
:10C490008091070890910808A0910908B0910A08B6
:10C4A0008A019B01080F191F2A1F3B1FC901B801F0
:10C4B0000E9470E820E030E048EC52E40E94D1E8AD
:10C4C00069837A838B839C83CE0101960E946DD60B
:10C4D000BC0180910D0890910E08CCDC8091D907A9
:10C4E000882399F14091FF0750910008609101085D
:10C4F000709102088091070890910808A09109089E
:10C50000B0910A088A019B01080F191F2A1F3B1FBF
:10C51000C901B8010E9470E820E030E048EC52E424
:10C520000E94D1E80E94D8EDE0910B08F0910C0830
:10C53000309721F060837183828393830E944D58EA
:10C54000E0910F08F091100819950F900F900F903F
:10C550000F90DF91CF911F910F9108950F931F932B
:10C56000CF93DF9300D01F92CDB7DEB78091FF0746
:10C5700090910008A0910108B0910208B7FF08C08F
:10C580001092FF0710920008109201081092020802
:10C590008091030890910408A0910508B0910608C5
:10C5A0004091FF07509100086091010870910208C6
:10C5B00084179507A607B70744F48093FF07909365
:10C5C0000008A0930108B0930208809134028823E8
:10C5D00071F14091FF07509100086091010870913E
:10C5E00002088091070890910808A0910908B0916D
:10C5F0000A088A019B01080F191F2A1F3B1FC90146
:10C60000B8010E9472E820E030E048EC52E40E9459
:10C61000D1E869837A838B839C83CE0101960E9443
:10C620006DD6BC0180910D0890910E0823DC80919D
:10C63000D907882361F14091FF075091000860916C
:10C640000108709102088091070890910808A09154
:10C650000908B0910A088A019B01080F191F2A1FB7
:10C660003B1FC901B8010E9472E820E030E048ECAD
:10C6700052E40E94D1E8E0910B08F0910C08309749
:10C6800021F060837183828393830E944D580F90C1
:10C690000F900F900F90DF91CF911F910F91089500
:10C6A0000F931F93CF93DF9300D01F92CDB7DEB7C8
:10C6B0008091FF0790910008A0910108B0910208B5
:10C6C000B7FF08C01092FF071092000810920108EF
:10C6D000109202088091030890910408A091050827
:10C6E000B09106084091FF07509100086091010841
:10C6F0007091020884179507A607B70744F4809342
:10C70000FF0790930008A0930108B093020880915E
:10C710003402882371F14091FF0750910008609125
:10C720000108709102088091070890910808A09173
:10C730000908B0910A088A019B01080F191F2A1FD6
:10C740003B1FC901B8010E9472E82AE037ED43E2BD
:10C750005CE30E94D1E869837A838B839C83CE015A
:10C7600001960E9437D5BC0180910D0890910E086A
:10C7700081DB8091D907882389F14091FF0750918F
:10C78000000860910108709102088091070890915B
:10C790000808A0910908B0910A088A019B01080FB6
:10C7A000191F2A1F3B1FC901B8010E9472E82AE025
:10C7B00037ED43E25CE30E94D1E8E0910B08F09191
:10C7C0000C08309721F060837183828393830E94E9
:10C7D0004D58E0910F08F091100819950F900F90A7
:10C7E0000F900F90DF91CF911F910F910895CF92ED
:10C7F000DF92EF92FF920F931F93CF93DF9300D0BE
:10C800001F92CDB7DEB78091FF0790910008A091ED
:10C810000108B0910208B7FF08C01092FF071092FC
:10C82000000810920108109202088091030890916C
:10C830000408A0910508B09106084091FF075091A7
:10C840000008609101087091020884179507A607F7
:10C85000B70744F48093FF0790930008A093010862
:10C86000B093020880913402882371F14091FF0750
:10C8700050910008609101087091020880910708AA
:10C8800090910808A0910908B0910A086A017B01FB
:10C89000C80ED91EEA1EFB1EC701B6010E9472E82F
:10C8A0002AE037ED43E25CE30E94D1E869837A83B2
:10C8B0008B839C83CE0101960E94ECD5BC018091B4
:10C8C0000D0890910E08D6DA1091D907112361F165
:10C8D0008091FF0790910008A0910108B091020893
:10C8E00040910708509108086091090870910A0862
:10C8F0006C017D01C40ED51EE61EF71EC701B601F0
:10C900000E9472E82AE037ED43E25CE30E94D1E83E
:10C91000E0910B08F0910C08309721F0608371834F
:10C92000828393830E944D58812F0F900F900F9018
:10C930000F90DF91CF911F910F91FF90EF90DF90BB
:10C94000CF90089554DF882329F0E0910F08F091EB
:10C950001008199408954BCF0F931F93CF93DF9333
:10C9600000D01F92CDB7DEB78091FF0790910008ED
:10C97000A0910108B0910208B7FF08C01092FF070C
:10C98000109200081092010810920208809103088A
:10C9900090910408A0910508B09106084091FF0706
:10C9A0005091000860910108709102088417950762
:10C9B000A607B70744F48093FF0790930008A0935D
:10C9C0000108B093020880913402882371F14091EC
:10C9D000FF07509100086091010870910208809152
:10C9E000070890910808A0910908B0910A088A01E7
:10C9F0009B01080F191F2A1F3B1FC901B8010E9484
:10CA000072E82FE632E143E85AE30E94D1E86983F5
:10CA10007A838B839C83CE0101960E94E179BC01CD
:10CA200080910D0890910E0825DA8091D90788230E
:10CA300089F14091FF0750910008609101087091C1
:10CA400002088091070890910808A0910908B09108
:10CA50000A088A019B01080F191F2A1F3B1FC901E1
:10CA6000B8010E9472E82FE632E143E85AE30E94DF
:10CA7000D1E8E0910B08F0910C08309721F0608329
:10CA80007183828393830E944D58E0910F08F09147
:10CA9000100819950F900F900F900F90DF91CF9184
:10CAA0001F910F910895CF92DF92EF92FF920F9313
:10CAB0001F93CF93DF9300D01F92CDB7DEB7809145
:10CAC000FF0790910008A0910108B0910208B7FFFC
:10CAD00008C01092FF0710920008109201081092EF
:10CAE00002088091030890910408A0910508B09174
:10CAF00006084091FF07509100086091010870916D
:10CB0000020884179507A607B70744F48093FF0728
:10CB100090930008A0930108B0930208809134021A
:10CB2000882371F14091FF0750910008609101083E
:10CB3000709102088091070890910808A091090857
:10CB4000B0910A086A017B01C80ED91EEA1EFB1EBD
:10CB5000C701B6010E9472E82AE037ED43E25CE3C8
:10CB60000E94D1E869837A838B839C83CE010196EE
:10CB70000E9457D7BC0180910D0890910E087AD978
:10CB80001091D907112361F18091FF07909100085E
:10CB9000A0910108B091020840910708509108083F
:10CBA0006091090870910A086C017D01C40ED51EC0
:10CBB000E61EF71EC701B6010E9472E82AE037EDB3
:10CBC00043E25CE30E94D1E8E0910B08F0910C088D
:10CBD000309721F060837183828393830E944D5844
:10CBE000812F0F900F900F900F90DF91CF911F9199
:10CBF0000F91FF90EF90DF90CF90089554DF88233E
:10CC000029F0E0910F08F0911008199408954BCF86
:10CC10000F931F93CF93DF931F921F92CDB7DEB771
:10CC20008091FF0790910008A0910108B09102083F
:10CC3000B7FF08C01092FF07109200081092010879
:10CC4000109202088091030890910408A0910508B1
:10CC5000B09106084091FF075091000860910108CB
:10CC60007091020884179507A607B70744F48093CC
:10CC7000FF0790930008A0930108B09302088091E9
:10CC80003402882341F14091FF07509100086091E0
:10CC90000108709102088091070890910808A091FE
:10CCA0000908B0910A088A019B01080F191F2A1F61
:10CCB0003B1FC901B8010E9472E80E94D3ED7A833C
:10CCC0006983CE0101960E9441D8BC0180910D0874
:10CCD00090910E08CFD88091D907882331F14091E7
:10CCE000FF0750910008609101087091020880913F
:10CCF000070890910808A0910908B0910A088A01D4
:10CD00009B01080F191F2A1F3B1FC901B8010E9470
:10CD100072E8E0910B08F0910C08309721F06083E5
:10CD20007183828393830E944D580F900F90DF91FF
:10CD3000CF911F910F910895CF93DF9300D0CDB77E
:10CD4000DEB78091FF0790910008A0910108B09193
:10CD50000208B7FF08C01092FF0710920008109257
:10CD60000108109202088091030890910408A09194
:10CD70000508B09106084091FF07509100086091A6
:10CD800001087091020884179507A607B70744F4B5
:10CD90008093FF0790930008A0930108B0930208C6
:10CDA000809134028823B1F020910708309108085F
:10CDB0008091FF0790910008820F931F9A838983C7
:10CDC000CE0101960E9441D8BC0180910D0890913E
:10CDD0000E0850D88091D9078823B1F040910708F8
:10CDE000509108082091FF0730910008240F351F4B
:10CDF000E0910B08F0910C08309711F031832083FB
:10CE00008B830E944D588B810F900F900F90DF9174
:10CE1000CF91089591CF90DF882329F0E0910F08FA
:10CE2000F091100819940895AF92BF92CF92DF92BB
:10CE3000EF92FF920F931F93CF93DF93CDB7DEB79F
:10CE40006F970FB6F894DEBF0FBECDBF809134024E
:10CE5000811105C08091D907882309F4CDC188EDDF
:10CE600091E19093D7118093D61181E090E0909357
:10CE7000101480930F14109212141092111440E0A9
:10CE800050E0BA018CED91E10E94308F8091D61173
:10CE90009091D7112BE1FC013496DE01159601909B
:10CEA0000D922A95E1F7FC01828193819C838B830B
:10CEB00080E893E09A83898340E050E0BE016F5F91
:10CEC0007F4F8AE094E00E9450C6CE0101960E94F6
:10CED000AF4FA0901114B09012141092D707809108
:10CEE000FF0790910008A0910108B09102088130DD
:10CEF0009048A105B10540F01092FF07109200087C
:10CF000010920108109202081091FF078091DB0730
:10CF10001816DCF4282F082E000C330B2150310991
:10CF2000412F012E000C550B4217530774F01FEFD1
:10CF3000180F812F90E0A0E0B0E08093FF0790935E
:10CF40000008A0930108B09302081092C9078091CD
:10CF5000C807181714F41093C8078091C807082E43
:10CF6000000C990B0496212F012E000C330B821715
:10CF7000930724F48CEF810F8093C8070091C807B2
:10CF8000F12C21E0A21AB108002359F06DE871E1FB
:10CF90008CED91E10E943C9180918D118F32D9F4FA
:10CFA0001EC080913402882349F081E0111180E095
:10CFB00024E040E750E36F2D0E949CD88091D90770
:10CFC000882321F31111E2CF0E944D588091C907A7
:10CFD0008823E1F211C1013041F092E001C091E0FB
:10CFE0006501EE24E394E00E63C08091340288234F
:10CFF00051F081E0113009F080E020E24CE650E38E
:10D000006F2D0E949CD88091D907882331F311306D
:10D0100021F780912D138823D1F0815080932D1317
:10D02000EFE18E9FC0011124FC01E550FE4E2BE183
:10D03000ACEDB1E101900D922A95E1F7FC01E950C8
:10D04000FE4E828193819093DB118093DA111092CE
:10D05000C8070FC08AE00E945C87CE0101960E943B
:10D06000AF4F1092FF071092000810920108109223
:10D07000020881E08093C90783E080933402BCC03A
:10D080000913B1C060E070E0C6010E941074909175
:10D090008C1180913402992309F489C081110DC04B
:10D0A0008091D907811111C09E2DF1E0CF1AD108CE
:10D0B0002FEFC216D20621F798C081E0101380E04E
:10D0C00041E06F2D0E94567AEBCF1013EDCF1D82F9
:10D0D00018861C821B8280E893E09A838983809162
:10D0E000DF11882319F008ED11E102C007EB11E10F
:10D0F0007801F4E0EF0EF11C21E04DE851E1B701B9
:10D10000CE0105960E941294811124C0E8EBF3E44D
:10D1100084918F010F5F1F4F882321F00E945C874D
:10D12000F801F6CFE6E5F0E384918F010F5F1F4F22
:10D13000811103C00DE811E104C00E945C87F80171
:10D14000F3CFF80181918F01882309F483CF0E94E6
:10D150005C87F7CF80912D138A30C8F491E0980F47
:10D1600090932D13FFE18F9FC0011124DC01A55086
:10D17000BE4E2BE1F70101900D922A95E1F7F801DF
:10D1800022813381FC01E950FE4E338322838BE1FF
:10D19000FE013596ACEDB1E101900D928A95E1F773
:10D1A0008B819C819093DB118093DA1156CF882379
:10D1B00039F081E0101380E040E06F2D0E94567A34
:10D1C0008091D907882309F46FCF10136DCF8DE8B4
:10D1D00091E10E94CD760E9447588091C90788232B
:10D1E00009F462CF09C09F5F60CFF3940F5F85E0C1
:10D1F000F812CACE9093DB076F960FB6F894DEBF95
:10D200000FBECDBFDF91CF911F910F91FF90EF9097
:10D21000DF90CF90BF90AF9008954F925F926F9242
:10D220007F928F929F92AF92BF92CF92DF92EF92B6
:10D23000FF920F931F93CF93DF9300D01F92CDB730
:10D24000DEB710911F021F3FF9F00E94D75BC0901C
:10D25000CA07D090CB07E090CC07F090CD07DC0157
:10D26000CB018C199D09AE09BF09B7FD0DC02091F6
:10D270005B1180915A1130E090E001968F709927F0
:10D280002817390709F018C20E94E3D880917E144C
:10D2900082FF40C08091E70781113EC081E080930A
:10D2A000E7079091DA0789278093D9071092DA0768
:10D2B00083E08093340210927E140E94D75BDC01DD
:10D2C000CB018C509E4FAF4FBF4F80937F149093F4
:10D2D0008014A0938114B093821480ED97E09C8316
:10D2E0008B8382E390E09A838983BE016D5F7F4FD9
:10D2F000CE0101960E942C7916E0115069F08CE560
:10D3000091E10E940E4562E070E080E090E00E94B2
:10D310009F5BF3CF1092E7071091090110951170F0
:10D320008091E6071817A9F0112309F4E6C10E94BD
:10D33000E2778091E607823029F060E082E890E3AE
:10D340000E9437D91093E60783E0809334020E944D
:10D35000575E0E94D75B6B017C018091E207909140
:10D36000E307A091E407B091E507A7019601281B08
:10D37000390B4A0B5B0B57FF05C08091D8078823F8
:10D3800009F4F6C1D701C6018C599F4FAF4FBF4F6B
:10D390008093E2079093E307A093E407B093E50737
:10D3A00080917D1418162CF480917D14843074F4CF
:10D3B00008C080917D14992781950CF4909504976D
:10D3C0002CF48091D90781119FC0AFC08091D707FD
:10D3D000882309F472C080917D14181664F480913A
:10D3E0007D14082E000C990B97FD03969595879553
:10D3F000959587950EC080917D14082E000C990B91
:10D4000097FD039695958795959587959195819527
:10D4100091098090D3079090D407A090D507B09041
:10D42000D60781149104A104B104D1F1BC01990F74
:10D43000880B990B0E9472E82B013C01C701B601D1
:10D44000681979098A099B090E9470E89B01AC015F
:10D45000C301B2010E946BED20E030E04AE754E4E2
:10D460000E94D1E84B015C0120E030E040E253E44F
:10D470000E94B5EE87FF0FC020E030E046E952E49D
:10D48000C501B4010E94B5EE87FD0AC02AE030E074
:10D4900040E050E009C024E630E040E050E004C045
:10D4A00021E030E040E050E0C092D307D092D407B2
:10D4B000E092D507F092D60704C021E030E040E0CA
:10D4C00050E0A0917D140A2E000CBB0B0E9479EC59
:10D4D00024E030E040E050E00E9453EC8091FF07F0
:10D4E00090910008A0910108B0910208820F931F4B
:10D4F000A41FB51F8093FF0790930008A093010815
:10D50000B093020810927D14D701C6018856954C3D
:10D51000AF4FBF4F8093DE079093DF07A093E007E4
:10D52000B093E10782E080933402809132029091BF
:10D5300033028B5F924541F480912002882309F4E5
:10D54000E7C08150809320022FB7F8948091CE07D6
:10D550009091CF07A091D007B091D1072FBF3AE0AB
:10D56000B695A795979587953A95D1F7009741E09D
:10D57000A407B10520F08FEF9FEFA0E0B0E09695F3
:10D58000879520913402211105C03091D8073111BF
:10D59000EBC055C0009741F04091DC075091DD078A
:10D5A0004817590708F04BC08091D807811111C066
:10D5B000223050F0243028F0243031F4109234021C
:10D5C00003C081E0809334020E947B7481E08093E9
:10D5D000D80784E00E943D5E81E080931C11E091B9
:10D5E0003202F091330219951092D9078091D80731
:10D5F000882351F00E9465C391E0811101C090E041
:10D600009093D807911194C08090DC079090DD072B
:10D61000A12CB12C0E94D75BDC01CB018C199D0998
:10D62000AE09BF0988169906AA06BB0640F40E94F7
:10D63000D75B6C197D097093DD076093DC078091DF
:10D640003202909133028B5F924521F08091D20794
:10D65000882379F088E9C80E8AE3D81EE11CF11C02
:10D66000C092DE07D092DF07E092E007F092E10778
:10D670000FC08091DE079091DF07A091E007B09185
:10D68000E107C81AD90AEA0AFB0AF7FE0E944758BE
:10D690008091D80781116CC080913402813049F0AB
:10D6A00008F466C0843008F063C081E080933402DF
:10D6B0005FC0109234025CC024E01202F001112419
:10D6C000E05BFC4F20E030E040E752E46081718194
:10D6D000828193810E946BEDC12C7B018C0129E03A
:10D6E00035E045E055E061E075E08DEF94E00E94A3
:10D6F000B7988FEF80931F02C7CD10928A111092B6
:10D700008B11823009F41ECE60E085E790E318CEDD
:10D710008CE0809320028091DC079091DD070197D7
:10D720009093DD078093DC0781E0809334020CCF77
:10D730008090DC079090DD07A12CB12C0E94D75B74
:10D74000DC01CB018C199D09AE09BF098816990629
:10D75000AA06BB0668F40E94D75B6C197D0970931A
:10D76000DD076093DC0704C0009709F432CF14CFC3
:10D770000F900F900F900F90DF91CF911F910F910D
:10D78000FF90EF90DF90CF90BF90AF909F908F90E1
:10D790007F906F905F904F9008950E94575E3E98E3
:10D7A000469A3C98449A3A98429AEAE0F1E080819D
:10D7B0008E7F80839FB7F894EBE0F1E080818160F9
:10D7C00080839FBF82E08093E6070E94E3D8109297
:10D7D0007D140895CF93DF931F921F92CDB7DEB7CC
:10D7E00089839A830E94275840E050E0BA018981DA
:10D7F0009A810F900F90DF91CF910C94EB5D80E0B8
:10D8000090E0A0E2B1E48093F8079093F907A09329
:10D81000FA07B093FB0740E050E0BA018091FD07A2
:10D820009091FE070C94EB5D80E090E0A0E8BFE3F0
:10D830008093F8079093F907A093FA07B093FB073A
:10D8400040E050E0BA018091FD079091FE070C94F2
:10D85000EB5D8DEC9CECACECBDE38093F807909312
:10D86000F907A093FA07B093FB0740E050E0BA0134
:10D870008091FD079091FE070C94EB5DCF92DF92B3
:10D88000EF92FF92CF93C82F0E94D75B6B017C0170
:10D8900024EA30E74DE75FE36091F8077091F907FC
:10D8A0008091FA079091FB070E946CE887FD05C004
:10D8B00046E950E060E070E003C040E050E0BA01AB
:10D8C000C40ED51EE61EF71EC092CA07D092CB0723
:10D8D000E092CC07F092CD07C0931F02CF91FF904A
:10D8E000EF90DF90CF9008958091D90781110C942B
:10D8F0004D586091FF077091000880910108909148
:10D900000208611571058105910571F10E9472E8A7
:10D910002091F8073091F9074091FA075091FB07E1
:10D920000E94D1E89B01AC016091090570910A0544
:10D9300080910B0590910C050E948FEC6093090576
:10D9400070930A0580930B0590930C051092FF07C6
:10D9500010920008109201081092020883E090E0F3
:10D960008DDF81E08093340280913402882349F076
:10D9700089E095E00E940FD7BC018BEB91E30C94FA
:10D980003A5F08952F923F924F925F926F927F92EB
:10D990008F929F92AF92BF92CF92DF92EF92FF92BF
:10D9A0000F931F93CF93DF9300D000D0CDB7DEB796
:10D9B0002091D9072223D1F026960FB6F894DEBF26
:10D9C0000FBECDBFDF91CF911F910F91FF90EF90D0
:10D9D000DF90CF90BF90AF909F908F907F906F908F
:10D9E0005F904F903F902F900C944D588B011C01ED
:10D9F0008091FF0790910008A0910108B091020862
:10DA0000892B8A2B8B2B09F497C00E944D499801D2
:10DA1000220F331F220F331F3E832D83F901E35062
:10DA2000FB4F408051806280738080913102811170
:10DA300015C020E030E04AE754E4C301B2010E947F
:10DA40008EEC4B015C0120E030E04AE754E4C30176
:10DA5000B2010E948FEC6B017C0110C0ED81FE8150
:10DA6000E851F84F80809180A280B380ED81FE81E3
:10DA7000EB5DFD4FC080D180E280F3808091FF0795
:10DA800090910008A0910108B091020889839A83BF
:10DA9000AB83BC83BC01CD010E9472E82091F807E2
:10DAA0003091F9074091FA075091FB070E94D1E8A5
:10DAB0009B01AC01C301B2010E948FECAD81BE811C
:10DAC000A350BB4F3D01FD0160837183828393832B
:10DAD00029813A814B815C8157FF0DC0A5019401DA
:10DAE0000E946CE887FF1BC0D3018D929D92AD927E
:10DAF000BC92139714C029813A814B815C81232BFE
:10DB0000242B252B61F0A70196010E94B5EE181673
:10DB100034F4D301CD92DD92ED92FC921397C801BB
:10DB2000ADDE1092FF0710920008109201081092CB
:10DB3000020881E08093340280913402882329F125
:10DB4000C801880F991F880F991F83509B4F0E940F
:10DB50000FD7BC01C10126960FB6F894DEBF0FBEE9
:10DB6000CDBFDF91CF911F910F91FF90EF90DF908C
:10DB7000CF90BF90AF909F908F907F906F905F906D
:10DB80004F903F902F900C943A5F26960FB6F894E2
:10DB9000DEBF0FBECDBFDF91CF911F910F91FF90E0
:10DBA000EF90DF90CF90BF90AF909F908F907F903D
:10DBB0006F905F904F903F902F90089562E070E0DB
:10DBC00084EB91E3DFCE61E070E08DEA91E3DACEA1
:10DBD00060E070E086EA91E3D5CEAF92BF92CF923B
:10DBE000DF92EF92FF920F931F93CF93DF931092E8
:10DBF000D7078091FF0790910008A0910108B0918C
:10DC0000020881309048A105B10540F01092FF074D
:10DC1000109200081092010810920208C091FF07AC
:10DC20008091F7071816DCF4282F082E000C330B10
:10DC3000215031094C2F0C2E000C550B4217530765
:10DC400074F0CFEFC80F8C2F90E0A0E0B0E080938D
:10DC5000FF0790930008A0930108B0930208109268
:10DC6000C9078091C807C81714F4C093C8078091EA
:10DC7000C807082E000C990B04962C2F0C2E000CB4
:10DC8000330B8217930724F48CEF8C0F8093C80713
:10DC9000D091C80710E083E6E82E81E3F82E9DE3DB
:10DCA000C92E91E3D92E29E8A22E21E3B22ED1115B
:10DCB00017C080913402882349F081E0C11180E0CF
:10DCC00024E041EA51E3612F0E949CD88091D9075A
:10DCD000882309F47DC0C1117BC00E944D5874C0D7
:10DCE000D130D1F480913402882351F081E0C130E9
:10DCF00009F080E023E047E951E3612F0E949CD8BE
:10DD00008091D907882309F463C0C13009F060C04D
:10DD10008CEC9CEA5FDD58C0D230D9F4809134029B
:10DD2000882351F081E0C23009F080E020E24DE824
:10DD300051E3612F0E949CD88091D907882309F470
:10DD400047C0C23009F044C0B0922308A092220814
:10DD500039C0D330E9F480913402882351F081E056
:10DD6000C33009F080E020E248E751E3612F0E94D0
:10DD70009CD88091D907882359F1C33049F5D092B6
:10DD80002308C09222080E94DE480E9447581CC007
:10DD9000D430F1F480913402882351F081E0C43012
:10DDA00009F080E020E247E651E3612F0E949CD811
:10DDB0008091D907882361F0C43051F4F092230890
:10DDC000E09222080E94DE488091C90781117EC03E
:10DDD0008091110890911208209115083091160831
:10DDE000232B11F4892B31F1D53031F58091340298
:10DDF000882351F081E0C53009F080E020E24AE557
:10DE000051E3612F0E949CD88091D907882309F49F
:10DE10005BC0C53009F058C0109214081092130866
:10DE20000E9446D10E9447588091C907882309F46F
:10DE30004BC04CC005E001C006E0D0131DC080916E
:10DE40003402882349F081E0CD1380E023E04EE4E2
:10DE500051E3612F0E949CD88091D907882359F003
:10DE6000CD1309C085E590E7B5DC8091C907811124
:10DE70002DC00C2F01C00D2F81E0800FD81749F065
:10DE80001F5FDF5F153009F012CF0E5F0093F707B9
:10DE90001DC080913402882349F081E0CD1380E0D9
:10DEA00023E042E451E3612F0E949CD88091D9077E
:10DEB000882331F3CD13E4CF81E79FE68BDC80919B
:10DEC000C9078823E9F202C006E0D6CFDF91CF91DF
:10DED0001F910F91FF90EF90DF90CF90BF90AF9088
:10DEE00008951F93CF93DF931092D7078091FF0778
:10DEF00090910008A0910108B091020881309048EB
:10DF0000A105B10540F01092FF0710920008109291
:10DF1000010810920208C091FF078091F6071816B9
:10DF2000DCF4282F082E000C330B215031094C2F24
:10DF30000C2E000C550B4217530774F0CFEFC80F8F
:10DF40008C2F90E0A0E0B0E08093FF079093000852
:10DF5000A0930108B09302081092C9078091C807E6
:10DF6000C81714F4C093C8078091C807082E000C86
:10DF7000990B04962C2F0C2E000C330B8217930751
:10DF800024F48CEF8C0F8093C8071091C807D0E061
:10DF9000111117C080913402882349F081E0C1112A
:10DFA00080E024E045E351E36D2F0E949CD88091EE
:10DFB000D907882309F46DC0C1116BC00E944D5868
:10DFC00064C01130F9F480913402882351F081E06B
:10DFD000C13009F080E020E249E251E36D2F0E9458
:10DFE0009CD88091D907882309F453C0C13009F027
:10DFF00050C04091130E5091140E60910B0E709111
:10E000000C0E1CC01230F9F480913402882351F0B8
:10E0100081E0C23009F080E020E249E151E36D2F58
:10E020000E949CD88091D907882399F1C23089F544
:10E030004091130E5091140E6FEF7FEF80910F0EF1
:10E040009091100E20C0133021F580913402882366
:10E0500051F081E0C33009F080E020E249E051E373
:10E060006D2F0E949CD88091D907882391F0C330EE
:10E0700081F44091130E5091140E60910B0E70912B
:10E080000C0E80E090E00E94997A8091C90781117E
:10E0900008C0DF5F1F5FD53009F07ACF84E080933E
:10E0A000F607DF91CF911F9108951F93CF93DF93D0
:10E0B0001092D7078091FF0790910008A091010866
:10E0C000B091020881309048A105B10540F010924E
:10E0D000FF07109200081092010810920208C091E8
:10E0E000FF078091F5071816DCF4282F082E000C86
:10E0F000330B215031094C2F0C2E000C550B4217BD
:10E10000530774F0CFEFC80F8C2F90E0A0E0B0E081
:10E110008093FF0790930008A0930108B093020832
:10E120001092C9078091C807C81714F4C093C80794
:10E130008091C807082E000C990B04962C2F0C2EEA
:10E14000000C330B8217930724F48CEF8C0F809311
:10E15000C8071091C807D0E0111117C08091340290
:10E16000882349F081E0C11180E024E041E051E3DF
:10E170006D2F0E949CD88091D907882309F46DC027
:10E18000C1116BC00E944D5864C01130F9F48091E8
:10E190003402882351F081E0C13009F080E020E2B0
:10E1A00045EF50E36D2F0E949CD88091D9078823BA
:10E1B00009F453C0C13009F050C04091110E509184
:10E1C000120E6091090E70910A0E1CC01230F9F403
:10E1D00080913402882351F081E0C23009F080E060
:10E1E00020E245EE50E36D2F0E949CD88091D90724
:10E1F000882399F1C23089F54091110E5091120E89
:10E200006FEF7FEF80910D0E90910E0E20C01330B6
:10E2100021F580913402882351F081E0C33009F068
:10E2200080E020E245ED50E36D2F0E949CD8809164
:10E23000D907882391F0C33081F44091110E509199
:10E24000120E6091090E70910A0E80E090E00E941B
:10E25000997A8091C907811108C0DF5F1F5FD530AF
:10E2600009F07ACF84E08093F507DF91CF911F9179
:10E270000895FF920F931F93CF93DF931092D707C8
:10E280008091FF0790910008A0910108B0910208C9
:10E2900081309048A105B10540F01092FF0710921F
:10E2A00000081092010810920208C091FF078091A7
:10E2B000F4071816DCF4282F082E000C330B21501D
:10E2C00031094C2F0C2E000C550B4217530774F0DC
:10E2D000CFEFC80F8C2F90E0A0E0B0E08093FF0755
:10E2E00090930008A0930108B09302081092C90708
:10E2F0008091C807C81714F4C093C8078091C80755
:10E30000082E000C990B04962C2F0C2E000C330BAE
:10E310008217930724F48CEF8C0F8093C807109119
:10E32000C807D0E0FF24F394111117C08091340284
:10E33000882349F081E0C11180E024E040ED50E302
:10E340006D2F0E949CD88091D907882309F4E4C0DE
:10E35000C111E2C00E944D58DBC0113021F58091FF
:10E360003402882379F083E292E00E9441D89C0134
:10E3700081E0C13009F080E000E04AEC50E36D2F0D
:10E380000E948CDE8091D907882309F4C5C0C13072
:10E3900009F0C2C027EE33E04AE050E063E272E0E9
:10E3A00084EC90E3B3C0123071F58091340288237D
:10E3B00079F081E198E00E9441D89C0181E0C2306F
:10E3C00009F080E000E04DEB50E36D2F0E948CDE01
:10E3D0008091D907882309F49FC0C23009F09CC0FE
:10E3E000F092D7071092D3071092D4071092D50756
:10E3F0001092D6072AE932E744E051E061E178E083
:10E4000086EB90E32FC0133081F58091340288238E
:10E4100079F085E198E00E9441D89C0181E0C33009
:10E4200009F080E000E042EB50E36D2F0E948CDEAB
:10E430008091D907882309F46FC0C33009F06CC0FC
:10E44000F092D7071092D3071092D4071092D507F5
:10E450001092D6072DE932E747E850E065E178E011
:10E460008EEA90E30E946DE053C0143061F5809114
:10E470003402882379F083E198E00E9441D89C011E
:10E4800081E0C43009F080E000E044EA50E36D2F01
:10E490000E948CDE8091D9078823F1F1C430E1F528
:10E4A000F092D7071092D3071092D4071092D50795
:10E4B0001092D6072FEF30E040E050E063E178E0C3
:10E4C0008AE990E323C0153039F58091340288231E
:10E4D00079F081E292E00E9441D89C0181E0C53050
:10E4E00009F080E000E045E950E36D2F0E948CDEEA
:10E4F0008091D907882381F0C53071F427EE33E08D
:10E500004AE050E061E272E080E990E30E9417E0A7
:10E510008091C907811108C0DF5F1F5FD53009F006
:10E5200003CF86E08093F407DF91CF911F910F9185
:10E53000FF90089580E00C9413D10C94E0D0EF92FA
:10E54000FF921F93CF93DF937C017093FE0760933C
:10E55000FD071092D7078091FF0790910008A091C6
:10E560000108B091020881309048A105B10540F042
:10E570001092FF07109200081092010810920208F2
:10E58000C091FF078091FC071816DCF4282F082E95
:10E59000000C330B215031094C2F0C2E000C550B65
:10E5A0004217530774F0CFEFC80F8C2F90E0A0E014
:10E5B000B0E08093FF0790930008A0930108B09308
:10E5C00002081092C9078091C807C81714F4C093B5
:10E5D000C8072091C807022E000C330B2C5F3F4F59
:10E5E0008C2F0C2E000C990B2817390724F48CEF74
:10E5F0008C0F8093C8071091C807D0E091E081E0AC
:10E60000E816F10459F122E0E216F10409F448C0D9
:10E61000E114F10409F066C0111189C09923B1F029
:10E620001C16A4F08091FF0790910008A0910108AA
:10E63000B09102080196A11DB11D8093FF07909330
:10E640000008A0930108B0930208CF5F80913402C4
:10E65000882309F4D7C063E072E365C0111167C075
:10E660009923B1F01C16A4F08091FF079091000847
:10E67000A0910108B09102080196A11DB11D8093DF
:10E68000FF0790930008A0930108B0930208CF5FA2
:10E6900080913402882309F4B5C06CEF71E343C064
:10E6A000111145C09923B1F01C16A4F08091FF0709
:10E6B00090910008A0910108B09102080196A11D57
:10E6C000B11D8093FF0790930008A0930108B093B9
:10E6D0000208CF5F80913402882309F493C065EF6C
:10E6E00071E321C0111123C09923B1F01C16A4F0CD
:10E6F0008091FF0790910008A0910108B091020855
:10E700000196A11DB11D8093FF0790930008A0936F
:10E710000108B0930208CF5F80913402882309F486
:10E7200071C06CEE71E38D2F0E9457E36BC0113006
:10E73000C9F480913402882351F081E0C13009F09E
:10E7400080E024E042EE51E36D2F0E949CD880913E
:10E75000D907882309F456C0C13009F053C00E947C
:10E760004D584CC01230B9F480913402882351F0D6
:10E7700081E0C23009F080E023E048ED51E36D2FE5
:10E780000E949CD88091D9078823E1F1C230D1F54D
:10E790008FEF9BE631C01330B9F4809134028823A7
:10E7A00051F081E0C33009F080E023E04FEC51E309
:10E7B0006D2F0E949CD88091D907882319F1C3300E
:10E7C00009F584E19CE618C01430E1F4809134022C
:10E7D000882351F081E0C43009F080E023E044EC6C
:10E7E00051E36D2F0E949CD88091D907882351F066
:10E7F000C43041F489E29CE60E94EA6B8091C9072B
:10E80000811108C0DF5F1F5F90E0D53009F0F7CEBF
:10E81000D093FC07DF91CF911F91FF90EF90089567
:10E82000EF92FF920F931F93CF93DF93CDB7DEB795
:10E830006F970FB6F894DEBF0FBECDBF7B0106ED1C
:10E8400011E128ED31E1F8013183208322E030E04D
:10E850003093101420930F1490931214809311147A
:10E8600040E050E0BA018CED91E10E94308FF80158
:10E87000808191812BE1FC013496DE011596019097
:10E880000D922A95E1F7FC01828193819C838B8311
:10E8900080E893E09A838983A701BE016F5F7F4F71
:10E8A0008AE094E00E9450C6CE0101960E94AF4FCC
:10E8B0006F960FB6F894DEBF0FBECDBFDF91CF913C
:10E8C0001F910F91FF90EF90089510928A118091FF
:10E8D0005813882321F085E593E10C948C910895D9
:10E8E000E091F810F091F9100190F081E02D682F7F
:10E8F00088EF90E11994CF93DF93809135118111C6
:10E9000007C081E0809335118CEF90E10E940251A5
:10E91000C091FE10D091FF10E0912D11F0912E11B9
:10E9200082E01995E0912D11F0912E1181E0199559
:10E9300020E030E044E1BE018CEF90E10E94805085
:10E940002FE231E147E1BE018CEF90E10E9480505F
:10E95000E0912D11F0912E1180E0DF91CF9119946B
:10E960006F927F928F929F92AF92BF92DF92EF92BF
:10E97000FF920F931F93CF93DF93CDB7DEB7AD9781
:10E980000FB6F894DEBF0FBECDBF20918B112223AE
:10E9900009F4EFC1D62E7C0180915813882309F425
:10E9A0009FC0442309F4BAC180917013882329F1D0
:10E9B000E3E5F3E384918F010F5F1F4F882321F07C
:10E9C0000E945C87F801F6CFE0E1F3E384918F01C8
:10E9D0000F5F1F4F882321F00E945C87F801F6CF5C
:10E9E00061E070E080E090E00E94C9878AE00E94C8
:10E9F0005C8787E093E30E94B78A8FE28093751368
:10EA0000B12C21E006E713E19FE1A92E80912D139F
:10EA1000B816B8F4AB9CC0011124B80185509E4EC5
:10EA20002DA70E943C91C8012DA58C010196F801EB
:10EA30003081332321F02D3811F02F5FF6CFB394BE
:10EA4000E5CF27FD08C0B80185E593E10E943C9120
:10EA5000E8EBF3E403C0F8011082FACF84918F0150
:10EA60000F5F1F4F882321F00E945C87F801F6CFCB
:10EA7000B7018EEE92E30E94558260917013FDE81B
:10EA80006F9FB00111246B587C4E83EE92E30E947D
:10EA900055824091061450910714609108147091AA
:10EAA00009148DED92E30E94ED818AE00E945C875B
:10EAB0008091701394E0899FF0011124EF58FC4E6F
:10EAC0004091061450910714609108147091091434
:10EAD00040835183628373838F5F809370130DC073
:10EAE0001092701382E0B82E1BC1B70180ED92E343
:10EAF0000E9455828AE00E945C87E7DE1D821886AC
:10EB00001C821B8280E893E09A83898387EB91E1E2
:10EB10009093D7118093D611F70180818F3209F03D
:10EB200067C087010F5F1F4FCE0101963C010115A1
:10EB3000110509F463C06FE270E0C8010E94C8EFDC
:10EB40005C01009709F45BC00817190708F057C06B
:10EB50004C01801A910AA401B801CE0180960E944E
:10EB6000F1EFE0E2F0E0EC0FFD1FE80DF91D10827F
:10EB7000FE01B0964F018F01F80181918F0188232A
:10EB800019F00E945C87F8CF8AE00E945C87609150
:10EB9000D6117091D7116115710511F06C5F7F4F1F
:10EBA00021E0AE01405E5F4FCE0105960E941294B7
:10EBB000811116C0ECEBF2E384918F010F5F1F4FC0
:10EBC000882321F00E945C87F801F6CFF40181913F
:10EBD0004F01882319F00E945C87F8CF8EE287C02E
:10EBE0007092D7116092D61185010F5F1F4F9FCF92
:10EBF00088ED91E19093D7118093D6118701909180
:10EC0000D6118091D711692F782FDD2009F459C0D2
:10EC10006115710511F06C5F7F4F21E0A80185E55A
:10EC200093E10E941294882309F447C080916613EF
:10EC300090916713A0916813B091691380930214A7
:10EC400090930314A0930414B0930514B8018EEAB2
:10EC500092E30E94558240910214509103146091F6
:10EC600004147091051486EA92E30E94ED818AE013
:10EC70000E945C87109206141092071410920814D8
:10EC800010920914E7E9F2E384917F019FEFE91AFA
:10EC9000F90A882321F00E945C87F701F5CFB801BB
:10ECA00080E090E0BDDD80919A11882319F08AE917
:10ECB00091E101C0C80160E02AC0B80183E892E395
:10ECC00010C06115710511F06C5F7F4F26E5A8013A
:10ECD00085E593E10E94129481110CC0B8018FE682
:10ECE00092E30E9455828EE20E945C878AE00E9435
:10ECF0005C870FC081E080938811B7018DE592E3B6
:10ED00000E9455828AE00E945C8760E0C8010E94F0
:10ED10004CD9CE0101960E94AF4F2BC0BB24B394B7
:10ED2000E8EBF3E484918F010F5F1F4F882321F0FC
:10ED30000E945C87F801F6CFE8EDF2E384918F0141
:10ED40000F5F1F4F882321F00E945C87F801F6CFE8
:10ED5000E1E0BE1619F00BEE13E002C001EF13E084
:10ED6000F80181918F01882309F4BFCE0E945C874E
:10ED7000F7CFAD960FB6F894DEBF0FBECDBFDF91D3
:10ED8000CF911F910F91FF90EF90DF90BF90AF90C8
:10ED90009F908F907F906F900895CF92DF92EF9227
:10EDA000FF920F931F93CF93DF93CDB7DEB7EDB6EE
:10EDB000FEB6DC010D900020E9F79D01281B390B00
:10EDC0002C5F3F4F4DB75EB7421B530B0FB6F89405
:10EDD0005EBF0FBE4DBF0DB71EB70F5F1F4F9F9396
:10EDE0008F9386E592E39F938F931F930F930E94D7
:10EDF00005E8680154E0C50ED11C0F900F900F90EC
:10EE00000F900F900F90F6018081882349F0082E13
:10EE1000000C990B0E948CEFF60181936F01F3CFE8
:10EE200060E0C8010E94C248882319F0C8010E940E
:10EE3000888A82E592E390932308809322080E94B7
:10EE4000DE480FB6F894FEBE0FBEEDBEDF91CF9147
:10EE50001F910F91FF90EF90DF90CF900895AF92A8
:10EE6000BF92CF92DF92EF92FF920F931F93CF93B7
:10EE7000DF93CDB7DEB7AA970FB6F894DEBF0FBE0B
:10EE8000CDBF8091B6118F938091B5118F9389E496
:10EE900092E39F938F937E0181E2E80EF11CFF9233
:10EEA000EF920E9405E80F900F900F900F900F9037
:10EEB0000F9010E0F70101900020E9F73197EE196B
:10EEC000FF091E1784F46701C10ED11C17FDDA94E7
:10EED000F6018081082E000C990B0E948CEFF60140
:10EEE00080831F5FE7CF40E050E0BA018BEB91E1F8
:10EEF0000E94308F00E0CE0101966C018091BE111E
:10EF0000823028F4011114C08FEF9FEF16C080915A
:10EF1000C3119091C411A091C511B091C6118F7108
:10EF20009927AA27BB27892B8A2B8B2B59F71AC025
:10EF30008091B5119091B61101969093B61180937E
:10EF4000B511AA960FB6F894DEBF0FBECDBFDF9104
:10EF5000CF911F910F91FF90EF90DF90CF90BF90D6
:10EF6000AF90089540E050E0B6018BEB91E10E9434
:10EF70006B8418163CF6F60101900020E9F73197F2
:10EF80001E2F1C19115068F05601A10EB11C17FD5F
:10EF9000BA94F501808190E00E948CEFF5018083A6
:10EFA000F1CF8A858E3709F4A9CF45E050E0B7014B
:10EFB000C6010E94E3EF892B09F0A0CFC701EDDE67
:10EFC00001E09CCFCF92DF92EF92FF921F93CF93FD
:10EFD000DF9310928B118091BE11882321F08BEB6F
:10EFE00091E10E948C911092321310922F1385E3BD
:10EFF00080932E130E94D75BEB01A89561E080916E
:10F000002E130E949C5A8EE293E10E9485962398CB
:10F01000229A219A209A289A85E08093301382E5DB
:10F020008CBD1DBC1AE08FEF0E948A961150D9F753
:10F0300020E030E0A90160E08EE293E10E94969624
:10F04000182F80933113813049F00E94D75B6C1BDD
:10F050007D0B613D774060F381E054C02AEA31E0E6
:10F0600040E050E068E08EE293E10E94969682FFD5
:10F0700003C0109332130EC014E00E948F96809349
:10F0800031131150D1F78A3A11F082E03BC082E08F
:10F090008093321380913213823021F0C12CD12C15
:10F0A000760105C0C12CD12CE12C80E4F82E20E0A3
:10F0B00030E0A90167E38EE293E10E949696A701F2
:10F0C000960169E28EE293E10E9496968093311355
:10F0D000882349F00E94D75B6C1B7D0B613D774014
:10F0E00030F38AE00FC080913213823011F520E0B6
:10F0F00030E0A9016AE38EE293E10E9496968823AC
:10F1000051F088E080932F138EE293E10E94859660
:10F11000E8EBF3E41AC00E948F96807C803C19F4DF
:10F1200083E0809332130E948F960E948F960E94F4
:10F130008F968EE293E10E9485961092301381E0C3
:10F140000E94F0C3811132C015C08491EF01219655
:10F15000882321F00E945C87FE01F7CFEBE3F2E306
:10F160008491EF012196882309F457C00E945C879F
:10F17000FE01F6CF80E00E94F0C3811117C0E3E5E5
:10F18000F3E38491EF012196882321F00E945C87AC
:10F19000FE01F7CFE7E2F2E38491EF0121968823A5
:10F1A00009F43BC00E945C87FE01F6CF63E373E184
:10F1B0008BEB91E10E94E990811116C0E3E5F3E346
:10F1C0008491EF012196882321F00E945C87FE0143
:10F1D000F7CFE6E1F2E38491EF0121968823E9F08D
:10F1E0000E945C87FE01F7CF81E080938B11E8EBF2
:10F1F000F3E48491EF012196882321F00E945C873B
:10F20000FE01F7CFEAE0F2E38491EF012196882333
:10F2100021F00E945C87FE01F7CF8BE1EBEBF1E17F
:10F22000ACEDB1E101900D928A95E1F78091B911B1
:10F230009091BA119093DB118093DA1187EB91E1F1
:10F240009093D7118093D611DF91CF911F91FF90AA
:10F25000EF90DF90CF9008950F931F93CF93DF939C
:10F260008C01EB019091681120916911921307C0F4
:10F270008CE591E10E940E450E9488D3F3CFF801FE
:10F28000A081B181488159818091671134E0839FC9
:10F29000F0011124E05AFE4EB387A28755874487B8
:10F2A0009F5F909368118F5F821719F080936711A9
:10F2B00002C010926711DF91CF911F910F910895B5
:10F2C000CF93DF93CDB7DEB780912108811110C0B5
:10F2D0009E01275F3F4F4F81588562E470E087E6CB
:10F2E00092E00E9434E80E949FC583E0809334023C
:10F2F000DF91CF91089580917A1190917B118130A7
:10F300009105B9F1029759F40E9469C560937C1187
:10F3100070937D1180937E1190937F1118C010928D
:10F32000801110928111109282111092831110920B
:10F3300084111092851110928611109287111092EB
:10F340007C1110927D1110927E1110927F1181E03C
:10F3500090E090937B1180937A110E94D75B609329
:10F36000801170938111809382119093831181E0B9
:10F37000089580E0089580917A1190917B11019712
:10F3800091F482E090E090937B1180937A110E9437
:10F39000D75B60938411709385118093861190934D
:10F3A000871181E0089580E00895BC0180E090E03D
:10F3B0004AE00E9463878DE00E945C878AE00C949B
:10F3C0005C878F929F92AF92BF92CF92DF92EF9223
:10F3D000FF92CF9320E030E04AE754E4FC016081E3
:10F3E0007181828193810E94D1E80E94D3ED6B01EB
:10F3F0007C01611571058105910561F097FF0AC0D7
:10F40000F094E094D094C094C11CD11CE11CF11C78
:10F410008DE201C080E280931A08C701B60128EE90
:10F4200033E040E050E00E9453EC8AE0882E912CBB
:10F43000A12CB12CCA01B901A50194010E9453EC81
:10F44000605D60931B088EE280931C08C701B601C3
:10F4500024E630E040E050E00E9453ECCA01B901DC
:10F46000A50194010E9453EC605D60931D08C701E3
:10F47000B601A50194010E9453ECC62FCA01B9013F
:10F48000A50194010E9453EC605D60931E08C05D6D
:10F49000C0931F088AE198E0CF91FF90EF90DF9032
:10F4A000CF90BF90AF909F908F900895FF920F9351
:10F4B0001F93CF93DF931F92CDB7DEB7982F862F80
:10F4C000692F49830E940E5E909130118091180837
:10F4D0004981891738F19091321180911708981756
:10F4E00008F180919A118823D1F01092AF110AE9A6
:10F4F00011E1442319F082E00E94075F85E1F82EB4
:10F50000F80181918F01882321F00E94F05EF81AA2
:10F51000F7CFFF2039F080E2E3D9FA94FACF0DE873
:10F5200011E1E7CF0F90DF91CF911F910F91FF90E5
:10F5300008950F931F93CF93DF93EB018A01181661
:10F5400019066CF4843121E0920714F083E191E014
:10F55000909312088093110880E00E9413D1D7FD88
:10F5600006C0D0931608C09315080E94E0D01093EF
:10F57000140800931308DF91CF911F910F910C9401
:10F580004758CF93DF931F92CDB7DEB7698341E031
:10F5900050E0BE016F5F7F4F04960E9403950F906D
:10F5A000DF91CF9108958091F40C80FF03C0899A78
:10F5B0008FEF02C0899881E0809335028091F40C2E
:10F5C00081FF03C08F988FEF02C08F9A81E08093F4
:10F5D00036028091F40C9FB782FF09C0F8948091A5
:10F5E0000B01826080930B019FBF8FEF08C0F894DE
:10F5F00080910B018D7F80930B019FBF81E08093F1
:10F6000037028091F40C83FF03C016988FEF02C07D
:10F61000169A81E080933802089590915A11809152
:10F620005B11981731F080915B118F5F8F70809321
:10F630005B1108951F920F920FB60F9211240BB613
:10F640000F92BF92CF92DF92EF92FF920F931F9390
:10F650002F933F934F935F936F937F938F939F93DA
:10F66000AF93BF93EF93FF93CF93DF9300D01F929D
:10F67000CDB7DEB780916E008B7F80936E00809156
:10F680006F008D7F80936F007894C090150DD0909F
:10F69000160DE090170DF090180DC114D104E1047F
:10F6A000F10409F442C080910B02811104C08091E1
:10F6B000F0048823D1F10E945849F9EBCF16FBE002
:10F6C000DF06E104F10488F008EBC01A0BE0D00A71
:10F6D000E108F108C092150DD092160DE092170DB9
:10F6E000F092180D88EB9BE009C0C6011092150D31
:10F6F0001092160D1092170D1092180D909389000C
:10F700008093880020918800309189008091840046
:10F710009091850040962817390708F06DC08091B8
:10F7200084009091850040961FC08091F50C9091C7
:10F73000F60C009709F493C08C0101501109109345
:10F74000F60C0093F50C10921A141092191465DF40
:10F75000012B41F48AE59BE39093230880932208D0
:10F760000E94DE4888EC90E09093890080938800A6
:10F7700043C0C8011ADE24E630E080910B028823E2
:10F7800009F4B9C4C901293BBBE03B0708F0ECC54B
:10F7900090938900809388008091070D9091080DC7
:10F7A000A091090DB0910A0D820F931FA11DB11DEB
:10F7B0008093070D9093080DA093090DB0930A0D47
:10F7C000209188003091890080918400909185007B
:10F7D00040962817390748F480918400909185005D
:10F7E00040969093890080938800BB2029F0109266
:10F7F0001A141092191411DFF8948091B706882317
:10F8000021F080916E008B7F03C080916E00846038
:10F8100080936E0080916F00826080936F000F90E4
:10F820000F900F900F90DF91CF91FF91EF91BF91CB
:10F83000AF919F918F917F916F915F914F913F9188
:10F840002F911F910F91FF90EF90DF90CF90BF907D
:10F850000F900BBE0F900FBE0F901F901895E09168
:10F860001914F0911A14309709F0B1C190915A11FE
:10F8700080915B11981751F1E0915B111DE4E19FBC
:10F88000F0011124EC5DF74FC090CE07D090CF0768
:10F89000E090D007F090D1079F01275B3F4FD9013F
:10F8A0004D915D916D917C91D701C601841B950BA3
:10F8B000A60BB70B8093CE079093CF07A093D007EA
:10F8C000B093D1078081886080830BC08FB7F89494
:10F8D0001092CE071092CF071092D0071092D10746
:10F8E0008FBFF0931A14E0931914309709F46CC188
:10F8F00052A18091F40C418158130AC0242F30E0AA
:10F9000080913902082E000C990B2817390729F02D
:10F910005093F40C4093390246DE1092110D109270
:10F92000120D1092130D1092140DE0911914F09114
:10F930001A1487A990AD8134BCE99B0728F4813261
:10F94000EEE49E0748F002C080E49CE99695879516
:10F950009695879524E007C08131F7E29F0730F044
:10F960009695879522E02093100D08C021E0209302
:10F97000100D8032910510F480E290E07C0100E2ED
:10F98000E01AF108E11418E0F106E0F0EF2DFF278E
:10F99000EE0FFF1FEE0FFF1FCF01865A984CFC01A0
:10F9A0003296459154916E2DAA27659F9001649FD0
:10F9B000210D3A1F06942A1F3A1F1124FC0185913C
:10F9C00094911CC09701369527952C7F265A3C4C64
:10F9D000F90185919491F901329665917491A7018D
:10F9E00047705527649F9001659F300D749F300DBF
:10F9F0001124B3E036952795BA95E1F7821B930B56
:10FA00008436910570F407EF13E0D8018D918D01D4
:10FA1000882319F00E945C87F8CFC701C6DC84E612
:10FA200090E090930F0D80930E0D8091100D8093B8
:10FA30000D0DE0911914F0911A1483AD94AD9093CB
:10FA40000C0D80930B0D8134BCE99B0728F48132A7
:10FA5000EEE49E0748F002C080E49CE99695879505
:10FA60009695879524E007C08131F7E29F0730F033
:10FA70009695879522E02093100D08C021E02093F1
:10FA8000100D8032910510F480E290E07C0100E2DC
:10FA9000E01AF108E11418E0F106E0F0EF2DFF277D
:10FAA000EE0FFF1FEE0FFF1FCF01865A984CFC018F
:10FAB0003296459154916E2DAA27659F9001649FBF
:10FAC000210D3A1F06942A1F3A1F1124FC0185912B
:10FAD00094911CC09701369527952C7F265A3C4C53
:10FAE000F90185919491F901329665917491A7017C
:10FAF00047705527649F9001659F300D749F300DAE
:10FB0000112453E0369527955A95E1F7821B930B04
:10FB10008436910570F407EF13E0D8018D918D01C3
:10FB2000882319F00E945C87F8CFC7013EDC84E689
:10FB300090E0AC0160E070E04093070D5093080D39
:10FB40006093090D70930A0D90938900809388004B
:10FB5000E0911914F0911A1482899389A489B589C6
:10FB6000B695A79597958795B095A0959095819511
:10FB70009F4FAF4FBF4F8093030D9093040DA09301
:10FB8000050DB093060D8093FF0C9093000DA0938C
:10FB9000010DB093020D8093FB0C9093FC0CA0938D
:10FBA000FD0CB093FE0C8093F70C9093F80CA0938F
:10FBB000F90CB093FA0C10921514109216141092BE
:10FBC00017141092181403C080ED97E0CDCD8091EA
:10FBD0000B028111C6C38091F0048111C2C3209130
:10FBE000100D222309F4AFC1E0911914F0911A14F9
:10FBF0004091F70C5091F80C6091F90C7091FA0C4F
:10FC000082819381A481B581840F951FA61FB71FA0
:10FC10008093F70C9093F80CA093F90CB093FA0C26
:10FC2000181619061A061B060CF4889AE091191486
:10FC3000F0911A144091FB0C5091FC0C6091FD0C5A
:10FC40007091FE0C86819781A085B185840F951FE8
:10FC5000A61FB71F8093FB0C9093FC0CA093FD0C88
:10FC6000B093FE0C181619061A061B060CF48E9A91
:10FC7000E0911914F0911A144091FF0C5091000D6D
:10FC80006091010D7091020D82859385A485B585E3
:10FC9000840F951FA61FB71F8093FF0C9093000D34
:10FCA000A093010DB093020D181619061A061B0633
:10FCB00044F49FB7F89480910B01886080930B0106
:10FCC0009FBFE0911914F0911A144091030D5091C7
:10FCD000040D6091050D7091060D86859785A089AC
:10FCE000B189840F951FA61FB71F8093030D9093B2
:10FCF000040DA093050DB093060D181619061A06EB
:10FD00001B060CF4149A8091F70C9091F80CA091BA
:10FD1000F90CB091FA0C181619061A061B0684F590
:10FD2000E0911914F0911A144289538964897589F4
:10FD3000841B950BA60BB70B8093F70C9093F80CD4
:10FD4000A093F90CB093FA0C8091350240911B14EA
:10FD500050911C1460911D1470911E14082E000CFB
:10FD6000990BAA0BBB0B840F951FA61FB71F80937F
:10FD70001B1490931C14A0931D14B0931E14889808
:10FD80008091FB0C9091FC0CA091FD0CB091FE0CAD
:10FD9000181619061A061B0684F5E0911914F0913D
:10FDA0001A144289538964897589841B950BA60BA3
:10FDB000B70B8093FB0C9093FC0CA093FD0CB093BD
:10FDC000FE0C8091360240911F14509120146091D6
:10FDD000211470912214082E000C990BAA0BBB0B56
:10FDE000840F951FA61FB71F80931F149093201494
:10FDF000A0932114B09322148E988091FF0C9091BF
:10FE0000000DA091010DB091020D181619061A06E9
:10FE10001B06BCF5E0911914F0911A14428953891C
:10FE200064897589841B950BA60BB70B8093FF0C17
:10FE30009093000DA093010DB093020D80913702B5
:10FE4000409123145091241460912514709126142C
:10FE5000082E000C990BAA0BBB0B840F951FA61F35
:10FE6000B71F8093231490932414A0932514B09368
:10FE700026149FB7F89480910B01877F80930B0124
:10FE80009FBF8091030D9091040DA091050DB0913D
:10FE9000060D181619061A061B0684F5E0911914AA
:10FEA000F0911A144289538964897589841B950BD2
:10FEB000A60BB70B8093030D9093040DA093050D33
:10FEC000B093060D80913802409127145091281468
:10FED0006091291470912A14082E000C990BAA0B1A
:10FEE000BB0B840F951FA61FB71F809327149093F9
:10FEF0002814A0932914B0932A14149880911514EF
:10FF000090911614A0911714B09118140196A11D88
:10FF1000B11D8093151490931614A0931714B093E9
:10FF200018142150E0911914F0911A144289538940
:10FF30006489758984179507A607B70708F451CE19
:10FF4000BB24B39401C0B12C4091151450911614E8
:10FF50006091171470911814E0901914F0901A140D
:10FF6000F70186899789A08DB18D84179507A6071B
:10FF7000B70708F4C6C04091070D5091080D609175
:10FF8000090D70910A0D068D178D20A131A1AA27A8
:10FF9000419FB12D529FC001629F900D619F800DC6
:10FFA000911D429FB00D811D9A1F519FB00D811D63
:10FFB0009A1F609FB00D811D9A1F509FB10D8A1F1F
:10FFC0009A1FB6958A1F9A1F349F800D911D359FE9
:10FFD000900D112423AD34AD820F931F90930C0D1F
:10FFE00080930B0D47A950AD61AD72ADA0E0B0E0BC
:10FFF000481759076A077B0720F450930C0D40936C
:020000021000EC
:100000000B0D80910B0D90910C0D8134BCE99B0779
:1000100028F48132EEE49E0748F002C080E49CE9B7
:10002000969587959695879524E007C08131F7E2EC
:100030009F0730F09695879522E02093100D08C019
:1000400021E02093100D8032910510F480E290E0C1
:100050008C0100521109011528E01207E8F0E12F88
:10006000FF27EE0FFF1FEE0FFF1FCF01865A984CA0
:10007000FC01329625913491AA27039FA001029F8B
:10008000410D5A1F06944A1F5A1F1124FC01259145
:100090003491241B350B1FC09801369527952C7F72
:1000A000265A3C4CF90145915491F90132966591DB
:1000B0007491980127703327629FC001639F900D50
:1000C000729F900D1124F3E096958795FA95E1F7CC
:1000D0009A01281B390B2436310508F04ECB77EFF7
:1000E000E72E73E0F72ED7018D917D01882309F467
:1000F00040CBE2D6F8CF8091F004811143CBC90107
:1001000047CB4091151450911614609117147091BB
:100110001814F701828D938DA48DB58D84179507E2
:10012000A607B70708F0EAC00091110D1091120D53
:100130002091130D3091140D09831A832B833C8376
:10014000468D578D60A171A1AA27059FB12D169FDD
:100150006001269FD00C259FC00CD11C069FB00DBE
:10016000C11CDA1E159FB00DC11CDA1E249FB00DF4
:10017000C11CDA1E149FB10DCA1EDA1EB695CA1E26
:10018000DA1E709FC00CD11C719FD00C112480917D
:100190000B0D90910C0DFF96C816D90680F48C19A2
:1001A0009D0940815181628173816C01E12CF12CA8
:1001B000C416D506E606F70620F4CA0102C08081FF
:1001C000918181341CE9910728F481322EE4920751
:1001D00048F002C080E49CE99695879596958795AE
:1001E00024E007C0813137E2930730F09695879578
:1001F00022E02093100D08C021E02093100D8032E2
:10020000910510F480E290E08C0100521109011573
:1002100048E01407E8F0E12FFF27EE0FFF1FEE0F75
:10022000FF1FCF01865A984CFC01329625913491DC
:10023000AA27039FA001029F410D5A1F06944A1F3F
:100240005A1F1124FC0125913491241B350B1FC02A
:100250009801369527952C7F265A3C4CF9014591FB
:100260005491F90132966591749198012770332762
:10027000629FC001639F900D729F900D112423E037
:10028000969587952A95E1F79A01281B390B243614
:10029000310578F487EFE82E83E0F82ED7018D91B1
:1002A0007D01882311F008D6F9CFC8017ED824E655
:1002B00030E080910B02811104C08091F00488230A
:1002C00039F0C901293BBBE03B0708F068C001C019
:1002D000C901909389008093880089819A81AB81BC
:1002E000BC81820F931FA11DB11D8093110D9093AE
:1002F000120DA093130DB093140D62CA20910E0D30
:1003000030910F0D80910B02811104C08091F00497
:100310008823F1F0293BEBE03E07D0F0C90168EB00
:100320007BE00E9453EF883E43E0940708F052C000
:100330008854944FA901481B590B60E070E040932A
:10034000150D5093160D6093170D7093180D9C01A9
:10035000309389002093880080910D0D8093100DBB
:100360002FCA0E9458493BCC68EB7BE00E9453EFB8
:10037000883E03E0900780F48854944FA901481BFD
:10038000590B60E070E04093150D5093160D60938B
:10039000170D7093180DFCC988EB9BE0EFCF68EB4D
:1003A0007BE00E9453EF883E13E0910780F488546D
:1003B000944FA901481B590B60E070E04093150D64
:1003C0005093160D6093170D7093180D82CF88EB24
:1003D0009BE0EFCF88EB9BE0ADCFCF92DF92EF9227
:1003E000FF92CF93DF936A017B01FC018491EF01BF
:1003F0002196882319F060D5FE01F8CF4AE0C701A5
:10040000B601DF91CF91FF90EF90DF90CF905BC569
:10041000CF92DF92EF92FF92CF93DF936A017B013D
:10042000FC018491EF012196882319F045D5FE0146
:10043000F8CF42E0C701B601DF91CF91FF90EF9076
:10044000DF90CF90C0C5CF92DF92EF92FF92CF9313
:10045000DF936A017B01FC018491EF0121968823DF
:1004600019F02AD5FE01F8CF42E0C701B601DF91AD
:10047000CF91FF90EF90DF90CF90A5C50F931F9382
:10048000CF93DF938B01FC018491EF0121968823A8
:1004900019F012D5FE01F8CFB801110F880B990B96
:1004A000DF91CF911F910F9174C50F931F93CF933D
:1004B000DF931F921F92CDB7DEB7FC0184918F01AD
:1004C0000F5F1F4F811102C08B0107C069837A83C0
:1004D000F3D4F80169817A81F1CFF80181918F011C
:1004E000882311F0E9D4F9CF0F900F90DF91CF91CD
:1004F0001F910F910895CF938091F3108823B9F144
:100500004091EB105091EC106091ED107091EE1055
:100510002BEE3EE08091F4109091F5100E94AE9188
:10052000C82F811102C0C0E023C04091EF1050914C
:10053000F0106091F1107091F210411551056105B4
:10054000710591F02BEE3EE08091F4109091F51042
:100550000E94AE91882339F31092EF101092F010A0
:100560001092F1101092F2101092F31001C0C1E03D
:100570008C2FCF910895CF92DF92EF92FF92CF937D
:100580006B017C01C42F8091EB109091EC10A09135
:10059000ED10B091EE108C159D05AE05BF05C9F0AC
:1005A000AADF811102C080E018C02BEE3EE0B70147
:1005B000A6018091F4109091F5100E940597882370
:1005C00091F3C092EB10D092EC10E092ED10F0920B
:1005D000EE1081E0C1118093F310CF91FF90EF9066
:1005E000DF90CF9008954F925F926F927F928F929B
:1005F0009F92AF92BF92CF92DF92EF92FF920F93B2
:100600001F93CF93DF93EC016A017B01280139012D
:10061000423051056105710510F480E064C08985A0
:100620009A85AB85BC850196A11DB11D84179507E0
:10063000A607B70790F38F89803149F48D2C9E2C43
:10064000AF2CBB248B899C89AD89BE890FC08032B9
:1006500021F78B889C88AD88BE88DB01CA0157E0F2
:10066000B695A795979587955A95D1F7880E991EB7
:10067000AA1EBB1E41E0C501B4017DDF882369F2DB
:100680009F89903161F4DD24EE24FF249601220F2E
:10069000331FF901E551F14F5182408211C0E894B6
:1006A000C7F8DD24EE24FF249601220F331F220F0A
:1006B000331FF901E551F14F40825182628273820A
:1006C0009A89923080F04D815E816F817885840EA9
:1006D000951EA61EB71E8092EF109092F010A09269
:1006E000F110B092F210DF91CF911F910F91FF9016
:1006F000EF90DF90CF90BF90AF909F908F907F90C2
:100700006F905F904F900895CF92DF92EF92FF929B
:100710000F931F93CF93DF93FC0181859285A3856F
:10072000B4850196A11DB11D84179507A607B707CB
:1007300010F480E061C08789803149F4BB27A72F7E
:10074000962F852FC388D488E588F6880FC080321D
:1007500081F783899489A589B6896A017B01C7E0FD
:10076000F694E794D794C794CA95D1F78C0D9D1D44
:10077000AE1DBF1DE9016A017B018F014091EB10A5
:100780005091EC106091ED107091EE108417950768
:10079000A607B70799F4F80187898031B1F4B7014A
:1007A000A601552766277727440F551FFA01E55103
:1007B000F14F80819181A0E0B0E019C040E0BC0120
:1007C000CD01D9DE8111E7CFB4CFB701A6014F77B4
:1007D000552766277727440F551F440F551FFA01E9
:1007E000E551F14F80819181A281B381BF708883EF
:1007F0009983AA83BB8381E0DF91CF911F910F91F1
:10080000FF90EF90DF90CF9008954F925F926F929C
:100810007F92AF92BF92CF92DF92EF92FF920F93AF
:100820001F93CF93DF9300D01F92CDB7DEB78C011B
:1008300049835A836B837C835901C12CD12C760167
:10084000412C82E0582E612C712C49815A816B8198
:100850007C819E012F5F3F4FC80156DF882341F105
:10086000D301C201F801058404C0880F991FAA1F93
:10087000BB1F0A94D2F7C80ED91EEA1EFB1E49817F
:100880005A816B817C818789803139F481E0483FCE
:100890005F4F6105710538F4D8CF81E0483F5F4F65
:1008A0006F4F7F4090F2F501C082D182E282F382E5
:1008B0000F900F900F900F90DF91CF911F910F919C
:1008C000FF90EF90DF90CF90BF90AF907F906F90B0
:1008D0005F904F900895DF92EF92FF920F931F93D6
:1008E000CF93DF937C01EB018A018DE0D82E40E2AB
:1008F00050E0BE01C7010E94C68F8032910539F0D9
:1009000021E0892B09F420E0822F81953EC02881C7
:10091000222399F1253E59F32E3249F30115110591
:1009200041F13B853F733F3021F54A8D5B8D452B6F
:1009300001F52F713FEF320F3230D8F430E0215003
:100940003109D29EC001D39E900D1124D801A80F69
:10095000B91FFE0120E0AD01253088F431813D93BF
:100960002F5F32962D30C1F7288126FF02C0FA0191
:1009700015862B8523FDBBCF08C080E006C02B3039
:1009800010F43481ECCF3681EACFDF91CF911F9103
:100990000F91FF90EF90DF900895CF92DF92EF924A
:1009A000FF92C0906302D0906402E0906502F090E4
:1009B00066028091790E882321F120E030E0A901C0
:1009C000C701B6010E946CE88823D9F020E030E02E
:1009D00040E05FE3C701B6010E94D1E89B01AC0192
:1009E0000E94D1E82BED3FE049E450E40E94D1E8B9
:1009F0009B01AC0160E070E080E89FE30E946BED3A
:100A000004C060E070E080E89FE36093430270936D
:100A100044028093450290934602FF90EF90DF904E
:100A2000CF9008954F925F926F927F92AF92BF9254
:100A3000CF92DF92EF92FF920F931F93CF93DF93AA
:100A4000009709F456C0FC01208121FD52C0EB0142
:100A50008C0147A050A461A472A4AFA0B8A4C9A4FB
:100A6000DAA49501A601C301B2010E946CE887FFD8
:100A700040C0A3019201C301B2010E94D1E82B0141
:100A80003C01F80183A994A9A5A9B6A9BC01CD018F
:100A900090589B01AC010E948FECF80127A530A96A
:100AA00041A952A90E94D1E89B01AC01C301B20146
:100AB0000E948EEC0E94FAEE7B018C019B01AC013E
:100AC000B501C6010E946CE887FF02C0750186016E
:100AD0009701A801B501C6010E946CE8882349F07E
:100AE000A701B8014FA358A769A77AA78881816099
:100AF0008883DF91CF911F910F91FF90EF90DF904E
:100B0000CF90BF90AF907F906F905F904F9008957F
:100B10002F923F924F925F926F927F928F929F920D
:100B2000AF92BF92CF92DF92EF92FF920F931F93FB
:100B3000CF93DF93CDB7DEB768970FB6F894DEBFDB
:100B40000FBECDBF1C015B018A01DC01D7966D9100
:100B50007D918D919C91DA970E9470E86B017C01E8
:100B6000F50120813181428153810E94D1E80E94A8
:100B700055ED0E94D8ED69877A878B879C87D801CD
:100B80002D913D914D915C91C701B6010E94D1E834
:100B90000E9455ED0E94D8ED6D877E878F87988BD8
:100BA00029853A854B855C852837310541055105F6
:100BB00040F488E790E0A0E0B0E089879A87AB87AF
:100BC000BC872D853E854F855889283731054105DD
:100BD000510540F488E790E0A0E0B0E08D879E8763
:100BE000AF87B88B91012D5B3F4FD9018D919D91BE
:100BF0000D90BC91A02D8D839E83AF83B887BC01DF
:100C0000CD010E9472E869837A838B839C83698516
:100C10007A858B859C850E9470E8698B7A8B8B8B9B
:100C20009C8B20E030E0A90169817A818B819C81D5
:100C30000E946CE8882339F1A7019601C701B6012B
:100C40000E94D1E84B015C0129893A894B895C8972
:100C5000CA01B9010E94D1E89B01AC01C501B401F0
:100C60000E948EEC4B015C0129813A814B815C81B1
:100C7000CA01B9010E948FEC9B01AC01C501B4010E
:100C80000E946BED03C060E070E0CB010E9455ED67
:100C90000E94D3ED2B013C016D817E818F8198856F
:100CA00090958095709561957F4F8F4F9F4F0E94D3
:100CB00072E84B015C016D857E858F8598890E9465
:100CC00070E86D837E838F83988720E030E0A901F0
:100CD000C501B4010E946CE8882349F12D813E8151
:100CE0004F815885CA01B9010E94D1E86D8B7E8B76
:100CF0008F8B988FA7019601C701B6010E94D1E89A
:100D00009B01AC016D897E898F89988D0E948EEC44
:100D10006B017C01A5019401C501B4010E948FEC17
:100D20009B01AC01C701B6010E946BED03C060E0FE
:100D300070E0CB010E9404EEF10182889388A488C0
:100D4000B58875016401C418D508E608F7080E9443
:100D5000D3EDC61AD70AE80AF90AF7FE6BC020E0FD
:100D600030E0A90169817A818B819C810E946CE8C5
:100D7000882309F447C029813A814B815C81CA01EB
:100D8000B9010E948FEC6B017C01C501B4010E9486
:100D900070E89B01AC01C701B6010E94D1E86B016C
:100DA0007C0129893A894B895C89CA01B9010E9471
:100DB000D1E89B01AC01C701B6010E948EEC6B012A
:100DC0007C012D813E814F815885CA01B9010E9465
:100DD000D1E89B01AC01C701B6010E948FEC6B0109
:100DE0007C0120E030E040E850E469817A818B8129
:100DF0009C810E94D1E89B01AC01C701B6010E9411
:100E00006BED03C060E070E0CB010E9455ED0E94E5
:100E1000D3ED2B013C0197FF03C0412C512C320133
:100E2000481459046A047B0410F024013501C12CD4
:100E3000D12C76018FB7F894D1019C9193FD22C0FB
:100E4000F101468A578A608E718EC40CD51CE61C4F
:100E5000F71C5A96CD92DD92ED92FC925D97298512
:100E60003A854B855C85DB962D933D934D935C9342
:100E7000DE97FF962D853E854F85588920833183E7
:100E8000428353838FBF68960FB6F894DEBF0FBEC0
:100E9000CDBFDF91CF911F910F91FF90EF90DF9029
:100EA000CF90BF90AF909F908F907F906F905F900A
:100EB0004F903F902F9008959091C00095FFFCCFE8
:100EC0008093C60008958F929F92AF92BF92EF9247
:100ED000FF921F93CF93DF93CDB7DEB7A0970FB6E6
:100EE000F894DEBF0FBECDBF611571058105910578
:100EF00079F110E0842E912CA12CB12CEE24E394F6
:100F0000F12CEC0EFD1EE10EF11C17FDFA94A5016B
:100F100094010E9431ECF7016083B901CA011F5F9F
:100F2000611571058105910549F7115010F1E1E056
:100F3000F0E0EC0FFD1FE10FF11D17FDFA95808128
:100F40008A3010F097E301C090E3890FB5DFEDCF51
:100F500080E3A0960FB6F894DEBF0FBECDBFDF9141
:100F6000CF911F91FF90EF90BF90AF909F908F9087
:100F7000A3CFA0960FB6F894DEBF0FBECDBFDF9112
:100F8000CF911F91FF90EF90BF90AF909F908F9067
:100F90000895CF92DF92EF92FF926B017C0197FF51
:100FA0000AC08DE289DFF094E094D094C094C11C13
:100FB000D11CE11CF11C4AE0C701B601FF90EF9083
:100FC000DF90CF9080CF8F929F92AF92BF92CF92BF
:100FD000DF92EF92FF92CF936B017C01B42E20E061
:100FE00030E0A9010E946CE887FF06C08DE264DF53
:100FF000F7FAF094F7F8F094C0E060E070E080E079
:101000009FE3CB1541F02DEC3CEC4CEC5DE30E94F2
:10101000D1E8CF5FF6CF9B01AC01C701B6010E94BA
:101020008FEC6B017C010E94D8ED4B015C014AE022
:101030004ADFCC2379F1C501B4010E9470E89B011D
:10104000AC01C701B6010E948EEC6B017C018EE2FF
:1010500033DF20E030E040E251E4C701B6010E94F6
:10106000D1E84B015C010E94D3ED6B01770FEE08D4
:10107000FF08C701B6018DDFC701B6010E9472E803
:101080009B01AC01C501B4010E948EEC6B017C0197
:10109000C150F9F6CF91FF90EF90DF90CF90BF90C5
:1010A000AF909F908F9008958FB7F8949091DE0D38
:1010B0002091DD0D291759F0E92FF0E0E35AF24FA6
:1010C000208130E09F5F9F779093DE0D02C02FEF6D
:1010D0003FEF8FBFC90108951F920F920FB60F9275
:1010E00011240BB60F922F933F938F939F93EF93FF
:1010F000FF932091C6009FB7F894E091DD0D81E049
:101100008E0F8F773091DE0D831731F0F0E0E35AC8
:10111000F24F20838093DD0D9FBFFF91EF919F9150
:101120008F913F912F910F900BBE0F900FBE0F909C
:101130001F901895CF92DF92EF92FF92CF93DF939B
:10114000EC01C090E807D090E907E090EA07F09042
:10115000EB07A7019601688179818A819B810E94B2
:101160006CE887FF04C0C882D982EA82FB82C09003
:10117000EC07D090ED07E090EE07F090EF07A701A5
:1011800096016C817D818E819F810E946CE887FF32
:1011900004C0CC82DD82EE82FF82C090F007D09046
:1011A000F107E090F207F090F307A7019601688538
:1011B00079858A859B850E946CE887FF04C0C88674
:1011C000D986EA86FB86C0902502D0902602E09060
:1011D0002702F0902802A7019601688179818A810F
:1011E0009B810E94B5EE181624F4C882D982EA8247
:1011F000FB82C0902902D0902A02E0902B02F0904E
:101200002C02A70196016C817D818E819F810E94B5
:10121000B5EE181624F4CC82DD82EE82FF82C090F7
:101220002D02D0902E02E0902F02F0903002A70104
:101230009601688579858A859B850E94B5EE18168A
:1012400024F4C886D986EA86FB86DF91CF91FF9089
:10125000EF90DF90CF9008954F925F926F927F92C0
:101260008F929F92AF92BF92CF92DF92EF92FF92B6
:101270000F931F93CF93DF9300D000D0CDB7DEB78D
:101280007C01FC01E255F34C149182E0E816F10474
:1012900029F481E00E944DBC811123C16701CC0C6F
:1012A000DD1CCC0CDD1CC6018E55934C0E944749B9
:1012B0004B015C01612F110F770B880B990B0E947A
:1012C00072E82B013C0120E030E040EC5FE3C50117
:1012D000B4010E94D1E8A30192010E94D1E8AB01C0
:1012E000BC0100E010E09801C7010E9461BA92E0E1
:1012F000E916F10479F48EE99CE30E94474920E065
:1013000030E040EA50E40E946CE887FD09C08EE9B5
:101310009CE303C0C6018A56934C0E94474904C00F
:1013200060E070E080EA90E49B01AC01C301B2018F
:101330000E94D1E84B015C0120E030E0A9010E944D
:101340006CE8882309F458C000E010E09801B5016A
:10135000A4017058C7010E9461BA86E0E0E6F3E09C
:10136000DE01119601900D928A95E1F7F701EE0FDB
:10137000FF1F81E090E08C0F9D1FE80FF91F808117
:10138000918118161906C4F0E8EBF3E484918F01FB
:101390000F5F1F4F882319F08FDDF801F7CFE4E7C7
:1013A000FCE384918F010F5F1F4F882319F084DDC8
:1013B000F801F7CF8AE090E0BC01990F880B990BF8
:1013C0000E9472E89B01AC01F601EA59FC4F608172
:1013D0007181828193810E946BED2B013C01A501FB
:1013E0009401C501B4010E948FECAB01BC019301D3
:1013F0008201C7010E9461BA81E0F701E056FB4F0C
:101400008083F701E351FB4F8083F601EF5BF24FDE
:101410001082118212821382C7010E943FBEC60150
:101420008859934C0E944749860103501B4FF6018F
:10143000EB5CF24F20813181428153810E948FEC1D
:10144000F8016083718382839383F2E0EF16F104E5
:10145000D1F42091750E3091760E4091770E509117
:10146000780E6091050570910605809107059091B1
:1014700008050E948EEC6093050570930605809325
:101480000705909308050E943D49F601E35BF24F82
:10149000D601A350BB4F8D919D910D90BC91A02D75
:1014A00080839183A283B38382E0E816F104C9F4B8
:1014B00080E026960FB6F894DEBF0FBECDBFDF9159
:1014C000CF911F910F91FF90EF90DF90CF90BF9041
:1014D000AF909F908F907F906F905F904F900C9403
:1014E0004DBC26960FB6F894DEBF0FBECDBFDF9180
:1014F000CF911F910F91FF90EF90DF90CF90BF9011
:10150000AF909F908F907F906F905F904F900895D5
:101510000F931F93CF93DF938C01E8EBF3E4849157
:10152000EF012196882319F0C7DCFE01F8CFB8013E
:101530008BE59CE30E94558282E2BEDC8AE0BCDC43
:1015400081E0DF91CF911F910F9108955F9AEDEEA9
:10155000F4E010828A9A11829FB7F894A8E0B1E073
:101560008C9181608C939FBF1282129A08958C0196
:10157000E3E5F3E38491EF012196882319F09CDCE5
:10158000FE01F8CFEBE3FCE38491EF012196882381
:1015900019F092DCFE01F8CF0E9446D1D7DF0E94FD
:1015A000CD6B61E0C8010E9437D90E9447580E9464
:1015B0007B7484E00E943D5E8091FD108695869547
:1015C000109233118093341187E692E00E94285FD5
:1015D0008091FD1086958695880F10923311809327
:1015E00034118CE29CE30E941B5F8091FD10869574
:1015F0008695982F990F890F10923311809334118B
:101600008FE19CE30E941B5F0E9465C38111D1CFD3
:101610002FEF8BE49DE1215080409040E1F700C026
:101620000000F8942FEF84E39CE02150804090402C
:10163000E1F700C000000E9446D1A895FECF4F926E
:101640005F926F927F928F929F92AF92BF92CF9252
:10165000DF92EF92FF920F931F93CF93DF930E943D
:101660000D690E94D75B6B017C0110913A02112336
:1016700009F45FC08091290D90912A0D009709F41B
:1016800058C04091DF0D5091E00D6091E10D7091D7
:10169000E20D46015701841A950AA60AB70AB7FC5B
:1016A0005AC083309105F9F034F401970CF441C02D
:1016B000E8EBF3E406C0049709F03BC0E8EBF3E481
:1016C00026C08491EF012196882319F0F5DBFE01F5
:1016D000F8CFE1EAFBE38491EF012196882349F1F9
:1016E000EBDBFE01F8CFE8EBF3E48491EF01219608
:1016F000882319F0E1DBFE01F8CFEAE8FBE38491EF
:10170000EF0121968823A9F0D7DBFE01F8CF849161
:10171000EF012196882319F0CFDBFE01F8CFE2E735
:10172000FBE38491EF012196882319F0C5DBFE01CC
:10173000F8CF212F30E0A8EEB3E00E947FECC60E78
:10174000D71EE81EF91EC092DF0DD092E00DE09288
:10175000E10DF092E20D8091AF06843010F40E940A
:1017600087BF0E94D75BC090310DD090320DE090C2
:10177000330DF090340DC114D104E104F10459F19A
:1017800000912D0D10912E0D20912F0D3091300DC7
:101790000C0D1D1D2E1D3F1D5B016C01A01AB10A11
:1017A000C20AD30AD7FC17C0E3E5F3E38491EF0143
:1017B0002196882319F080DBFE01F8CF60912B0D74
:1017C00070912C0D85EE9BE30E9455828AE074DBBC
:1017D0008CED9BE355C0C0903B02D0903C02E09062
:1017E0003D02F0903E02C114D104E104F104D9F0AD
:1017F00000912D0D10912E0D20912F0D3091300D57
:101800000C0D1D1D2E1D3F1DDC01CB01801B910BFE
:10181000A20BB30BB7FD07C090915A1180915B11D9
:10182000981709F460C18091E70D9091E80D9099A7
:1018300002C0019604C0181619062CF40197909363
:10184000E80D8093E70D8091E70D9091E80D8E3EB5
:101850009240BCF0E3E5F3E38491EF012196882305
:1018600019F02ADBFE01F8CFECEBFBE38491EF01EA
:101870002196882319F020DBFE01F8CF83EB9BE350
:1018800076DE6091130890915A1180915B11981740
:1018900091F0E0915B118DE4E89FF0011124E5598E
:1018A000F74F608180915B1190915A11891719F05F
:1018B0008F5F8F70F9CF70E089E00E94D85A8091D5
:1018C000080E882309F4F9C000915B0210915C02B4
:1018D000D0915D02C0915E02609111087091120872
:1018E0006E5F7F4F072E000C880B990B0E9472E8E9
:1018F00098014D2F5C2F0E946CE887FDDEC0F090B0
:101900005B11912CA12CB12CE12C8DE4882E8091BF
:101910005A11F81609F45BC08F2D90E0889EF001F3
:10192000899EF00D1124EC5DF74F42815381648153
:101930007581452B462B472B81F446815781608565
:101940007185452B462B472B41F442855385648591
:101950007585452B462B472BA9F1889E9001899EC2
:10196000300D1124F901EC5DF74F6F016685778525
:10197000808991890E9472E82B013C01F6016289FD
:101980007389848995890E9470E89B01AC01C30129
:10199000B2010E946BEDF60123A134A145A156A12D
:1019A0000E94D1E83B016C019B01AC01692D7A2DAD
:1019B0008B2D9E2D0E946CE887FF04C0962CA72CCF
:1019C000BC2CED2C81E08F0D8F70F82EA0CF2091D4
:1019D0005302309154024091550250915602692DA4
:1019E0007A2D8B2D9E2D0E94D1E89B01AC01B80170
:1019F0008D2F9C2F0E948FEC6B017C0198014D2F45
:101A00005C2F0E946CE887FD14C000915702109172
:101A10005802D0915902C0915A0298014D2F5C2F63
:101A2000B601C7010E94B5EE18161CF08601DE2D26
:101A3000CF2DC090E30DD090E40DE090E50DF09037
:101A4000E60DA7019601B8018D2F9C2F0E946CE82E
:101A500087FF1CC020E037ED43EA5CE3B8018D2F1F
:101A60009C2F0E94D1E84B015C0128E431EE4AE74B
:101A70005FE3C701B6010E94D1E89B01AC01C5013B
:101A8000B4010E948FEC8B01D82FC92FC801AD2F54
:101A9000BC2F8093E30D9093E40DA093E50DB093DC
:101AA000E60DB8018D2F9C2F0E94D3ED7093120884
:101AB0006093110880E00E9413D10E9488D38CE5C6
:101AC00091E1DF91CF911F910F91FF90EF90DF9007
:101AD000CF90BF90AF909F908F907F906F905F90CE
:101AE0004F900C940E455F9A1092ED048A9A1092D2
:101AF000EE049FB7F89480910801816080930801FB
:101B00009FBF1092EF04129A8ECECF93DF9380E0A6
:101B100090E00E94C5D4CDE1DDE0688379838A83BB
:101B20009B8381E090E00E94C5D46C837D838E838B
:101B30009F8382E090E00E94C5D4688779878A8776
:101B40009B87DF91CF910895CF93DF930E944D49FA
:101B5000E091AE06F0E0E35FFA4F8081882371F0F8
:101B6000EFE6FBE38491EF012196882319F0A4D9D5
:101B7000FE01F8CF8AE0DF91CF919EC9DF91CF912E
:101B80000895CF93DF938FB7F8949091DE0D9093E3
:101B9000DD0D8FBFE6E6FBE38491EF0121968823FC
:101BA00019F08AD9FE01F8CF8091190D90911A0D84
:101BB000A0911B0DB0911C0DBC01CD016F5F7F4F3B
:101BC0008F4F9F4FE6D98AE077D9DF91CF91BCCF75
:101BD0003F924F925F926F927F928F929F92AF92BD
:101BE000BF92CF92DF92EF92FF920F931F93CF930A
:101BF000DF93CDB7DEB72C970FB6F894DEBF0FBEDC
:101C0000CDBF5C01DC0159968D909C905A97F401F0
:101C100081859285A385B4859C01AD012F5F3F4FDF
:101C20004F4F5F4F29873A874B875C87D5011496C2
:101C3000CD90DD90ED90FC901797C114D104E10494
:101C4000F10439F0BFEFCB1ADB0AEB0AFB0A312CA7
:101C500007C0F401C080D180E280F3803324339444
:101C6000260137011D821E821F821886F40181859C
:101C70009285A385B4852D813E814F815885281793
:101C800039074A075B0708F064C089859A85AB85E8
:101C9000BC858C159D05AE05BF0550F482E0C82EAD
:101CA000D12CE12CF12C92E0492E512C612C712C7D
:101CB0009E012F5F3F4FB701A601C4010E9484839C
:101CC000882309F446C089819A81AB81BC81892B24
:101CD0008A2B8B2B41F0260137019FEF491A590AB5
:101CE000690A790A05C0C414D504E604F70491F022
:101CF0002D813E814F8158852F5F3F4F4F4F5F4F62
:101D00002D833E834F8358873FEFC31AD30AE30ADC
:101D1000F30AACCF0FEF1FEF2FEF3FE0B301A201AB
:101D2000C4010E94F382F82E882399F0D5011496FD
:101D30004D915D916D917C9117974115510561050C
:101D4000710549F093018201C4010E94F38281115F
:101D500002C0F12C29C0D50114964D925D926D926E
:101D60007C921797332051F0D301C2010196A11D37
:101D7000B11DF40180839183A283B383F50185892A
:101D80009689A789B08D892B8A2B8B2B69F4D50175
:101D900055964D925D926D927C92589711968C91CA
:101DA0001197806811968C938F2D2C960FB6F8940E
:101DB000DEBF0FBECDBFDF91CF911F910F91FF907E
:101DC000EF90DF90CF90BF90AF909F908F907F90DB
:101DD0006F905F904F903F900895CF93DF93EC0109
:101DE0008B818823B9F1898187FF30C06C857D851F
:101DF0008E859F8541E00E94BB82882359F1E88946
:101E000080E2E89FF0011124DF01A551B14F109746
:101E100009F18C91853EF1F08B81823050F4498933
:101E20005A896B897C895C964D935D936D937C9305
:101E30005F978D899E89AF89B88DE551F14F938F5A
:101E4000828FB58BA48B89818F778983DF91CF9126
:101E50000C947B8281E0888380E0DF91CF910895AC
:101E60008F929F92AF92BF92CF92DF92EF92FF92AA
:101E70000F931F93CF93DF93EC018B81811102C0ED
:101E800080E077C009891A892B893C8904171507D6
:101E900026073707A8F36A017B01823029F4C88638
:101EA000D986EA86FB860DC0C114D104E104F10491
:101EB00051F41C821D821E821F82188619861A8682
:101EC0001B8681E056C088849984AA84BB84E98DEE
:101ED000FA8D258530E0275F3F4FB501A4014150C1
:101EE000510961097109022E04C0769567955795CD
:101EF00047950A94D2F7D701C6010197A109B10904
:101F000004C0B695A795979587952A95D2F784171B
:101F10009507A607B70720F089288A288B2849F457
:101F20004D895E896F89788D4C835D836E837F8355
:101F300004C0841B950BA60BB70B4C015D018E01F1
:101F40000C5F1F4F81149104A104B10409F4A7CFC1
:101F50004C815D816E817F819801898D9A8D0E946F
:101F6000848391E0891A9108A108B1088111EACF10
:101F700087CFDF91CF911F910F91FF90EF90DF906E
:101F8000CF90BF90AF909F908F9008952F923F92E7
:101F90004F925F926F927F928F929F92AF92BF9279
:101FA000CF92DF92EF92FF920F931F93CF93DF9325
:101FB00000D01F92CDB7DEB79C838B834B015A01B3
:101FC000DC0113968C91811103C08FEF9FEFEAC063
:101FD000EB81FC81818180FFF8CFAB81BC81519680
:101FE0000D911D912D913C91549718964D915D91B5
:101FF0006D917C911B97C501A0E0B0E0680179016B
:10200000C41AD50AE60AF70AC816D906EA06FB0674
:1020100018F45801A41AB50A75018B819C810496A5
:102020009A838983612C92E0792EE114F10409F4FA
:102030008BC0AB81BC8118964D915D916D917C9167
:102040001B976A01B1E0DB22EB81FC8123811A013D
:102050002B0189E056944794379427948A95D1F7B9
:10206000818D928D223061F4FC01828D938DA48D3F
:10207000B58DBC01CD01620D731D841D951D4AC037
:10208000DC0114961C9111501221C114D10401F5E8
:1020900011111EC0452B462B472B59F4EB81FC81B7
:1020A00085899689A789B08D84839583A683B78314
:1020B0000FC0AB81BC8114964D915D916D917C9167
:1020C000179729813A810E948483882309F47DCF60
:1020D000EB81FC81218D328D84819581A681B78130
:1020E0000297A109B109F901058404C0880F991F5D
:1020F000AA1FBB1F0A94D2F746855785608971894C
:10210000840F951FA61FB71FBC01CD01610F711D64
:10211000811D911D93012C193D0987012E153F0545
:1021200008F489010115F2E01F0771F52091EB1009
:102130003091EC104091ED105091EE106217730742
:102140008407950719F420C0C5012CC09401AB0188
:10215000BC018091F4109091F51057D6882309F4B2
:1021600034CF800E911EEB81FC8180859185A28504
:10217000B385800F911FA11DB11D80879187A28714
:10218000B387E01AF10A51CF40E00E94BB82882356
:1021900009F41BCFB6016551714FA801C4010E941B
:1021A000A1EFDFCF0F900F900F900F90DF91CF91A5
:1021B0001F910F91FF90EF90DF90CF90BF90AF9065
:1021C0009F908F907F906F905F904F903F902F9057
:1021D00008950F931F93CF93DF93FC012381222354
:1021E00011F080E044C08B01EC01FB018789803154
:1021F00039F18032B1F783E08B83F801428D538D42
:10220000648D758D4D8B5E8B6F8B788F9E012F5EED
:102210003F4FC8010E940584882319F31A8F098F44
:1022200081E089831C821D821E821F821886198686
:102230001A861B861C861D861E861F86188A17C056
:1022400082E08B831D8A1E8A1F8A188EFB01808D77
:10225000918DA0E0B0E025E0880F991FAA1FBB1F59
:102260002A95D1F7898B9A8BAB8BBC8BD7CFDF911B
:10227000CF911F910F9108950F931F93CF93DF93E9
:10228000EB01FC012381211102C080E040C02250FB
:10229000223028F48FE28883198281E038C08C01D3
:1022A000FC01648575858685978540E00E94BB8228
:1022B000882359F3F8014089F0E24F9FA0011124CF
:1022C0009A012551314F232B01F320E030E090E0BB
:1022D0006EE2F901E40FF51FE551F14F70817032A4
:1022E00071F02830310529F4DE01A90FB11D6C937E
:1022F0009F5FDE01A90FB11D70817C939F5F2F5FEF
:102300003F4F2B30310529F7C90FD11D1882DF91BE
:10231000CF911F910F910895CF93DF93EC015DDD75
:102320001B82DF91CF9108950F931F93CF93DF937B
:102330008B010E94D75BEB01F2D48F3F49F00E94E2
:10234000D75B6C1B7D0B60177107B0F380E001C099
:1023500081E0DF91CF911F910F9108950F931F930B
:10236000CF93DF93EC0189018C81833039F089E0D0
:10237000440F551F661F771F8A95D1F79A01AB014D
:1023800068E1CE01D3D4882311F086E02FC08EEF10
:102390008EBD80E090E00DB407FEFDCFF801E80FA0
:1023A000F91F20812EBD0DB407FEFDCF21812EBD6A
:1023B0000296811522E0920771F70DB407FEFDCF5A
:1023C0008FEFA8D48FEFA6D4AAD48B838F718530DA
:1023D00029F083E18983CE0198D409C068E572E0D1
:1023E000CE01A2DF182F811106C087E18983CE01BB
:1023F0008CD410E00FC020E030E0A9016DE0CE01E8
:1024000095D4811103C08BD4882311F086E1EECFDF
:10241000CE017BD4812FDF91CF911F910F91089531
:102420004F925F926F927F929F92AF92BF92CF92A4
:10243000DF92EF92FF920F931F93CF93DF931F9240
:10244000CDB7DEB78C017B016A01A22EDB01599664
:102450008D919C915A97F801928F818F40E050E0C6
:10246000BA01C701FDDC912CF70180859185A28519
:10247000B385418952896389748984179507A607B2
:10248000B70708F063C025E0B695A795979587959F
:102490002A95D1F7F82FFF70BF2ED70113968C9194
:1024A000823008F469C041E050E0BE016F5F7F4FA9
:1024B000C7016CDD019719F4898190E002C08FEFAC
:1024C0009FEF019609F458C0F70180859185A28598
:1024D000B3854F96A11DB11D80879187A287B387D1
:1024E000F0E2BF9EC0011124BC016551714F61151E
:1024F000710509F441C0DB012C91222319F0253E1E
:10250000D1F47CC191100EC04091EB105091EC10B1
:102510006091ED107091EE10F80144875587668741
:102520007787B08AFC01E551F14F8081882361F003
:102530009924939499CF4BE050E0C6010E9494EF08
:10254000892B09F091CF1AC0992493948A2D827413
:10255000823491F4992009F49CC0D8015096BC9023
:1025600050971C966D917D918D919C911F9741E0A4
:102570000E94BB82811180C080E043C1A7FCFCCFD8
:10258000F0E2BF9EA00111249A012551314FD901DB
:102590001B968C91817121F08A2D827109F068C09F
:1025A0008091EB109091EC10A091ED10B091EE1095
:1025B000F80184879587A687B787B08AFA01E55125
:1025C000F14F4489558960E070E0BA0155274427EE
:1025D000D80155964D935D936D937C935897828D5A
:1025E000938DA0E0B0E0482B592B6A2B7B2BD801B0
:1025F00055964D935D936D937C935897D9011B9697
:102600008C91887159F4848D958DA68DB78DF801C4
:10261000818B928BA38BB48B81E010C0803141F50C
:1026200098012F5E3F4FD80159968D919C915A97F2
:102630000E9405848823E1F084E0F80183838A2DD9
:102640008F70D80111968C931197F801148215821E
:102650001682178218961D921D921D921C921B972E
:10266000A4FEC0C0C8010E94BEC58111BBC084CFFA
:10267000D80113961C9280CFF8016089F0E26F9F19
:10268000B00111246551714F6115710509F08AC0BF
:1026900073CFD70113968C911397823009F46CCFC6
:1026A00051968D919D910D90BC91A02D803E9F4F94
:1026B000AF41B10508F060CFC7018ADA882309F479
:1026C0005BCF0E947B82882309F456CFD7015996AD
:1026D0002D913C915A9714968D919D910D90BC919E
:1026E000A02D0297A109B109F901058404C0880F42
:1026F000991FAA1FBB1F0A94D2F74684578460888B
:102700007188480E591E6A1E7B1E81E08093F3106B
:102710004092EB105092EC106092ED107092EE101F
:1027200080E092E0EBEEFEE0DF019C011D92215083
:102730003040E1F7BB24B394D7015996ED91FC9159
:102740005A978481B81690F42BEE3EE0B301A201B3
:102750004B0D511D611D711D8091F4109091F5106C
:10276000FDDD882309F408CFB394E6CF80E092E042
:10277000A0E0B0E0058404C0880F991FAA1FBB1F0A
:102780000A94D2F7F7014189528963897489840FC9
:10279000951FA61FB71F818B928BA38BB48B6BEEFB
:1027A0007EE0B12C80E2DB011D928A95E9F78BE097
:1027B000F601DB0101900D928A95E1F781E298E242
:1027C000FB01918B808B20E038E037872687938B45
:1027D000828B918F808F378B268B0E947B82811119
:1027E000CFCECACEA5FE08C0F801418952896389BF
:1027F0007489C80135DB05C081E003C0911098CE13
:1028000083CE0F90DF91CF911F910F91FF90EF90AA
:10281000DF90CF90BF90AF909F907F906F905F9030
:102820004F9008952F923F924F925F926F927F92B6
:102830008F929F92AF92BF92CF92DF92EF92FF92D0
:102840000F931F93CF93DF93CDB7DEB7C554D10954
:102850000FB6F894DEBF0FBECDBF3C015B018A010D
:10286000322E1C8E1F8E19821C82672B11F410E0F1
:10287000A7C0FC0183818111FACFFA0180818F32D8
:1028800061F4CA018C010196F80120812F32D1F345
:10289000F50183818250823010F475010AC0618D88
:1028A000728DCE01019695DC882309F3CE01019645
:1028B0007C016E019CE1C90ED11C26014E01E7E3AB
:1028C0008E0E911CFBE0F80D2596FFAF2597CE01EB
:1028D000019624969FAF8EAF24972696CFAE26976B
:1028E0002D2C35C080E2819325969FAD25979E13B0
:1028F000F9CFD80190E027E04A2F3B2F8D9181112D
:1029000028C08FA9803209F4B2CF842F932F8C0175
:10291000FC01208101962F32D1F3222309F44AC011
:1029200021E0A401B701C6017BDD882309F49FCF14
:10293000EA14FB0411F0C701EFDCC414D50499F1CB
:1029400026969FAD2697822D7601C92ED82EF401AA
:10295000C9CF8F32B1F28E3219F0E1EBFCE30AC03D
:102960002A3009F484CF98E02AE0C6CF3196381790
:1029700009F47DCF34913111F9CF291708F477CFBD
:10298000813208F474CF8F3709F471CF31E0390FF9
:10299000F401E90FF11D9FE9980F9A3108F4805274
:1029A0008083932FA9CF23969FAD239724968FAD35
:1029B0002497CACF232DA401B701C30131DD182FFD
:1029C000CE0101960E94A94FCE014C960E94A94FBC
:1029D000812FCB5BDF4F0FB6F894DEBF0FBECDBFAC
:1029E000DF91CF911F910F91FF90EF90DF90CF90EB
:1029F000BF90AF909F908F907F906F905F904F901F
:102A00003F902F9008952F923F924F925F926F9236
:102A10007F928F929F92AF92BF92CF92DF92EF926E
:102A2000FF920F931F93CF93DF9300D01F92CDB7E8
:102A3000DEB78C014B011A01DC0113968C911397C0
:102A40008130C1F411968C9181FF14C082FF18C0AF
:102A5000F801418952896389748980859185A285AD
:102A6000B38584179507A607B70751F0C801F8D9B1
:102A7000811106C081E0F80180838FEF9FEF2EC1A6
:102A8000610184C0D80159968D919C915A97FC019F
:102A9000248121502A013B0139E0769467945794B0
:102AA00047943A95D1F7722E74207A01F1E0FF2213
:102AB000772009F477C080E092E08E199F095601D3
:102AC0008C159D0508F45C01D80159962D913C9117
:102AD0005A9714968D919D910D90BC91A02D0297BF
:102AE000A109B109F901058404C0880F991FAA1F23
:102AF000BB1F0A94D2F74685578560897189840F78
:102B0000951FA61FB71F9C01AD01270D311D411D4B
:102B1000511D29013A01A11432E0B30609F089C020
:102B20008091EB109091EC10A091ED10B091EE100F
:102B300084159505A605B70569F41092F3108FEF7B
:102B40009FEFDC018093EB109093EC10A093ED10BD
:102B5000B093EE109401B301A2018091F410909112
:102B6000F510FCDB882309F485CFF8018085918579
:102B7000A285B3858A0D9B1DA11DB11D80879187FC
:102B8000A287B3878A0C9B1CCA18DB08D801189649
:102B90004D915D916D917C911B97C114D10409F009
:102BA00071CF7DC0E114F10409F085CF14964D91E9
:102BB0005D916D917C9117974115510561057105E6
:102BC00059F455968D919D910D90BC91A02D009733
:102BD000A105B10541F521C09E012F5F3F4F0E9425
:102BE0008483882309F446CF89819A81AB81BC8193
:102BF000F801218D328DF9012789203139F4883F80
:102C0000FFEF9F07A105B10540F40DC0883F2FEFEE
:102C10009207A2072FE0B20730F0C8010E94E88DAA
:102C2000811149CF27CFF80184839583A683B78389
:102C300042CFE114F10419F5D80118964D915D9138
:102C40006D917C911B9751968D919D910D90BC91AA
:102C5000A02D481759076A077B0788F00E947B82DE
:102C6000882309F407CF81E08093F3104092EB10A2
:102C70005092EC106092ED107092EE1008C041E09E
:102C8000C301B2010E94BB82882309F4F3CEA501DF
:102C9000B401C7018551914F0E94A1EF66CF5196B3
:102CA0008D919D910D90BC91A02D84179507A6073D
:102CB000B70740F4F801418B528B638B748B818191
:102CC00080688183D80111968C9183FD02C0C10177
:102CD00005C0C80182D88111FACFCCCE0F900F90D9
:102CE0000F900F90DF91CF911F910F91FF90EF9078
:102CF000DF90CF90BF90AF909F908F907F906F901C
:102D00005F904F903F902F90089561E0FC0180818B
:102D10000C946D5A8EBD0DB407FEFDCF08958FEF54
:102D20008EBD0DB407FEFDCF8EB50895CF92DF9214
:102D3000EF92FF921F93CF93DF9300D01F92CDB7F6
:102D4000DEB76C01162FFC019281892F806A86956F
:102D50008CBD90FD03C081E0963009F480E08DBD0C
:102D600060E0F601808129833A834B835C830E9473
:102D70006D5A6CE271E0C601D7DA812F8064CADF38
:102D800088E1E82EF12C5C814B813A812981DA01BE
:102D9000C9010E2C04C0B695A795979587950A94FE
:102DA000D2F729833A834B835C83B4DFF8E0EF1AD0
:102DB000F10829813A814B815C8188EFE8168FEF19
:102DC000F80629F7112321F0183021F08FEF03C006
:102DD00085E901C087E89EDF1C3009F4A0DF10E020
:102DE0009EDFF601838387FF04C01F3F11F01F5F42
:102DF000F7CF0F900F900F900F90DF91CF911F9111
:102E0000FF90EF90DF90CF900895EF92FF920F9395
:102E10001F93CF93DF93EC0179018C81833039F0DC
:102E200089E0440F551F661F771F8A95D1F79A01D5
:102E3000AB0161E1CE017ADF882329F084E0898348
:102E4000CE0163DF35C00E94D75B8B0168DF8B83C7
:102E50008F3F49F40E94D75B601B710B6D3271404C
:102E6000A8F381E103C08E3F39F08FE08983CE0162
:102E70004CDF8FEF4FDF1CC08FEF8EBDF701D70106
:102E8000A150BE4F0DB407FEFDCF9EB591938EBDF0
:102E9000EA17FB07B9F70DB407FEFDCF8EB58C938B
:102EA0003EDF3DDFCE0131DF8FEF34DF81E001C057
:102EB00080E0DF91CF911F910F91FF90EF900895E7
:102EC0008F929F92AF92BF92CF92DF92EF92FF923A
:102ED0000F931F93CF93DF9300D01F92CDB7DEB730
:102EE00089E3882E8EE0982E91E2A92E9EE0B92EDD
:102EF0000FEE1DE0C12CD12C7601C394F401619139
:102F00007191819191914F01F501219131914191FF
:102F100051915F0129833A834B835C830E9470E85F
:102F200029813A814B815C810E94D1E80E94D8EDD1
:102F3000F80161937193819391938F01C616D7061F
:102F4000E806F90610F46B017C01F9E48F16FEE047
:102F50009F06A1F66FEF7FEFCB01A70196010E94BC
:102F600031EC2093040E3093050E4093060E5093DF
:102F7000070E0F900F900F900F90DF91CF911F9140
:102F80000F91FF90EF90DF90CF90BF90AF909F9008
:102F90008F9008952F923F924F925F926F927F92FF
:102FA0008F929F92AF92BF92CF92DF92EF92FF9259
:102FB0000F931F93CF93DF9300D01F92CDB7DEB74F
:102FC0007B016A011901A1E2BEE02D913D914D9175
:102FD0005C91FC0160817181828193810E94D1E8C2
:102FE0000E94C0EE2B013C010AE411E1D8016D936F
:102FF0007D938D939C9313972091250E3091260EEF
:103000004091270E5091280EF701608171818281D5
:1030100093810E94D1E80E94C0EE4B015C01D8016F
:1030200014966D937D938D939C9317972091290E01
:1030300030912A0E40912B0E50912C0EF60160819A
:103040007181828193810E94D1E80E94C0EE6B0160
:103050007C01D80118966D937D938D939C931B975B
:1030600020912D0E30912E0E40912F0E5091300E4A
:10307000F10160817181828193810E94D1E80E9477
:10308000C0EED8011C966D937D938D939C931F97F2
:1030900069837A838B839C830E94E3D42FB7F8944F
:1030A000EBE1F4E1408251826282738284829582F4
:1030B000A682B782C086D186E286F38669817A814C
:1030C0008B819C8164877587868797872FBF109235
:1030D000361110923711109238111092391180E187
:1030E000EAE3F1E1DF011D928A95E9F70F900F9075
:1030F0000F900F90DF91CF911F910F91FF90EF9064
:10310000DF90CF90BF90AF909F908F907F906F9007
:103110005F904F903F902F9008950F931F93CF9300
:10312000DF93C1E2DEE001E115E029913991499197
:10313000599160E070E080E89FE30E946BEDF80138
:1031400061937193819391938F01FEE0C133DF0707
:1031500061F729E035E045E055E061E075E08DEF8D
:1031600094E018DFDF91CF911F910F91A9CE2F929C
:103170003F924F925F926F927F928F929F92AF9207
:10318000BF92CF92DF92EF92FF920F931F93CF9354
:10319000DF93CDB7DEB7C557D1090FB6F894DEBFC0
:1031A0000FBECDBF3B014A015901EFA6FBAA0BAFF1
:1031B00021961FAF21973C2C2091210E3091220E99
:1031C0004091230E5091240EDC016D917D918D91E3
:1031D0009C910E94D1E80E94C0EEAE966CAF7DAF8C
:1031E0008EAF9FAFAE972091250E3091260E409165
:1031F000270E5091280EF3016081718182819381A5
:103200000E94D1E80E94C0EEE2966CAF7DAF8EAF17
:103210009FAFE2972091290E30912A0E40912B0EFC
:1032200050912C0ED4016D917D918D919C910E94B5
:10323000D1E80E94C0EEE6966CAF7DAF8EAF9FAF37
:10324000E69720912D0E30912E0E40912F0E509129
:10325000300EF50160817181828193810E94D1E8F5
:103260000E94C0EE6A966CAF7DAF8EAF9FAF6A973B
:1032700080914A1190914B11A0914C11B0914D1138
:10328000AE96CCACDDACEEACFFACAE97C81AD90AAA
:10329000EA0AFB0A80914E1190914F11A0915011B2
:1032A000B0915111E2968CAC9DACAEACBFACE29744
:1032B000881A990AAA0ABB0A809152119091531157
:1032C000A0915411B0915511E6960CAD1DAD2EADE7
:1032D0003FADE697081B190B2A0B3B0B0FAB18AF42
:1032E00029AF3AAF8091EE0D83FF0EC06A962CADE8
:1032F0003DAD4EAD5FAD6A97209356113093571197
:103300004093581150935911809156119091571133
:10331000A0915811B09159116A964CAC5DAC6EAC4D
:103320007FAC6A97481A590A6A0A7B0A09F499C05D
:103330008091E90D811145C06091980470919904C4
:1033400080919A0490919B040E94D3ED072E000C6B
:10335000880B990B0E9472E820913F023091400245
:1033600040914102509142020E946CE887FF29C0BF
:103370006A968CAD9DADAEADBFAD6A978093561188
:1033800090935711A0935811B0935911E8EBF3E4BF
:1033900084918F010F5F1F4F882321F00E945C876B
:1033A000F801F6CFE0EEFCE384918F010F5F1F4F31
:1033B000882321F00E945C87F801F6CF412C512C24
:1033C00032014BA65CA66DA67EA677FE0BC0002739
:1033D0001127980104191509260937090BA71CA7FD
:1033E0002DA73EA760912D0E70912E0E80912F0E6D
:1033F0009091300E0E94D3ED9B01AC01A8ECB0E09F
:103400000E946FEC2BA53CA54DA55EA56217730726
:10341000840795074CF56A968CAD9DADAEADBFADFA
:103420006A978093561190935711A0935811B093B7
:103430005911E8EBF3E484918F010F5F1F4F88234C
:1034400021F00E945C87F801F6CFE1ECFCE3849167
:103450008F010F5F1F4F882321F00E945C87F801C6
:10346000F6CF412C512C3201D701C6018827B7FD78
:1034700083959927AA27BB27282EB7FE03C0E82FDC
:10348000E2602E2E0FA918AD29AD3AAD37FF03C06B
:10349000122D1460212E77FE03C0222D2860222ECB
:1034A000032D10E0C301B2010E9472E8F801EE0F93
:1034B000FF1FEE0FFF1FED5BFD4F20813181428129
:1034C00053810E94D1E82B013C01000F111FF8012C
:1034D000EF5DFD4F60817181072E000C880B990B09
:1034E0000E9472E89B01AC01C301B2010E94D1E8C5
:1034F0002AE037ED43E25CE30E94D1E82B013C0176
:1035000020E030E0A9010E94B5EE18164CF420E04E
:1035100030E040E05FE3C301B2010E948FEC08C0DD
:10352000A301920160E070E080E09FE30E948EECD6
:103530000E94D3ED6CAF7DAF8EAF9FAF80915A11DB
:103540008F5F8F706F968FAF6F9780915B116F96C3
:103550000FAD6F97801303C00E941F8BF6CFE091D1
:103560005A110E2F10E01CA70BA71DE4E19FF001DC
:103570001124EC5DF74F108222A2D701C601F7FE9D
:1035800007C088279927DC018C199D09AE09BF095E
:1035900082839383A483B5838DE40BA51CA5809FB0
:1035A000F001819FF00D1124EC5DF74FD501C401AE
:1035B000B7FE07C088279927DC0188199909AA094D
:1035C000BB0986839783A087B1878DE40BA51CA5D3
:1035D000809FF001819FF00D1124EC5DF74F8FA9C2
:1035E00098ADA9ADBAADB7FF07C0B095A0959095BD
:1035F00081959F4FAF4FBF4F82879387A487B58731
:103600008DE40BA51CA5809FF001819FF00D112476
:10361000EC5DF74F2CAD3DAD4EAD5FAD26873787E6
:10362000408B518B42815381648175810681178162
:1036300020853185041715072607370714F48A01FA
:103640009B018DE4ABA5BCA58A9FF0018B9FF00D7B
:103650001124EC5DF74F82859385A485B58580178D
:103660009107A207B30764F48CAD9DADAEADBFADBD
:1036700080179107A207B30764F4D901C8010DC0F0
:103680000CAD1DAD2EAD3FAD081719072A073B073E
:1036900024F08CAD9DADAEADBFAD2DE40BA51CA54A
:1036A000209FF001219FF00D1124EC5DF74F828BDC
:1036B000938BA48BB58B0697A105B10510F40C94E0
:1036C00058A5DF01A95BBF4F8091130890911408A2
:1036D0008D939C933182452B462B472B09F05F98A5
:1036E0008DE40BA51CA5809FF001819FF00D112496
:1036F000EC5DF74F86819781A085B185892B8A2B58
:103700008B2B09F08A988DE40BA51CA5809FF001F6
:10371000819FF00D1124EC5DF74F82859385A48580
:10372000B585892B8A2B8B2B41F09FB7F89480911C
:1037300008018E7F809308019FBF2CAD3DAD4EAD3B
:103740005FAD232B242B252B71F08091030E882352
:1037500019F081508093030E31100EC0129880E250
:103760008093030E09C02090490E30904A0E0091BC
:103770004B0E10914C0E08C020904D0E30904E0E06
:1037800000914F0E1091500E9101A8016FA57BA9D9
:103790008BAD21969FAD21970E946CE887FD02C0FA
:1037A0000C9450A5C701B6010E9472E82091110542
:1037B0003091120540911305509114050E94D1E8F3
:1037C0006FA778AB89AB9AAB698B7A8B8B8B9C8B11
:1037D000C501B4010E9472E82091150530911605CB
:1037E00040911705509118050E94D1E84B015C01EA
:1037F0006D8B7E8B8F8B988F6FA978AD89AD9AADCD
:103800000E9472E82091190530911A0540911B051C
:1038100050911C050E94D1E86B017C01698F7A8F61
:103820008B8F9C8F20911D0530911E0540911F05A7
:1038300050912005C301B2010E94D1E86D8F7E8FA7
:103840008F8F98A32DE44BA55CA5249FF001259FA5
:10385000F00D1124EC5DF74F428053806480758039
:1038600056E04516510461047104E4F44680578023
:1038700060847184A6E04A1651046104710494F4D2
:103880004284538464847584B6E04B165104610409
:10389000710444F4DC01CB01BF7787A790ABA1ABE7
:1038A000B2AB34C02FA538A949A95AA9CA01B90198
:1038B0000E94D1E82B013C01A5019401C501B4018E
:1038C0000E94D1E89B01AC01C301B2010E948FECC0
:1038D0004B015C01A7019601C701B6010E94D1E826
:1038E0009B01AC01C501B4010E948FEC0E94FAEE6D
